:020000040800F2
:100000000050002055500008594F0008614F00086B
:10001000694F0008714F0008794F00080000000088
:10002000000000000000000000000000814F0008F8
:100030008D4F000800000000994F0008A54F0008F0
:100040009D5000089D5000089D5000089D500008DC
:100050009D5000089D5000089D5000089D500008CC
:100060009D5000089D5000089D500008B54F0008A5
:100070009D5000089D5000089D5000089D500008AC
:100080009D5000089D5000089D5000089D5000089C
:10009000C94F00089D5000089D5000089D50000861
:1000A0009D5000089D5000089D5000089D5000087C
:1000B0009D5000089D5000089D5000089D5000086C
:1000C0009D5000089D5000089D5000089D5000085C
:1000D0009D5000089D5000089D5000089D5000084C
:1000E0009D5000089D5000089D5000080000000031
:1000F0000000000000000000000000000000000000
:0C01000000000000000000005FF808F1A3
:10010C0010B5054C237833B9044B13B10448AFF345
:10011C0000800123237010BDE001002000000000CE
:10012C0074ED000808B5034B1BB103490348AFF34A
:10013C00008008BD00000000E401002074ED000800
:10014C00034613F8012B002AFBD1181A013870470B
:10015C0080B400AF124B1B78DBB2002B1BD0104BC2
:10016C0000221A700F4B1B889AB20F4B1A800D4B42
:10017C005B889AB20D4B1A800A4B9B889AB20C4B37
:10018C001A80084BDB889AB20A4B1A80054B1B89E4
:10019C009AB2094B1A8000BFBD4680BC704700BFA5
:1001AC0029020020080200202A0200202C02002034
:1001BC002E020020300200203202002080B483B0D6
:1001CC0000AF0023FB7110E0FB79214A32F81330A9
:1001DC0099B2FB791F4A52F82320FB790A441D4936
:1001EC0041F82320FB790133FB71FB79042BEBD90C
:1001FC00194B1B780133DAB2174B1A70164B1B785C
:10020C00042B20D90023BB7114E0BB79114A52F89E
:10021C002330124AA2FB03239A08BB7991B2104AED
:10022C0022F81310BB790B4A002142F82310BB793A
:10023C000133BB71BB79042BE7D9074B00221A7031
:10024C00084B01221A7000BF0C37BD4680BC7047AA
:10025C00FC0100201402002028020020CDCCCCCCC4
:10026C00080200202902002080B582B000AF0346AE
:10027C003960FB71FB799BB201339BB2396818462C
:10028C0001F0D2F9034618460837BD4680BD80B54B
:10029C0082B000AF03460A46FB711346BB80FB7964
:1002AC009BB201339BB2BA881146184601F0D8F9BB
:1002BC00034618460837BD4680BD90B482B000AFE7
:1002CC000446084611461A462346FB710346BB7189
:1002DC000B467B7113463B71FB792F2B06D9FB79AF
:1002EC00392B03D8FB79303BFB710BE0FB79602B8E
:1002FC0006D9FB79662B03D8FB79573BFB7101E0E0
:10030C00002370E0BB792F2B06D9BB79392B03D88E
:10031C00BB79303BBB710BE0BB79602B06D9BB7949
:10032C00662B03D8BB79573BBB7101E000235AE025
:10033C007B792F2B06D97B79392B03D87B79303BF2
:10034C007B710BE07B79602B06D97B79662B03D80C
:10035C007B79573B7B7101E0002344E03B792F2BE9
:10036C0006D93B79392B03D83B79303B3B710BE0F9
:10037C003B79602B06D93B79662B03D83B79573BED
:10038C003B7101E000232EE0FB799AB23B691A80A5
:10039C003B691B881B019AB23B691A803B691A881E
:1003AC00BB799BB213449AB23B691A803B691B8898
:1003BC001B019AB23B691A803B691A887B799BB204
:1003CC0013449AB23B691A803B691B881B019AB291
:1003DC003B691A803B691A883B799BB213449AB2E9
:1003EC003B691A80012318460837BD4690BC7047FC
:1003FC002DE9F043C1B006AF0DF052FB0346002BC4
:10040C0000F0C8860DF060FBC7F8E000D7F8E030CC
:10041C00002BC0F2BE86BD4B1B781A46D7F8E030D5
:10042C00D9B2BB4B995400BFB84B1B781A46B84B8A
:10043C001344012118460DF009FC0346012BF3D09F
:10044C00D7F8E0300D2B04D0D7F8E0300A2B40F071
:10045C009986AE4B1B78002B00F09086AC4B1B782A
:10046C00493B242B00F2788601A252F823F000BFFE
:10047C00C706000865110008651100086511000821
:10048C006511000865110008651100086511000868
:10049C006511000865110008651100086511000858
:1004AC006511000865110008651100086511000848
:1004BC006511000865110008651100086511000838
:1004CC006511000865110008651100086511000828
:1004DC0065110008EB06000865110008651100089D
:1004EC00F509000865110008651100086511000880
:1004FC001105000865110008651100086511000858
:10050C00AD07000807F11003824918460DF07CFF77
:10051C0000BF07F11003052118460DF097FB0346A9
:10052C00012BF6D000217C4803F068FF0346984667
:10053C000421794803F062FF034699460821764866
:10054C0003F05CFF03461C460C21734803F056FF76
:10055C0003461D460021714803F050FF03461E461A
:10056C0004216E4803F04AFF03467B6008216B4868
:10057C0003F044FF03463B600C21684803F03EFF48
:10058C00034607F1100005933A6804927B680393C5
:10059C000296019500944B46424661490DF034FF9A
:1005AC0000BF07F110031846FFF7CAFD03469AB2C5
:1005BC0007F11003114618460DF048FB0346012BBA
:1005CC00EFD0554B1B685B6B7B60534B1B68996B77
:1005DC003960514B1B68DB6B4F4A1268126C4F49E8
:1005EC000968496B4D480068806B4C4C2468E46B7F
:1005FC004A4D2D682D6C07F1100605950494039057
:10060C000291019200933B687A68464930460DF09E
:10061C00FBFE00BF07F110031846FFF791FD0346E0
:10062C009AB207F11003114618460DF00FFB034662
:10063C00012BEFD03C4B1B781D463C4B1B881E46B8
:10064C003B4B1B881A463B4B1B8819463A4B1B8865
:10065C001C463A4B1B8807F110000393029401913E
:10066C00009233462A4636490DF0CEFE00BF07F104
:10067C0010031846FFF764FD03469AB207F1100306
:10068C00114618460DF0E2FA0346012BEFD02D4B24
:10069C001B781A462C4B1B7807F110002B490DF0D8
:1006AC00B3FE00BF07F110031F2118460DF0CEFA60
:1006BC000346012BF6D000F061BD07F1100324496D
:1006CC0018460DF0A1FE00BF07F1100309211846D2
:1006DC000DF0BCFA0346012BF6D000F04FBD0B4BCE
:1006EC001B78022B4AD10A4B5B78302B04D1194B67
:1006FC0000221A7000F042BD054B5B78312B2BD1D8
:10070C00144B01221A7000F039BD00BF34020020D6
:10071C00380200208CED0008180300206003002034
:10072C0094ED0008ACED0008F00300202A02002034
:10073C002C0200202E020020300200203202002069
:10074C00E0ED0008560400205404002018EE0008C8
:10075C0038EE00085804002007F110039B49184696
:10076C000DF052FE00BF07F11003052118460DF0E5
:10077C006DFA0346012BF6D000F000BD07F1100313
:10078C00924918460DF040FE00BF07F110030521F9
:10079C0018460DF05BFA0346012BF6D000F0EEBCC8
:1007AC008B4B1B78082B40F0FE808A4B5B78302BF0
:1007BC0040F2E880874B5B78342B00F2E380854B6A
:1007CC005B78303BDAB2834B5A70824B5B7887F89C
:1007DC00DF30804B9B78662B03D1002387F8E73002
:1007EC0019E07C4B9B78622B03D1012387F8E7300F
:1007FC0011E007F11003784918460DF005FE00BF13
:10080C0007F11003102118460DF020FA0346012BB6
:10081C00F6D000F0B3BC6F4BDB782F2B40F2A180ED
:10082C006C4BDB78392B00F29C806A4B1B792F2B9D
:10083C0040F29780674B1B79392B00F29280654B05
:10084C005B792F2B40F28D80624B5B79392B00F258
:10085C008880604B9B792F2B40F283805D4B9B797A
:10086C00392B7ED85B4BDB792F2B7AD9594BDB7923
:10087C00392B76D8574BDB78303BDAB2554BDA70E4
:10088C00544BDB7887F8DE30524B1B79303BDAB2B5
:10089C00504B1A714F4B1B7987F8DD304D4B5B7900
:1008AC00303BDAB24B4B5A714A4B5B7987F8DC30F0
:1008BC00484B9B79303BDAB2464B9A71454B9B794E
:1008CC0087F8DB30434BDB79303BDAB2414BDA71E2
:1008DC00404BDB7987F8DA3097F8DE309BB2FB813E
:1008EC00FB891A46920013445B009BB2FB8197F87C
:1008FC00DD309AB2FB8913449BB2FB81FB891A460B
:10090C00920013445B009BB2FB8197F8DC309AB2E7
:10091C00FB8913449BB2FB81FB891A46920013445A
:10092C005B009BB2FB8197F8DB309AB2FB891344D6
:10093C009BB2FB81FB891A46920013445B009BB26D
:10094C00FB8197F8DA309AB2FB8913449BB2FB8196
:10095C00FA8997F8E71097F8DF30184603F0C4FDD2
:10096C0032E007F110031D4918460DF04DFD00BF94
:10097C0007F11003132118460DF068F90346012BFB
:10098C00F6D021E007F11003154918460DF03CFD97
:10099C0000BF07F11003132118460DF057F9034659
:1009AC00012BF6D0EAE307F110030E4918460DF0BF
:1009BC002BFD00BF07F110030A2118460DF046F974
:1009CC000346012BF6D0D9E3D8E300BF44EE000870
:1009DC0034020020380200204CEE000860EE0008C3
:1009EC0080EE000894EE0008BB4B1B78012B40F204
:1009FC009B83BA4B5B78722B40F08680B64B1B788E
:100A0C00042B69D1B54B9A78B44BD97807F10C0308
:100A1C0000930B4630213020FFF74FFC0346002B90
:100A2C0042D0BB89DBB207F10E0211461846FFF724
:100A3C001BFC0346A7F8D830B7F8D830002B19D1D7
:100A4C00BB891A46FB8907F11000A5490DF0DCFCA7
:100A5C0000BF07F110031846FFF772FB03469AB26A
:100A6C0007F11003114618460DF0F0F80346012B60
:100A7C00EFD082E3B7F8D82007F110039949184654
:100A8C000DF0C2FC00BF07F110031846FFF758FB2E
:100A9C0003469AB207F11003114618460DF0D6F82A
:100AAC000346012BEFD068E307F110038E4918467B
:100ABC000DF0AAFC00BF07F110031846FFF740FB2E
:100ACC0003469AB207F11003114618460DF0BEF812
:100ADC000346012BEFD050E307F11003834918466E
:100AEC000DF092FC00BF07F110031846FFF728FB2E
:100AFC0003469AB207F11003114618460DF0A6F8FA
:100B0C000346012BEFD038E3744B5B78772B69D11C
:100B1C00714B1B78082B4DD1704B9A786F4BD97851
:100B2C0007F10C0300930B4630213020FFF7C5FB77
:100B3C000346002B37D0694B1879684B5979674BB2
:100B4C009A79664BDC7907F10E0300932346FFF785
:100B5C00B4FB0346002B1FD0BB89DBB2FA891146CC
:100B6C001846FFF794FB0346A7F8D830B7F8D830EF
:100B7C00002B08D1BB891A46FB8907F110005C4990
:100B8C000DF042FC1CE0B7F8D82007F110035949CE
:100B9C0018460DF039FC13E007F1100356491846BE
:100BAC000DF032FC0CE007F11003544918460DF01F
:100BBC002BFC05E007F11003514918460DF024FCFD
:100BCC0000BF07F110031846FFF7BAFA03469AB2B2
:100BDC0007F11003114618460DF038F80346012BA7
:100BEC00EFD0CAE23D4B5B78642B40F0A9803A4BC6
:100BFC001B78022B40F08C80002387F8E63046E00F
:100C0C0007F10E0297F8E63011461846FFF72CFB59
:100C1C000346A7F8D830B7F8D830002B19D197F87D
:100C2C00E620FB8907F1100036490DF0EDFB00BF03
:100C3C0007F110031846FFF783FA03469AB207F13F
:100C4C001003114618460DF001F80346012BEFD0A6
:100C5C0018E0B7F8D82007F110032B4918460DF00F
:100C6C00D3FB00BF07F110031846FFF769FA0346E0
:100C7C009AB207F11003114618460CF0E7FF034631
:100C8C00012BEFD097F8E630013387F8E63097F870
:100C9C00E6301F2BB4D997F8E63003F00303DBB230
:100CAC00002B40F06A8207F11003184918460DF02A
:100CBC00ABFB00BF07F110031846FFF741FA0346E0
:100CCC009AB207F11003114618460CF0BFFF034609
:100CDC00012BEFD051E200BF34020020380200207B
:100CEC00A0EE0008B4EE0008C8EE0008DCEE000828
:100CFC00E4EE0008F8EE00080CEF000824EF000802
:100D0C0038EF000844EF000854EF000860EF0008CB
:100D1C0007F110031D4918460DF076FB00BF07F1D3
:100D2C0010031846FFF70CFA03469AB207F11003AA
:100D3C00114618460CF08AFF0346012BEFD01CE23B
:100D4C00134B5B78782B29D1124B1B78022B04D1D7
:100D5C0000F0C0FC00F00CFD0FE207F110030E498F
:100D6C0018460DF051FB00BF07F110031846FFF7B2
:100D7C00E7F903469AB207F11003114618460CF036
:100D8C0065FF0346012BEFD0F7E100BF64EF0008CD
:100D9C0038020020340200206CEF0008B44B5B7862
:100DAC00762B40F04C81B34B1B78022B40F02F81FB
:100DBC00B14B1B889C46B14B1B889E46B04B1B8885
:100DCC001A46B04B1B881946AF4B1B881C46AF4BC1
:100DDC001B881D46AE4B1B881E46AE4B1B8807F16D
:100DEC0010000593049603950294019100927346AA
:100DFC006246A9490DF008FB00BF07F11003184625
:100E0C00FFF79EF903469AB207F1100311461846F4
:100E1C000CF01CFF0346012BEFD0A04B1B8819468E
:100E2C009F4B1B881C469F4B1B881A469E4B1B884E
:100E3C0007F110000193009223460A469B490DF0DE
:100E4C00E3FA00BF07F110031846FFF779F90346E0
:100E5C009AB207F11003114618460CF0F7FE034640
:100E6C00012BEFD0924B1B881A46924B1B8807F133
:100E7C00100091490DF0C8FA00BF07F11003184695
:100E8C00FFF75EF903469AB207F1100311461846B4
:100E9C000CF0DCFE0346012BEFD0884B1B88194667
:100EAC00874B1B881C46874B1B881A46864B1B8816
:100EBC0007F110000193009223460A4683490DF076
:100ECC00A3FA00BF07F110031846FFF739F90346E0
:100EDC009AB207F11003114618460CF0B7FE034600
:100EEC00012BEFD07A4B1B8819467A4B1B881C467A
:100EFC00794B1B881A46794B1B8807F1100001931C
:100F0C00009223460A4676490DF07EFA00BF07F19F
:100F1C0010031846FFF714F903469AB207F11003B1
:100F2C00114618460CF092FE0346012BEFD06D4B88
:100F3C001B8819466C4B1B881C466C4B1B881A462D
:100F4C006B4B1B8807F110000193009223460A4655
:100F5C0068490DF059FA00BF07F110031846FFF766
:100F6C00EFF803469AB207F11003114618460CF03D
:100F7C006DFE0346012BEFD05F4B1B8819465F4B70
:100F8C001B881C465E4B1B881A465E4B1B8807F160
:100F9C0010000193009223460A465B490DF034FA87
:100FAC0000BF07F110031846FFF7CAF803469AB2C0
:100FBC0007F11003114618460CF048FE0346012BAE
:100FCC00EFD0524B1B881946514B1B881C46514B7A
:100FDC001B881A46504B1B8807F110000193009296
:100FEC0023460A464D490DF00FFA00BF07F11003D6
:100FFC001846FFF7A5F803469AB207F110031146FD
:10100C0018460CF023FE0346012BEFD0B5E007F198
:10101C001003434918460DF0F7F900BF07F1100310
:10102C001846FFF78DF803469AB207F110031146E4
:10103C0018460CF00BFE0346012BEFD09DE007F198
:10104C001003384918460DF0DFF900BF07F1100303
:10105C001846FFF775F803469AB207F110031146CC
:10106C0018460CF0F3FD0346012BEFD085E000BFD2
:10107C00380200203402002000040020020400206A
:10108C000404002006040020080400200A040020A8
:10109C000C0400200E04002074EF00081004002043
:1010AC00120400201404002016040020D0EF0008C5
:1010BC00180400201E04002014F000082004002056
:1010CC002204002024040020260400202CF0000818
:1010DC00280400202A040020380400203A040020B0
:1010EC0060F000082C0400202E0400203C0400209A
:1010FC003E04002094F0000830040020320400204C
:10110C004004002042040020C8F0000834040020F1
:10111C00360400204404002046040020FCF00008A3
:10112C0030F1000838F1000807F110031B4918468C
:10113C000DF06AF900BF07F110031846FFF700F82D
:10114C0003469AB207F11003114618460CF07EFDC7
:10115C000346012BEFD010E007F11003104918469D
:10116C000DF052F900BF07F11003022118460CF0E4
:10117C006DFD0346012BF6D000E000BF094B0022A9
:10118C001A7007E0074B1B780133DAB2054B1A7063
:10119C0000E000BFEC37BD46BDE8F08348F1000825
:1011AC005CF100083402002080B59AB000AF2F4BE0
:1011BC001A782F4B1B789A4217D02D4B1A782B4B41
:1011CC001A702B4B1B781A463B1D2A4918460DF0FA
:1011DC001BF93B1D1846FEF7B3FF03469AB2391DA7
:1011EC004FF0FF33244808F01FFB244B1A88244B84
:1011FC001B889A4217D0224B1A88204B1A80204BFE
:10120C001B881A463B1D1F4918460DF0FDF83B1D67
:10121C001846FEF795FF03469AB2391D4FF0FF337F
:10122C00154808F001FB184B1A78184B1B789A429A
:10123C0017D0164B1A78144B1A70144B1B781A468D
:10124C003B1D134918460DF0DFF83B1D1846FEF701
:10125C0077FF03469AB2391D4FF0FF33064808F06A
:10126C00E3FA00BF6837BD4680BD00BF9C0200207A
:10127C00F003002060F10008A80300209E0200206B
:10128C005404002070F10008A00200205604002035
:10129C0080F1000880B582B000AF03460A46FB71AE
:1012AC001346BB80FB799BB201339BB2BA881146C3
:1012BC00184600F0D5F9034618460837BD4680BDE0
:1012CC0080B483B000AF78607B681B889BB21846F3
:1012DC000C37BD4680BC7047B0B584B000AF7860A9
:1012EC000B467B8004F076FE7B8800221C4615465C
:1012FC0022462B467968012004F0FCFD0346FB7363
:10130C0004F08EFEFB7B18461037BD46B0BD80B591
:10131C0088B000AF78600023BB6004F05BFE002354
:10132C00FB607B687B610123BB6107F1080207F15D
:10133C000C031146184604F035FF0346FB7704F006
:10134C006FFEFB7F18462037BD4680BD80B487B04A
:10135C0000AF78607B6802337B617B6803F5806348
:10136C003B610CE07B691B88FB81FB894FF6FF72AC
:10137C00934201D17B6908E07B6904337B613B6953
:10138C00033B7A699A42EDD3002318461C37BD46BD
:10139C0080BC704780B489B000AFF8600B467A60AF
:1013AC007B81FB680233FB61FB6803F580637B6127
:1013BC000223FB7600233B837B68002B18D101238F
:1013CC0024E0FB691B887B827B8A4FF6FF72934279
:1013DC0014D0FB6902331B883B827A8A7B899A4240
:1013EC0003D13B8A3B830023FB76FB690433FB610F
:1013FC007B69043BFA699A42E3D900E000BFFB7EAB
:10140C00002B02D17B683A8B1A80FB7E184624375E
:10141C00BD4680BC7047000080B500AF0F48FFF799
:10142C0076FF0346002B01D0012315E00C48FFF793
:10143C006EFF0346002B01D001230DE04AF6AA21D2
:10144C000648FFF749FF0346002B01D0012303E0B8
:10145C00044B024A1A600023184680BD00F80008AD
:10146C0000FC00080000002080B483B000AF78605E
:10147C007B68054A934201D1044B00E0024B1846AD
:10148C000C37BD4680BC704700F8000800FC000813
:10149C0080B588B000AF03460A46FB801346BB807C
:1014AC003C4B1B687B617869FFF7DEFF386138695C
:1014BC00FFF72DFF0346002B01D0012365E045F219
:1014CC0055513869FFF708FF0346002B01D0012363
:1014DC005BE03B690233FB6100237B833CE07B8B4D
:1014EC002D4A32F81330FB81FA89FB889A4202D1DB
:1014FC00BB887B810BE007F10A02FB8919467869EE
:10150C00FFF748FF03467B737B7B002B20D1FB89C5
:10151C001946F869FFF7E0FE0346002B01D00123C2
:10152C0033E0FB6902337A8911461846FFF7D4FE83
:10153C000346002B01D0012327E0FB690433FB6138
:10154C003B6903F58063FA699A4202D303231CE0DA
:10155C0000BF7B8B01337B837B8B3F2BBFD978699F
:10156C00FFF7D5FE0346002B01D001230DE04AF610
:10157C00AA213869FFF7B0FE0346002B01D00123E6
:10158C0003E0044A3B691360002318462037BD462C
:10159C0080BD00BF0000002098F4000880B582B028
:1015AC0000AF1E48FFF78CFE0346FB801C48FFF77C
:1015BC0087FE0346BB80FB884FF6FF72934208D12F
:1015CC00BB884FF6FF72934203D1FFF725FF03460A
:1015DC0020E0FB884AF6AA22934209D1BB884FF639
:1015EC00FF72934204D10F4B0C4A1A60002311E096
:1015FC00BB884AF6AA22934209D1FB884FF6FF72A8
:10160C00934204D1074B064A1A60002302E0FFF70D
:10161C0003FF034618460837BD4680BD00F8000896
:10162C0000FC00080000002080B584B000AF034629
:10163C003960FB803B68002B01D101230AE0074B8A
:10164C001B68F9883A681846FFF7A4FE0346FB733B
:10165C00FB7B9BB218461037BD4680BD00000020B6
:10166C0080B584B000AF03460A46FB801346BB80AE
:10167C00174B1B681846FFF769FEF860FB68002BD8
:10168C0017D0FB881946F868FFF726FE0346002B97
:10169C0001D0012317E0FB680233BA8811461846C3
:1016AC00FFF71AFE0346002B01D001230BE00023A9
:1016BC0009E0BA88FB8811461846FFF7E9FE034695
:1016CC00FB72FB7A9BB218461037BD4680BD00BF3B
:1016DC000000002080B59AB000AF002387F8673077
:1016EC0035E097F867301E4A32F8132097F86730C8
:1016FC0011461846FFF7CEFD0346A7F86430B7F83D
:10170C006430002B0BD197F8672097F86730144999
:10171C0031F81330384613490CF076FE06E0B7F872
:10172C0064203B46104918460CF06EFE3B461846AA
:10173C00FEF706FD03469AB239464FF0FF330B48CD
:10174C0008F072F897F86730013387F8673097F82C
:10175C0067303F2BC5D900BF00BF6837BD4680BD81
:10176C0018F400088CF1000898F10008A803002078
:10177C00F0B5B9B006AF2822A94B1A803C22A94B70
:10178C001A804622A84B1A804622A84B1A80232284
:10179C00A74B1A802822A74B1A802822A64B1A8006
:1017AC002822A64B1A801422A54B1A801422A44B73
:1017BC005A801422A24B9A801422A14BDA80E62282
:1017CC00A04B1A806422A04B1A8082229F4B1A8055
:1017DC004FF496729E4B1A804FF4FA729D4B1A80FE
:1017EC0014229D4B1A803C229C4B1A8046229C4B07
:1017FC001A8028229B4B1A8028229B4B1A8032225B
:10180C009A4B1A800A229A4B1A804FF49B72994B6E
:10181C001A804FF4E172984B1A801E22974B1A8053
:10182C004FF49B72964B1A804FF4AA72954B1A8008
:10183C004FF4D772944B1A801E22944B1A804FF49B
:10184C00D772934B1A800A22924B1A804FF4A072D3
:10185C00914B1A808C22914B1A808C22904B1A80BF
:10186C001422904B1A804FF48C728F4B1A802822C2
:10187C008E4B1A804FF4DC728D4B1A8005228D4BE7
:10188C001A803B468C4918460CF0BEFD3B46184668
:10189C00FEF756FC03469AB239464FF0FF338748A1
:1018AC0007F0C2FF5E4B1B889C465E4B1B889E4616
:1018BC005D4B1B881A465D4B1B8819465C4B1B887D
:1018CC001C465C4B1B881D465B4B1B881E465B4BAA
:1018DC001B88384605930496039502940191009257
:1018EC007346624676490CF08FFD3B461846FEF770
:1018FC0027FC03469AB239464FF0FF336F4807F086
:10190C0093FF504B1B8819464F4B1B881C464F4B63
:10191C001B881A464E4B1B8838460193009223466F
:10192C000A4668490CF070FD3B461846FEF708FC69
:10193C0003469AB239464FF0FF33604807F074FF04
:10194C004B4B1B881A46494B1B8838465E490CF09A
:10195C005BFD3B461846FEF7F3FB03469AB239464D
:10196C004FF0FF33554807F05FFF3C4B1B8819467F
:10197C003B4B1B881C463B4B1B881A463A4B1B881F
:10198C0038460193009223460A4650490CF03CFD20
:10199C003B461846FEF7D4FB03469AB239464FF045
:1019AC00FF33464807F040FF324B1B881946324B39
:1019BC001B881C46374B1B881A46374B1B883846EE
:1019CC000193009223460A4641490CF01DFD3B460B
:1019DC001846FEF7B5FB03469AB239464FF0FF3373
:1019EC00364807F021FF254B1B881946244B1B88D2
:1019FC001C462A4B1B881A46294B1B8838460193D8
:101A0C00009223460A4633490CF0FEFC3B4618462E
:101A1C00FEF796FB03469AB239464FF0FF335BE074
:101A2C00000400200204002004040020060400200E
:101A3C00080400200A0400200C0400200E040020DE
:101A4C004C04002010040020120400201404002078
:101A5C00160400201C0400201A040020200400207E
:101A6C002204002024040020260400201E04002050
:101A7C0018040020280400202A0400202C04002034
:101A8C002E040020300400203204002034040020F6
:101A9C0036040020380400203A0400203C040020C6
:101AAC003E04002040040020420400204404002096
:101ABC004604002048040020ACF10008A8030020D4
:101ACC00B4F1000810F2000854F200086CF200089F
:101ADC00A0F20008D4F20008224807F0A5FE224B21
:101AEC001B881946214B1B881C46214B1B881A4608
:101AFC00204B1B8838460193009223460A461E4908
:101B0C000CF082FC3B461846FEF71AFB03469AB2D1
:101B1C0039464FF0FF33134807F086FE174B1B88EE
:101B2C001946174B1B881C46164B1B881A46164B1E
:101B3C001B8838460193009223460A4613490CF041
:101B4C0063FC3B461846FEF7FBFA03469AB239464D
:101B5C004FF0FF33034807F067FE00BFCC37BD469C
:101B6C00F0BD00BFA8030020300400203204002088
:101B7C00400400204204002008F300083404002034
:101B8C003604002044040020460400203CF30008E6
:101B9C0080B582B000AF7C4B1B780133DAB27A4B44
:101BAC001A70794B1B78092B40F2E781764B002297
:101BBC001A70764B1B78DBB2002B06D0734B1B785C
:101BCC00DBB2013BDAB2714B1A70714B1B78DBB292
:101BDC00002B06D06E4B1B78DBB2013BDAB26C4BA0
:101BEC001A706C4B1B78DBB2002B06D0694B1B7840
:101BFC00DBB2013BDAB2674B1A70674B1B780133CF
:101C0C00DAB2654B1A70644B1B7803F00303DAB23B
:101C1C00614B1A704FF48041604804F0EFFC0346AE
:101C2C00002B0CD15C4B1B781A465D4B9B5C5A4AC3
:101C3C00127843F00103D9B2594B99540BE0564B2F
:101C4C001B781A46564B9B5C534A127823F00103BF
:101C5C00D9B2534B99544FF40041504804F0CEFC88
:101C6C000346002B0CD14C4B1B781A464C4B9B5CFF
:101C7C00494A127843F00203D9B2494B99540BE00C
:101C8C00454B1B781A46464B9B5C434A127823F013
:101C9C000203D9B2424B99544FF48051414804F09D
:101CAC00ADFC0346002B0CD13B4B1B781A463C4B2E
:101CBC009B5C394A127843F00403D9B2384B9954DF
:101CCC000BE0354B1B781A46354B9B5C324A12782D
:101CDC0023F00403D9B2324B99544FF400513148DC
:101CEC0004F08CFC0346002B0CD12B4B1B781A46B2
:101CFC002B4B9B5C284A127843F00803D9B2284B33
:101D0C0099540BE0244B1B781A46254B9B5C224ABA
:101D1C00127823F00803D9B2214B99544FF4804127
:101D2C00204804F06BFC0346002B0CD11A4B1B789B
:101D3C001A461B4B9B5C184A127843F01003D9B21D
:101D4C00174B99540BE0144B1B781A46144B9B5CA5
:101D5C00114A127823F01003D9B2114B99544FF455
:101D6C000041104804F04AFC0346002B1CD10A4BDE
:101D7C001B781A460A4B9B5C074A127843F02003E7
:101D8C00D9B2074B99541BE05A04002004000020E0
:101D9C0005000020060000205B040020001001401C
:101DAC005C040020000C0140764B1B781A46764BE5
:101DBC009B5C744A127823F02003D9B2724B99546D
:101DCC00714B1A78704B5B781340DAB26E4B9B7880
:101DDC001340DAB26C4BDB781340DAB26B4B1B78E6
:101DEC001343DAB2694B1A70674B1A78664B5B78FF
:101DFC001343DAB2644B9B781343DAB2624BDB7851
:101E0C001343DAB2614B1B781340DAB25F4B1A7092
:101E1C00FEF7D4F95E4B1B780133DAB25C4B1A70C7
:101E2C005B4B1B78092B40F2A880594B00221A708F
:101E3C000023FB7113E0FB79564A32F813309BB246
:101E4C00002B09D0FB79534A32F8132092B2013A95
:101E5C0091B2504A22F81310FB790133FB71FB79D4
:101E6C00032BE8D94C4B1B889BB24FF6FF72934265
:101E7C0006D0494B1B889BB201339AB2464B1A8051
:101E8C00464B1B889BB2002B06D0444B1B889BB245
:101E9C00013B9AB2414B1A80414B1B78DBB2012BB0
:101EAC0027D1404B1B78002B11D03F4B1B78042BB8
:101EBC0006D900224FF400513C4804F0B6FB4FE029
:101ECC0001224FF40051394804F0AFFB48E0364B87
:101EDC001B78042B06D900224FF48071344804F08F
:101EEC00A4FB3DE001224FF48071314804F09DFBCE
:101EFC0036E02B4B1B78DBB2022B2BD1294B1B78FA
:101F0C00002B13D0284B1B7803F00103002B06D0B9
:101F1C0000224FF40051254804F087FB20E00122F9
:101F2C004FF40051214804F080FB19E01E4B1B7844
:101F3C0003F00103002B06D000224FF480711C48E3
:101F4C0004F073FB0CE001224FF48071184804F08C
:101F5C006CFB05E000224FF48071154804F065FB22
:101F6C00114B1B780133DAB20F4B1A700E4B1B78E6
:101F7C00092B02D90C4B00221A7000BF0837BD4642
:101F8C0080BD00BF5B0400205C040020F003002037
:101F9C0060040020F4030020FC030020FE0300205A
:101FAC005704002058040020610400200010014058
:101FBC000008014080B500AFAC4B1B7803F0010367
:101FCC00002B13D0AA4B1B78DBB2002B07D1A94BEB
:101FDC001B8843F001039AB2A64B1A8036E001220B
:101FEC004FF40051A44804F020FB2FE0A14B1B88B8
:101FFC0003F00103002B14D09E4B1B8823F001032C
:10200C009AB29C4B1A809B4B1B8843F480539AB218
:10201C00984B1A8000224FF40051974804F005FBAE
:10202C0011E0934B1B78DBB2BE2B0CD8914B1B8869
:10203C0043F002039AB28F4B1A8000224FF40051E6
:10204C008D4804F0F2FA8A4BC8221A70874B1B7821
:10205C0003F00203002B0CD0884B1B78DBB2002B57
:10206C0024D1844B1B8843F004039AB2814B1A8011
:10207C001CE0804B1B8803F00403002B07D07D4B26
:10208C001B8823F004039AB27A4B1A800BE07B4B2B
:10209C001B78DBB2BE2B06D8764B1B8843F00803AB
:1020AC009AB2744B1A80754BC8221A70714B1A88ED
:1020BC0041F20F0313409AB26E4B1A806D4B1B8882
:1020CC00002B40F0E080694B1B7803F03C03302B75
:1020DC0000F2BB8001A252F823F000BFAD21000832
:1020EC00572200085722000857220008092200082E
:1020FC00572200085722000857220008BB2100086D
:10210C005722000857220008572200083D220008D9
:10211C00572200085722000857220008D521000832
:10212C00572200085722000857220008572200089F
:10213C00572200085722000857220008572200088F
:10214C00572200085722000857220008572200087F
:10215C00572200085722000857220008EF210008D8
:10216C00572200085722000857220008572200085F
:10217C00572200085722000857220008572200084F
:10218C00572200085722000857220008572200083F
:10219C005722000857220008572200082322000863
:1021AC00374B64221A70334B00221A806BE0344B8D
:1021BC001B78DBB2002B4FD12E4B1B8843F0100346
:1021CC009AB22C4B1A8047E02D4B1B78DBB2002BBC
:1021DC0044D1284B1B8843F020039AB2254B1A801C
:1021EC003CE0274B1B78DBB2002B39D1214B1B88F1
:1021FC0043F480739AB21F4B1A8031E0204B1B784A
:10220C00DBB2002B2ED11B4B1B8843F400739AB20C
:10221C00184B1A8026E01A4B1B78DBB2002B23D10B
:10222C00144B1B8843F480639AB2124B1A801BE048
:10223C00134B1B78DBB2002B24D10E4B1B8843F4C1
:10224C0000639AB20B4B1A801CE00D4B64221A707F
:10225C00084B00221A8016E000BF14E000BF12E009
:10226C0000BF10E000BF0EE000BF0CE0F003002048
:10227C000400002054040020001001400500002040
:10228C000600002000BF00BF80BD00BF80B584B039
:10229C0002AF9D4B1B78192B00F2948601A252F8C9
:1022AC0023F000BF19230008EB2300083524000895
:1022BC007F240008C9240008512500089B2500082C
:1022CC00E52500082F26000879260008C3260008FB
:1022DC000D27000857270008C52700080D280008FF
:1022EC00552800089D280008E52800084D290008FD
:1022FC00DD290008792A0008932E0008E32A00083B
:10230C00A32D0008332E0008FB2E00087F4B1B88E2
:10231C0023F480539AB27D4B1A807C4B1B8803F0BC
:10232C000103002B14D07A4B02221A70794B002235
:10233C001A80754B12221A70774B00221A7001F01A
:10234C00C7F901F097FA01F067FB01F039FC0BE0DB
:10235C006E4B1B8803F00203002B05D06E4B002242
:10236C001A70694B13221A706B4B00221A706B4B4C
:10237C001A886B4B1B889A4223D9674B1B7883F0C6
:10238C000103DBB2002B1CD001224FF40041654845
:10239C0004F04BF9644B1B889BB2002B1DD15D4B99
:1023AC0000221A805A4B01221A70574B18221A70AD
:1023BC0001F0DAFC01F0AAFD01F07AFE01F04CFF0D
:1023CC000BE000224FF40041564804F02EF9574B15
:1023DC001A88554B1A8000F0F5BD00F0F3BD544B34
:1023EC001B88DAB2534B1B88D9B2534B1B88DBB218
:1023FC000A20019000930B460021012002F066FB9D
:10240C00444B1B889AB24D4B1B889A4202D33E4BCD
:10241C0011221A704A4B1B78002B40F0A2853A4BC4
:10242C0002221A7000F09DBD414B1B88DAB2414B61
:10243C001B88D9B2404B1B88DBB20A200190009359
:10244C000B460021012002F041FB324B1B889AB253
:10245C003A4B1B889A4202D32B4B11221A70384BE1
:10246C001B78002B00F07F85274B11221A7000F08F
:10247C007ABD2F4B1B88DAB22E4B1B88D9B22E4B50
:10248C001B88DBB20A20019000930B46012101202E
:10249C0002F01CFB1F4B1B889AB2284B1B889A42DC
:1024AC0002D3194B11221A70254B1B78002B40F0CC
:1024BC005C85154B04221A7000F057BD1C4B1B8811
:1024CC00DAB21C4B1B88D9B21B4B1B88DBB20A201F
:1024DC00019000930B460121012002F0F7FA0D4BFD
:1024EC001B889AB2154B1B889A4202D3064B1122B9
:1024FC001A70134B1B78002B00F03985024B1122FC
:10250C001A7000F034BD00BF5604002054040020A3
:10251C0057040020FC030020590400203202002044
:10252C001C04002000080140FE0300201A040020B7
:10253C004C040020200400201E0400201004002065
:10254C00F0030020934B5B88DAB2934B1B88D9B213
:10255C00924B1B88DBB20A20019000930B460021A2
:10256C00022002F0B3FA8E4B1B889AB28D4B1B885B
:10257C009A4202D38C4B11221A708C4B1B78002B75
:10258C0040F0F784884B06221A7000F0F2BC814BA5
:10259C005B88DAB2804B1B88D9B2804B1B88DBB2CC
:1025AC000A20019000930B460021022002F08EFAC3
:1025BC007B4B1B889AB27B4B1B889A4202D37A4B7B
:1025CC0011221A70794B1B78002B00F0D484764BB7
:1025DC0011221A7000F0CFBC6E4B5B88DAB26E4BD6
:1025EC001B88D9B26D4B1B88DBB20A20019000937B
:1025FC000B460121022002F069FA694B1B889AB242
:10260C00684B1B889A4202D3674B11221A70674B96
:10261C001B78002B40F0B184634B08221A7000F039
:10262C00ACBC5C4B5B88DAB25B4B1B88D9B25B4BA6
:10263C001B88DBB20A20019000930B46012102207B
:10264C0002F044FA564B1B889AB2564B1B889A429E
:10265C0002D3554B11221A70544B1B78002B00F0EF
:10266C008E84514B11221A7000F089BC494B9B8807
:10267C00DAB24F4B1B88D9B2484B1B88DBB20A200D
:10268C00019000930B460021032002F01FFA444BEB
:10269C001B889AB2474B1B889A4202D3424B112299
:1026AC001A70424B1B78002B40F06B843E4B0A2275
:1026BC001A7000F066BC374B9B88DAB23C4B1B8817
:1026CC00D9B2364B1B88DBB20A20019000930B4623
:1026DC000021032002F0FAF9314B1B889AB2354BDA
:1026EC001B889A4202D3304B11221A702F4B1B7845
:1026FC00002B00F048842C4B11221A7000F043BCC4
:10270C00244B9B88DAB22A4B1B88D9B2234B1B88EB
:10271C00DBB20A20019000930B460121032002F04A
:10272C00D5F91F4B1B889AB2224B1B889A4202D3B5
:10273C001D4B11221A701D4B1B78002B40F0258469
:10274C00194B0C221A7000F020BC124B9B88DAB289
:10275C00174B1B88D9B2114B1B88DBB20A20019096
:10276C0000930B460121032002F0B0F90C4B1B889F
:10277C009AB2104B1B889A4202D30B4B11221A703F
:10278C000A4B1B78002B00F00284074B11221A70A5
:10279C00FDE300BF4C040020220400201E04002096
:1027AC00FC0300201204002056040020F00300203B
:1027BC002404002014040020A34BDB88DAB2A34BC2
:1027CC001B88D9B2A24B1B88DBB20A200190009364
:1027DC000B460021042002F079F99E4B1B889AB21B
:1027EC009D4B1B889A4202D39C4B11221A709C4B16
:1027FC001B78002B40F0CD83984B0E221A70C8E347
:10280C00914BDB88DAB2914B1B88D9B2904B1B8869
:10281C00DBB20A20019000930B460021042002F049
:10282C0055F98C4B1B889AB28B4B1B889A4202D35E
:10283C008A4B11221A708A4B1B78002B00F0AB8349
:10284C00864B11221A70A6E37F4BDB88DAB27F4BE2
:10285C001B88D9B27E4B1B88DBB20A2001900093F7
:10286C000B460121042002F031F97A4B1B889AB2F5
:10287C00794B1B889A4202D3784B11221A70784BF1
:10288C001B78002B40F08983744B10221A7084E360
:10289C006D4BDB88DAB26D4B1B88D9B26C4B1B8845
:1028AC00DBB20A20019000930B460121042002F0B8
:1028BC000DF9684B1B889AB2674B1B889A4202D35E
:1028CC00664B11221A70664B1B78002B00F0678345
:1028DC00624B11221A7062E300220021012001F0E8
:1028EC0075FF00220021022001F070FF0022002160
:1028FC00032001F06BFF00220021042001F066FF91
:10290C0000220121012001F061FF0022012102209F
:10291C0001F05CFF00220121032001F057FF00228F
:10292C000121042001F052FF4D4B1B78002B40F08D
:10293C0038834C4B00221A70484B16221A7030E325
:10294C00444B1B889BB21D2B24D9464B01221A7079
:10295C0000F0BEFE0346FB7100F08CFF0346BB711A
:10296C0001F05AF803467B7101F02AF903463B71DA
:10297C00FB79042B0ED1BB79042B0BD17B79042B67
:10298C0008D13B79042B05D1364B00221A70334BFE
:10299C0016221A70344B1B8803F00203002B02D052
:1029AC002E4B13221A70304B1B8803F00103002BA3
:1029BC0000F0F9822C4B1B8803F48053002B00F0A1
:1029CC00F282264B14221A70224B00221A80EAE261
:1029DC0000220021012001F0F9FE0022002102203A
:1029EC0001F0F4FE00220021032001F0EFFE002292
:1029FC000021042001F0EAFE00220121012001F057
:102A0C00E5FE00220121022001F0E0FE002201215E
:102A1C00032001F0DBFE00220121042001F0D6FE90
:102A2C000F4B1B78002B40F0C0820E4B00221A700B
:102A3C000A4B00221A700C4B1B8823F002039AB22B
:102A4C00094B1A80B1E200BF4C0400202604002080
:102A5C001E040020FC030020160400205604002055
:102A6C00F003002057040020540400200022002111
:102A7C00012001F0ABFE00220021022001F0A6FE95
:102A8C0000220021032001F0A1FE002200210420DD
:102A9C0001F09CFE00220121012001F097FE002292
:102AAC000121022001F092FE00220121032001F0FD
:102ABC008DFE00220121042001F088FE984B00229B
:102ACC001A70984B1B889BB2132B40F27082964B5A
:102ADC0016221A706BE2954B1B8823F480539AB222
:102AEC00924B1A808F4B00221A80904B1B8803F05C
:102AFC000103002B0DD08A4B01221A708A4B17222E
:102B0C001A7001F031F901F001FA01F0D1FA01F07B
:102B1C00A3FB874B1A88874B1B889A4219D9012231
:102B2C004FF40041844803F080FD844B1B889BB21A
:102B3C00002B18D17A4B01221A707B4B18221A7079
:102B4C0001F012F901F0E2F901F0B2FA01F084FBA4
:102B5C0009E000224FF40041774803F066FD784B02
:102B6C001A88764B1A80714B1B8803F00203002BDA
:102B7C0003D06D4B19221A701BE26C4B1B8803F0AF
:102B8C001003002B17D0664B01221A706D4B1B885B
:102B9C00DAB26D4B1B88D9B26C4B1B88DBB20020B0
:102BAC00019000930B460021012001F08FFF5E4B3A
:102BBC0001221A70FDE15D4B1B8803F02003002BF2
:102BCC0017D0574B01221A705E4B1B88DAB25E4B42
:102BDC001B88D9B25D4B1B88DBB20020019000939F
:102BEC000B460121012001F071FF4F4B03221A709B
:102BFC00DFE14E4B1B8803F04003002B17D0484BF2
:102C0C0001221A704F4B5B88DAB2514B1B88D9B238
:102C1C004E4B1B88DBB20020019000930B46002129
:102C2C00022001F053FF404B05221A70C1E13F4BCB
:102C3C001B8803F08003002B17D0394B01221A702C
:102C4C00404B5B88DAB2424B1B88D9B23F4B1B8896
:102C5C00DBB20020019000930B460121022001F011
:102C6C0035FF314B07221A70A3E1304B1B8803F45C
:102C7C008073002B17D02A4B01221A70314B9B8882
:102C8C00DAB2344B1B88D9B2304B1B88DBB2002034
:102C9C00019000930B460021032001F017FF224BFB
:102CAC0009221A7085E1214B1B8803F40073002B59
:102CBC0017D01B4B01221A70224B9B88DAB2254B82
:102CCC001B88D9B2214B1B88DBB2002001900093EA
:102CDC000B460121032001F0F9FE134B0B221A7055
:102CEC0067E1124B1B8803F48063002B34D00C4B30
:102CFC0001221A70134BDB88DAB2164B1B88D9B23F
:102D0C00124B1B88DBB20020019000930B46002174
:102D1C00042001F0DBFE044B0D221A7049E100BFC8
:102D2C0057040020FC03002056040020540400200B
:102D3C00320200201C04002000080140FE03002089
:102D4C001A0400204C040020200400201E04002043
:102D5C0022040020240400209C4B1B8803F40063F5
:102D6C00002B00F026819A4B01221A70994BDB88BC
:102D7C00DAB2994B1B88D9B2984B1B88DBB2002076
:102D8C00019000930B460121042001F09FFE944B0F
:102D9C000F221A700DE1934B1B889BB2092B24D97F
:102DAC0000F0E2FF0346FB7101F0B0F80346BB7183
:102DBC0001F07EF903467B7101F04EFA03463B713C
:102DCC00FB79042B11D1BB79042B0ED17B79042B0D
:102DDC000BD13B79042B08D17D4B00221A70804B10
:102DEC0000221A70804B01221A70784B1B8803F05A
:102DFC000203002B02D07A4B19221A70734B1B88DA
:102E0C0003F00103002B00F0D680704B1B8803F4F9
:102E1C008053002B00F0CF80714B15221A70714B30
:102E2C0000221A80C7E06F4B1B889BB2092B40F223
:102E3C00C48000F099FF0346FB7101F067F803466C
:102E4C00BB7101F035F903467B7101F005FA0346BD
:102E5C003B71FB79042B40F0B080BB79042B40F024
:102E6C00AC807B79042B40F0A8803B79042B40F09C
:102E7C00A480574B00221A70594B00221A705A4BDF
:102E8C0001221A7099E000220021012001F09EFC21
:102E9C0000220021022001F099FC002200210320D5
:102EAC0001F094FC00220021042001F08FFC002290
:102EBC000121012001F08AFC00220121022001F0F5
:102ECC0085FC00220121032001F080FC002201215D
:102EDC00042001F07BFC3E4B00221A70414B1B88F6
:102EEC009BB2132B6BD93E4B00221A7067E0002269
:102EFC000021012001F06AFC00220021022001F0D7
:102F0C0065FC00220021032001F060FC002200215E
:102F1C00042001F05BFC00220121012001F056FC91
:102F2C0000220121022001F051FC0022012103208A
:102F3C0001F04CFC00220121042001F047FC2B4B3A
:102F4C001B78002B3DD1224B00221A70244B1622E9
:102F5C001A701E4B1B8823F002039AB21B4B1A806B
:102F6C002FE000BF2EE000BF2CE000BF2AE000BF26
:102F7C0028E000BF26E000BF24E000BF22E000BF35
:102F8C0020E000BF1EE000BF1CE000BF1AE000BF45
:102F9C0018E000BF16E000BF14E000BF12E000BF55
:102FAC0010E000BF0EE000BF0CE000BF0AE000BF65
:102FBC0008E000BF06E000BF04E000BF02E000BF75
:102FCC0000E000BF00BF0837BD4680BD54040020A0
:102FDC00570400204C040020240400201E04002070
:102FEC0056040020FC03002059040020F0030020AC
:102FFC0080B500AF02F04EF800F056F800F0B8FAC9
:10300C0000F098FA0AF0E6FC00F024F900F0C6F99A
:10301C0000F0A8F800F064FA05221E491E4802F0E0
:10302C0073F900211D4801F0FEF904211B4801F041
:10303C00FAF90821194801F0F6F90C21174801F0AA
:10304C00F2F90021164801F0EEF90421144801F0C0
:10305C00EAF90821124801F0E6F90C21104801F0B8
:10306C00E2F9FEF79BFA0346002B01D000BFFDE707
:10307C00FEF77EFB0B4B00221A70FDF7B9F9FDF73A
:10308C0067F8FEF797FFFFF701F9FEF78DF800BF21
:10309C00F3E700BFFC010020A4020020180300206D
:1030AC00600300205904002080B594B000AF07F1F4
:1030BC0028032822002118460BF0C8F907F1140345
:1030CC0000221A605A609A60DA601A613B1D002275
:1030DC001A605A609A60DA600123BB624FF4803345
:1030EC00FB6200233B630123BB6302237B644FF42D
:1030FC008033BB644FF48013FB6407F1280318463C
:10310C0005F00CF80346002B01D000F0DBFA0F237E
:10311C007B610223BB610023FB614FF480633B6244
:10312C0000237B6207F114030221184605F078FA9C
:10313C000346002B01D000F0C5FA12237B604FF43C
:10314C000043FB6000233B613B1D184605F0F8FB78
:10315C000346002B01D000F0B5FA00BF5037BD4636
:10316C0080BD000080B584B000AF3B1D00221A600A
:10317C005A609A60354B364A1A60344B4FF4807261
:10318C009A60324B01221A73304B00221A752F4B66
:10319C004FF46022DA612D4B00225A602B4B052232
:1031AC001A612A4801F0D8FF0346002B01D000F029
:1031BC0089FA04237B600123BB600323FB603B1D66
:1031CC001946224802F09AF90346002B01D000F070
:1031DC0079FA05237B600223BB603B1D19461B4813
:1031EC0002F08CF90346002B01D000F06BFA062399
:1031FC007B600323BB603B1D1946144802F07EF92B
:10320C000346002B01D000F05DFA07237B600423FA
:10321C00BB603B1D19460D4802F070F90346002BAC
:10322C0001D000F04FFA08237B600523BB603B1DE7
:10323C001946064802F062F90346002B01D000F053
:10324C0041FA00BF1037BD4680BD00BFA40200206C
:10325C000024014080B58EB000AF07F12803002296
:10326C001A605A609A60DA6007F1200300221A6033
:10327C005A603B1D00221A605A609A60DA601A612B
:10328C005A619A61444B4FF080421A60424B0022C3
:10329C005A60414B00229A603F4B44F24F62DA6015
:1032AC003D4B00221A613C4B00229A613A4805F0D2
:1032BC00FDFB0346002B01D000F004FA4FF48053C1
:1032CC00BB6207F128031946334805F05FFE03463D
:1032DC00002B01D000F0F6F92F4805F036FC034620
:1032EC00002B01D000F0EEF900233B6200237B623F
:1032FC0007F120031946284806F0E8F90346002B8D
:10330C0001D000F0DFF960237B604FF47A73BB606F
:10331C000023FB6004237B613B1D002219461E48E1
:10332C0005F072FD0346002B01D000F0CBF94FF4F1
:10333C00FA63BB603B1D04221946174805F064FD77
:10334C000346002B01D000F0BDF940F6B833BB604A
:10335C0000237B613B1D082219460F4805F054FDE4
:10336C000346002B01D000F0ADF94FF47A63BB603B
:10337C0004237B613B1D0C221946074805F044FDD4
:10338C000346002B01D000F09DF9034801F03EFDEF
:10339C0000BF3837BD4680BD1803002080B58EB005
:1033AC0000AF07F1280300221A605A609A60DA60B5
:1033BC0007F1200300221A605A603B1D00221A609C
:1033CC005A609A60DA601A615A619A61424B434AB8
:1033DC001A60414B00225A603F4B00229A603E4BD0
:1033EC0044F24F62DA603C4B00221A613A4B0022E5
:1033FC009A61394805F05AFB0346002B01D000F0C6
:10340C0061F94FF48053BB6207F128031946324827
:10341C0005F0BCFD0346002B01D000F053F92E48FB
:10342C0005F093FB0346002B01D000F04BF9002371
:10343C003B6200237B6207F120031946264806F005
:10344C0045F90346002B01D000F03CF960237B606A
:10345C0041F28833BB600023FB6004237B613B1D7E
:10346C00002219461C4805F0CFFC0346002B01D066
:10347C0000F028F941F27073BB603B1D0422194621
:10348C00154805F0C1FC0346002B01D000F01AF9D9
:10349C0041F65833BB603B1D082219460E4805F017
:1034AC00B3FC0346002B01D000F00CF94FF4FA5397
:1034BC00BB603B1D0C221946074805F0A5FC0346D2
:1034CC00002B01D000F0FEF8034801F09FFC00BF78
:1034DC003837BD4680BD00BF6003002000080040A7
:1034EC0080B500AF114B124A1A60104B4FF4E13209
:1034FC005A600E4B00229A600C4B0022DA600B4B88
:10350C0000221A61094B0C225A61084B00229A6165
:10351C00064B0022DA61054806F036F90346002B0B
:10352C0001D000F0CFF800BF80BD00BFA803002081
:10353C000038014080B582B000AF0C4B5B690B4A80
:10354C0043F001035361094B5B6903F001037B609A
:10355C007B68002200210B2002F0A1FA0B2002F064
:10356C00BAFA00BF0837BD4680BD00BF001002404C
:10357C0080B588B000AF07F1100300221A605A60C2
:10358C009A60DA604B4B9B694A4A43F01003936193
:10359C00484B9B6903F01003FB60FB68454B9B6930
:1035AC00444A43F020039361424B9B6903F0200390
:1035BC00BB60BB683F4B9B693E4A43F0040393617D
:1035CC003C4B9B6903F004037B607B68394B9B6924
:1035DC00384A43F008039361364B9B6903F00803A8
:1035EC003B603B6800224FF40051334803F01DF858
:1035FC00002240F63E41314803F017F800224FF408
:10360C0001412F4803F011F84FF400533B610123A3
:10361C007B610023BB610223FB6107F11003194698
:10362C00254802F067FE4FF440433B6100237B6169
:10363C000023BB6107F1100319461F4802F05AFE24
:10364C0010233B6103237B6107F1100319461C48CF
:10365C0002F050FE40F63E433B6101237B610023A8
:10366C00BB610223FB6107F110031946134802F0FA
:10367C0041FE4FF470433B6100237B610023BB612F
:10368C0007F1100319460D4802F034FE4FF40143C4
:10369C003B6101237B610023BB610223FB6107F1CA
:1036AC0010031946064802F025FE00BF2037BD4620
:1036BC0080BD00BF0010024000100140000C014012
:1036CC000008014080B400AF72B600BF00BFFDE738
:1036DC0080B59CB002AF5D4B1A785D4B1B789A425B
:1036EC0017D05B4B1A78594B1A70594B1B781A46EA
:1036FC003B1D584918460AF087FE3B1D1846FCF73F
:10370C001FFD03469AB2391D4FF0FF33524806F0A5
:10371C008BF8524B1B889AB2514B1B889A4202D29F
:10372C004B4B00221A704A4B1B78032B76D801A204
:10373C0052F823F0513700089D370008CD370008A8
:10374C00FF37000800220021012001F03FF8002281
:10375C000121012001F03AF8404B1B889AB2404BF2
:10376C001B889A4265D33F4B1B88DAB23E4B1B88B1
:10377C00D9B23E4B1B88DBB20020019000930B4664
:10378C000021012001F0A2F9314B01221A7050E006
:10379C00344B1B88DAB2344B1B88D9B2334B1B88A1
:1037AC00DBB20A20019000930B460021012001F0AE
:1037BC008DF90346002B3ED1254B02221A703AE0BC
:1037CC00264B1B889AB22A4B1B889A4235D3264B20
:1037DC001B88DAB2254B1B88DBB2002101910093C8
:1037EC0000230021012001F071F9194B03221A70FA
:1037FC0023E01D4B1B88DAB21C4B1B88DBB20A2161
:10380C000191009300230021012001F05FF9034690
:10381C00002B14D10E4B04221A7010E00022002150
:10382C00012000F0D3FF00220121012000F0CEFF87
:10383C0006E000BF04E000BF02E000BF00E000BFF4
:10384C00034B1B7818466837BD4680BD0700002027
:10385C006204002070F30008A8030020FC03002081
:10386C00280400204C040020000400201804002030
:10387C002A04002080B59CB002AF5D4B1A785D4BDA
:10388C001B789A4217D05B4B1A78594B1A70594BCC
:10389C001B781A463B1D584918460AF0B5FD3B1DCE
:1038AC001846FCF74DFC03469AB2391D4FF0FF3316
:1038BC00524805F0B9FF524B1B889AB2514B1B88EA
:1038CC009A4202D24B4B00221A704A4B1B78032BA4
:1038DC0076D801A252F823F0F538000841390008D7
:1038EC0071390008A339000800220021022000F0E1
:1038FC006DFF00220121022000F068FF404B1B8865
:10390C009AB2404B1B889A4265D33F4B5B88DAB224
:10391C003E4B1B88D9B23E4B1B88DBB2002001907A
:10392C0000930B460121022001F0D0F8314B01220B
:10393C001A7050E0344B5B88DAB2344B1B88D9B226
:10394C00334B1B88DBB20A20019000930B460121FC
:10395C00022001F0BBF80346002B3ED1254B02227E
:10396C001A703AE0264B1B889AB22A4B1B889A4253
:10397C0035D3264B1B88DAB2254B1B88DBB20021D2
:10398C000191009300230121022001F09FF8194BB3
:10399C0003221A7023E01D4B1B88DAB21C4B1B88C8
:1039AC00DBB20A210191009300230121022001F0D6
:1039BC008DF80346002B14D10E4B04221A7010E024
:1039CC0000220021022000F001FF00220121022030
:1039DC0000F0FCFE06E000BF04E000BF02E000BF08
:1039EC0000E000BF034B1B7818466837BD4680BD0E
:1039FC0008000020630400207CF30008A8030020CA
:103A0C00FC0300202C0400204C04002004040020A3
:103A1C00180400202E04002080B59CB002AF5D4B32
:103A2C001A785D4B1B789A4217D05B4B1A78594B1E
:103A3C001A70594B1B781A463B1D584918460AF008
:103A4C00E3FC3B1D1846FCF77BFB03469AB2391D81
:103A5C004FF0FF33524805F0E7FE524B1B889AB2E9
:103A6C00514B1B889A4202D24B4B00221A704A4B84
:103A7C001B78032B76D801A252F823F0993A000850
:103A8C00E53A0008153B0008473B000800220021DE
:103A9C00032000F09BFE00220121032000F096FE83
:103AAC00404B1B889AB2404B1B889A4265D33F4BC4
:103ABC009B88DAB23E4B1B88D9B23E4B1B88DBB2DB
:103ACC000020019000930B460021032000F0FEFF24
:103ADC00314B01221A7050E0344B9B88DAB2364BD2
:103AEC001B88D9B2334B1B88DBB20A2001900093A0
:103AFC000B460021032000F0E9FF0346002B3ED1CA
:103B0C00254B02221A703AE0264B1B889AB22B4B9B
:103B1C001B889A4235D3284B1B88DAB2254B1B885D
:103B2C00DBB200210191009300230021032000F05F
:103B3C00CDFF194B03221A7023E01F4B1B88DAB2FE
:103B4C001C4B1B88DBB20A2101910093002300213E
:103B5C00032000F0BBFF0346002B14D10E4B0422B4
:103B6C001A7010E000220021032000F02FFE00222A
:103B7C000121032000F02AFE06E000BF04E000BF94
:103B8C0002E000BF00E000BF034B1B78184668370B
:103B9C00BD4680BD090000206404002088F30008A5
:103BAC00A8030020FC030020300400204C0400205B
:103BBC000404002018040020080400203204002013
:103BCC0080B59CB002AF5D4B1A785D4B1B789A4266
:103BDC0017D05B4B1A78594B1A70594B1B781A46F5
:103BEC003B1D584918460AF00FFC3B1D1846FCF7C4
:103BFC00A7FA03469AB2391D4FF0FF33524805F02D
:103C0C0013FE524B1B889AB2514B1B889A4202D21C
:103C1C004B4B00221A704A4B1B78032B76D801A20F
:103C2C0052F823F0413C00088D3C0008BD3C0008D4
:103C3C00EF3C000800220021042000F0C7FD002208
:103C4C000121042000F0C2FD404B1B889AB2404B6E
:103C5C001B889A4265D33F4BDB88DAB23E4B1B88FC
:103C6C00D9B23E4B1B88DBB20020019000930B466F
:103C7C000021042000F02AFF314B01221A7050E081
:103C8C00344BDB88DAB2364B1B88D9B2334B1B88EA
:103C9C00DBB20A20019000930B460021042000F0B7
:103CAC0015FF0346002B3ED1254B02221A703AE039
:103CBC00264B1B889AB22B4B1B889A4235D3284B28
:103CCC001B88DAB2254B1B88DBB2002101910093D3
:103CDC0000230021042000F0F9FE194B03221A7076
:103CEC0023E01F4B1B88DAB21C4B1B88DBB20A216A
:103CFC000191009300230021042000F0E7FE03460D
:103D0C00002B14D10E4B04221A7010E0002200215B
:103D1C00042000F05BFD00220121042000F056FD80
:103D2C0006E000BF04E000BF02E000BF00E000BFFF
:103D3C00034B1B7818466837BD4680BD0A0000202F
:103D4C006504002094F30008A8030020FC03002065
:103D5C00340400204C04002004040020180400202B
:103D6C000C0400203604002080B59CB002AF5D4BE3
:103D7C001A785D4B1B789A4217D05B4B1A78594BCB
:103D8C001A70594B1B781A463B1D584918460AF0B5
:103D9C003BFB3B1D1846FCF7D3F903469AB2391D81
:103DAC004FF0FF33524805F03FFD524B1B889AB23F
:103DBC00514B1B889A4202D24B4B00221A704A4B31
:103DCC001B78032B76D801A252F823F0E93D0008AA
:103DDC00353E0008653E0008973E00080022002191
:103DEC00012000F0F3FC00220121012000F0EEFC88
:103DFC00404B1B889AB2404B1B889A4265D33F4B71
:103E0C001B88DAB23E4B1B88D9B23E4B1B88DBB207
:103E1C000020019000930B460121012000F056FE7A
:103E2C00314B01221A7050E0344B1B88DAB2344B00
:103E3C001B88D9B2334B1B88DBB20A20019000934C
:103E4C000B460121012000F041FE0346002B3ED120
:103E5C00254B02221A703AE0264B1B889AB22A4B49
:103E6C001B889A4235D3264B1B88DAB2254B1B880C
:103E7C00DBB200210191009300230121012000F00D
:103E8C0025FE194B03221A7023E01D4B1B88DAB256
:103E9C001C4B1B88DBB20A210191009300230121EA
:103EAC00012000F013FE0346002B14D10E4B04220C
:103EBC001A7010E000220021012000F087FC002283
:103ECC000121012000F082FC06E000BF04E000BFED
:103EDC0002E000BF00E000BF034B1B7818466837B8
:103EEC00BD4680BD0B00002066040020A0F3000836
:103EFC00A8030020FC030020380400204C04002000
:103F0C0002040020180400203A04002080B59CB064
:103F1C0002AF5D4B1A785D4B1B789A4217D05B4B06
:103F2C001A78594B1A70594B1B781A463B1D584935
:103F3C0018460AF069FA3B1D1846FCF701F90346CE
:103F4C009AB2391D4FF0FF33524805F06DFC524BBD
:103F5C001B889AB2514B1B889A4202D24B4B0022BF
:103F6C001A704A4B1B78032B76D801A252F823F017
:103F7C008D3F0008D93F0008094000083B4000086D
:103F8C0000220021022000F021FC0022012102204D
:103F9C0000F01CFC404B1B889AB2404B1B889A4289
:103FAC0065D33F4B5B88DAB23E4B1B88D9B23E4B94
:103FBC001B88DBB20020019000930B4600210220ED
:103FCC0000F084FD314B01221A7050E0344B5B88B9
:103FDC00DAB2344B1B88D9B2334B1B88DBB20A20C4
:103FEC00019000930B460021022000F06FFD034668
:103FFC00002B3ED1254B02221A703AE0264B1B882F
:10400C009AB22A4B1B889A4235D3264B1B88DAB2BC
:10401C00254B1B88DBB2002101910093002300216A
:10402C00022000F053FD194B03221A7023E01D4BA4
:10403C001B88DAB21C4B1B88DBB20A21019100935E
:10404C0000230021022000F041FD0346002B14D177
:10405C000E4B04221A7010E000220021022000F006
:10406C00B5FB00220121022000F0B0FB06E000BFEE
:10407C0004E000BF02E000BF00E000BF034B1B7870
:10408C0018466837BD4680BD0C0000206704002030
:10409C00ACF30008A8030020FC0300203C04002023
:1040AC004C04002006040020180400203E040020CC
:1040BC0080B59CB002AF5D4B1A785D4B1B789A4271
:1040CC0017D05B4B1A78594B1A70594B1B781A4600
:1040DC003B1D584918460AF097F93B1D1846FCF74A
:1040EC002FF803469AB2391D4FF0FF33524805F0B2
:1040FC009BFB524B1B889AB2514B1B889A4202D2A3
:10410C004B4B00221A704A4B1B78032B76D801A21A
:10411C0052F823F0314100087D410008AD41000800
:10412C00DF41000800220021032000F04FFB002299
:10413C000121032000F04AFB404B1B889AB2404BF4
:10414C001B889A4265D33F4B9B88DAB23E4B1B8847
:10415C00D9B23E4B1B88DBB20020019000930B467A
:10416C000121032000F0B2FC314B01221A7050E007
:10417C00344B9B88DAB2364B1B88D9B2334B1B8835
:10418C00DBB20A20019000930B460121032000F0C2
:10419C009DFC0346002B3ED1254B02221A703AE0BF
:1041AC00264B1B889AB22B4B1B889A4235D3284B33
:1041BC001B88DAB2254B1B88DBB2002101910093DE
:1041CC0000230121032000F081FC194B03221A70FB
:1041DC0023E01F4B1B88DAB21C4B1B88DBB20A2175
:1041EC000191009300230121032000F06FFC034692
:1041FC00002B14D10E4B04221A7010E00022002167
:10420C00032000F0E3FA00220121032000F0DEFA83
:10421C0006E000BF04E000BF02E000BF00E000BF0A
:10422C00034B1B7818466837BD4680BD0D00002037
:10423C0068040020B8F30008A8030020FC03002049
:10424C00400400204C040020060400201804002028
:10425C000A0400204204002080B59CB002AF5D4BE4
:10426C001A785D4B1B789A4217D05B4B1A78594BD6
:10427C001A70594B1B781A463B1D584918460AF0C0
:10428C00C3F83B1D1846FBF75BFF03469AB2391D7A
:10429C004FF0FF33524805F0C7FA524B1B889AB2C5
:1042AC00514B1B889A4202D24B4B00221A704A4B3C
:1042BC001B78032B76D801A252F823F0D9420008C0
:1042CC0025430008554300088743000800220021BD
:1042DC00042000F07BFA00220121042000F076FA81
:1042EC00404B1B889AB2404B1B889A4265D33F4B7C
:1042FC00DB88DAB23E4B1B88D9B23E4B1B88DBB253
:10430C000020019000930B460121042000F0DEFBFD
:10431C00314B01221A7050E0344BDB88DAB2344B4B
:10432C001B88D9B2334B1B88DBB20A200190009357
:10433C000B460121042000F0C9FB0346002B3ED1A3
:10434C00254B02221A703AE0264B1B889AB22A4B54
:10435C001B889A4235D3264B1B88DAB2254B1B8817
:10436C00DBB200210191009300230121042000F015
:10437C00ADFB194B03221A7023E01D4B1B88DAB2DC
:10438C001C4B1B88DBB20A210191009300230121F5
:10439C00042000F09BFB0346002B14D10E4B04228F
:1043AC001A7010E000220021042000F00FFA002205
:1043BC000121042000F00AFA06E000BF04E000BF6F
:1043CC0002E000BF00E000BF034B1B7818466837C3
:1043DC00BD4680BD0E00002069040020C4F3000817
:1043EC00A8030020FC030020440400204C040020FF
:1043FC000E040020180400204604002080B584B070
:10440C0000AF786039603968786804F086FE03463E
:10441C00FB73FB7B022B0CBF01230023DBB2184682
:10442C001037BD4680BD80B582B000AF7860396072
:10443C003968786804F084FC00BF0837BD4680BD3D
:10444C0080B584B000AFF860B9601346FB80BB68E0
:10445C00002B04D1FB681B68FA885A6313E0BB6815
:10446C00042B04D1FB681A68FB8893630BE0BB68D0
:10447C00082B04D1FB681A68FB88D36303E0FB6844
:10448C001A68FB881364B968F86804F0B7FB00BFBE
:10449C001037BD4680BD80B485B000AFF860B96000
:1044AC001346FB80BB68002B04D1FB681B68FA88A1
:1044BC005A6313E0BB68042B04D1FB681A68FB88B1
:1044CC0093630BE0BB68082B04D1FB681A68FB886C
:1044DC00D36303E0FB681A68FB88136400BF1437CE
:1044EC00BD4680BC7047000080B582B000AF03466B
:1044FC00FB710B46BB711346BB80FB79013B032B55
:10450C0000F2588101A252F823F000BF294500089F
:10451C00CB4500086D46000817470008BB79002BF7
:10452C0026D1BB88002B09D10021A548FFF77BFFC2
:10453C0000220221A34802F078F83CE10021A048B7
:10454C00FFF75CFF0346002B06D0BB881A46002100
:10455C009B48FFF7A0FF2EE101220221994802F0AF
:10456C0064F8BB881A4600219548FFF769FF22E1E1
:10457C00BB88002B09D104219148FFF754FF00227E
:10458C000221904802F051F815E104218C48FFF704
:10459C0035FF0346002B06D0BB881A4604218848F9
:1045AC00FFF779FF07E101220221864802F03DF86E
:1045BC00BB881A4604218248FFF742FFFBE0BB7917
:1045CC00002B26D1BB88002B09D108217C48FFF792
:1045DC002AFF002204217B4802F027F8EBE0082197
:1045EC007748FFF70BFF0346002B06D0BB881A4613
:1045FC0008217348FFF74FFFDDE0012204217148C9
:10460C0002F013F8BB881A4608216D48FFF718FF13
:10461C00D1E0BB88002B09D10C216948FFF703FFBF
:10462C0000220421674802F000F8C4E00C21644821
:10463C00FFF7E4FE0346002B06D0BB881A460C217C
:10464C005F48FFF728FFB6E0012204215D4801F026
:10465C00ECFFBB881A460C215948FFF7F1FEAAE083
:10466C00BB79002B28D1BB88002B0AD100215648DE
:10467C00FFF7D9FE00224FF48061524801F0D5FFBC
:10468C0099E000215048FFF7B9FE0346002B06D0F5
:10469C00BB881A4600214C48FFF7FDFE8BE0012237
:1046AC004FF48061474801F0C0FFBB881A460021D7
:1046BC004548FFF7C5FE7EE0BB88002B0AD10421DC
:1046CC004148FFF7B0FE00224FF480613D4801F0F5
:1046DC00ACFF70E004213C48FFF790FE0346002B32
:1046EC0006D0BB881A4604213748FFF7D4FE62E097
:1046FC0001224FF48061334801F097FFBB881A46C2
:10470C0004213148FFF79CFE55E0BB79002B28D1E2
:10471C00BB88002B0AD108212B48FFF784FE00220E
:10472C004FF40061274801F080FF44E0082126483F
:10473C00FFF764FE0346002B06D0BB881A460821FF
:10474C002148FFF7A8FE36E001224FF400611D4816
:10475C0001F06BFFBB881A4608211B48FFF770FE5F
:10476C0029E0BB88002B0AD10C211748FFF75BFE10
:10477C0000224FF40061134801F057FF1BE00C219D
:10478C001148FFF73BFE0346002B06D0BB881A46A8
:10479C000C210D48FFF77FFE0DE001224FF4006164
:1047AC00084801F042FFBB881A460C210648FFF767
:1047BC0047FE00E000BF00BF0837BD4680BD00BF0C
:1047CC0018030020000C01406003002080B584B069
:1047DC0000AF0346FB710B46BB7113467B717B79B3
:1047EC00FB60FB689B03FB60FB68B44AA2FB0323E2
:1047FC005B09FB60FB687B81FB79013B032B00F2BF
:10480C00578101A252F823F025480008C748000838
:10481C0069490008134A0008BB79002B26D17B8913
:10482C00002B09D10021A648FFF7FDFD0022022133
:10483C00A44801F0FAFE3CE10021A148FFF7DEFD9F
:10484C000346002B06D07B891A4600219C48FFF7B3
:10485C0022FE2EE1012202219A4801F0E6FE7B891C
:10486C001A4600219648FFF7EBFD22E17B89002BCD
:10487C0009D104219248FFF7D6FD0022022191486C
:10488C0001F0D3FE15E104218D48FFF7B7FD034677
:10489C00002B06D07B891A4604218948FFF7FBFDC3
:1048AC0007E101220221874801F0BFFE7B891A46ED
:1048BC0004218348FFF7C4FDFBE0BB79002B26D114
:1048CC007B89002B09D108217D48FFF7ACFD002224
:1048DC0004217C4801F0A9FEEBE008217848FFF7A1
:1048EC008DFD0346002B06D07B891A46082174489F
:1048FC00FFF7D1FDDDE001220421724801F095FEA5
:10490C007B891A4608216E48FFF79AFDD1E07B8916
:10491C00002B09D10C216A48FFF785FD00220421E8
:10492C00684801F082FEC4E00C216548FFF766FD83
:10493C000346002B06D07B891A460C216048FFF7F2
:10494C00AAFDB6E0012204215E4801F06EFE7B89CF
:10495C001A460C215A48FFF773FDAAE0BB79002BCD
:10496C0028D17B89002B0AD100215748FFF75BFD2A
:10497C0000224FF48061534801F057FE99E000216A
:10498C005148FFF73BFD0346002B06D07B891A46A6
:10499C0000214D48FFF77FFD8BE001224FF4806131
:1049AC00484801F042FE7B891A4600214648FFF731
:1049BC0047FD7EE07B89002B0AD104214248FFF79A
:1049CC0032FD00224FF480613E4801F02EFE70E073
:1049DC0004213D48FFF712FD0346002B06D07B89CE
:1049EC001A4604213848FFF756FD62E001224FF4C5
:1049FC008061344801F019FE7B891A460421324843
:104A0C00FFF71EFD55E0BB79002B28D17B89002BCD
:104A1C000AD108212C48FFF706FD00224FF4006153
:104A2C00284801F002FE44E008212748FFF7E6FC85
:104A3C000346002B06D07B891A4608212248FFF733
:104A4C002AFD36E001224FF400611E4801F0EDFD15
:104A5C007B891A4608211C48FFF7F2FC29E07B8968
:104A6C00002B0AD10C211848FFF7DDFC00224FF473
:104A7C000061144801F0D9FD1BE00C211248FFF72E
:104A8C00BDFC0346002B06D07B891A460C210E4830
:104A9C00FFF701FD0DE001224FF40061094801F020
:104AAC00C4FD7B891A460C210748FFF7C9FC00E0BE
:104ABC0000BF00BF1037BD4680BD00BF1F85EB5146
:104ACC0018030020000C01406003002090B585B055
:104ADC0000AF0446084611461A462346FB710346AE
:104AEC00BB710B467B7113463B7197F82430002B3E
:104AFC0002D00A2B16D09DE0FB79013B97F82020C1
:104B0C0091B24F4A084622F81300FB79013BC9B217
:104B1C004C4AD1547A79B979FB791846FFF756FE8D
:104B2C00002388E0FB79013B464AD35C1946FB79AC
:104B3C00013B434A32F813309BB2994278D0FB794F
:104B4C00013B3F4A32F813309AB2FB79013BD1B2A8
:104B5C003C4AD154FB79013B394A32F813309BB2B1
:104B6C00002B5DD07A793B799A4226D97B799AB21F
:104B7C003B799BB2D31AFB8197F820309AB2FB7920
:104B8C00013B2F4931F813309BB2D31A9BB2FA89EF
:104B9C0002FB03F3FB81FA8997F8203092FBF3F3C5
:104BAC00FB81FB89DBB27A79D31ADAB2B979FB795A
:104BBC001846FFF70BFE01233DE07A793B799A42C8
:104BCC0026D23B799AB27B799BB2D31AFB8197F8A8
:104BDC0020309AB2FB79013B194931F813309BB262
:104BEC00D31A9BB2FA8902FB03F3FB81FA8997F87B
:104BFC00203092FBF3F3FB81FB89DAB27B7913440F
:104C0C00DAB2B979FB791846FFF7E0FD012312E01F
:104C1C003A79B979FB791846FFF7D8FD00230AE0F9
:104C2C003A79B979FB791846FFF7D0FD002302E0F9
:104C3C00012300E0002318461437BD4690BD00BF89
:104C4C00F40300206C04002080B485B000AF154B39
:104C5C009B69144A43F001039361124B9B6903F067
:104C6C000103BB60BB680F4BDB690E4A43F08053FA
:104C7C00D3610C4BDB6903F080537B607B680A4B80
:104C8C005B68FB60FB6823F0E063FB60FB6843F050
:104C9C000073FB60044AFB68536000BF1437BD46C9
:104CAC0080BC7047001002400000014080B58AB003
:104CBC0000AF786007F1180300221A605A609A60FE
:104CCC00DA607B681B68334A93425FD1324B9B6935
:104CDC00314A43F4007393612F4B9B6903F40073C7
:104CEC007B617B692C4B9B692B4A43F004039361DA
:104CFC00294B9B6903F004033B613B69264B9B6981
:104D0C00254A43F008039361234B9B6903F0080386
:104D1C00FB60FB68F023BB610323FB6107F1180305
:104D2C0019461E4801F0E6FA0123BB610323FB611F
:104D3C0007F1180319461A4801F0DCFA194B1A4A04
:104D4C001A60184B00225A60164B00229A60154BC1
:104D5C008022DA60134B4FF480721A61114B4FF4BE
:104D6C0080625A610F4B20229A610E4B0022DA614D
:104D7C000C4800F0D1FE0346002B01D0FEF7A2FC3C
:104D8C007B68084A1A62074A7B68536200BF28375F
:104D9C00BD4680BD002401400010024000080140C7
:104DAC00000C0140D40200200800024080B485B001
:104DBC0000AF78607B681B68B3F1804F0CD1114B4E
:104DCC00DB69104A43F00103D3610E4BDB6903F03E
:104DDC000103FB60FB6810E07B681B680A4A934286
:104DEC000BD1084BDB69074A43F00403D361054B35
:104DFC00DB6903F00403BB60BB6800BF1437BD461E
:104E0C0080BC7047001002400008004080B588B09C
:104E1C0000AF786007F1100300221A605A609A60A4
:104E2C00DA607B681B68B3F1804F18D11D4B9B690E
:104E3C001C4A43F0040393611A4B9B6903F004036F
:104E4C00FB60FB680F233B6102237B610223FB6148
:104E5C0007F110031946144801F04CFA1DE07B6869
:104E6C001B68124A934218D10E4B9B690D4A43F0B2
:104E7C00080393610B4B9B6903F00803BB60BB6891
:104E8C004FF470733B6102237B610223FB6107F1DA
:104E9C0010031946064801F02DFA00BF2037BD4615
:104EAC0080BD00BF00100240000801400008004017
:104EBC00000C014080B588B000AF786007F110039A
:104ECC0000221A605A609A60DA607B681B681C4A80
:104EDC00934231D11B4B9B691A4A43F48043936133
:104EEC00184B9B6903F48043FB60FB68154B9B6973
:104EFC00144A43F004039361124B9B6903F00403BF
:104F0C00BB60BB684FF400733B6102237B610323DE
:104F1C00FB6107F1100319460B4801F0EBF94FF454
:104F2C0080633B6100237B610023BB6107F11003AD
:104F3C001946054801F0DEF900BF2037BD4680BD9B
:104F4C0000380140001002400008014080B400AF5E
:104F5C0000BFFDE780B400AF00BFFDE780B400AF39
:104F6C0000BFFDE780B400AF00BFFDE780B400AF29
:104F7C0000BFFDE780B400AF00BFBD4680BC7047EA
:104F8C0080B400AF00BFBD4680BC704780B400AF9A
:104F9C0000BFBD4680BC704780B500AF00F0C0F8C4
:104FAC0000F0B3FD00BF80BD80B500AF024800F03B
:104FBC006DFE00BF80BD00BFD402002080B500AFE5
:104FCC00024801F066FC00BF80BD00BF64120020E7
:104FDC0080B586B000AF7860144A154BD31A7B614C
:104FEC007B693B61134B1B68002B02D1114B124A9E
:104FFC001A60104B1A687B6813443A699A4207D2BC
:10500C0009F02CFA03460C221A604FF0FF3309E02A
:10501C00084B1B68FB60074B1A687B681344054AF6
:10502C001360FB6818461837BD4680BD0050002041
:10503C000004000070040020A818002080B400AF09
:10504C0000BFBD4680BC7047FFF7F8FF0B480C490A
:10505C000C4A002302E0D458C4500433C4188C42C8
:10506C00F9D3094A094C002301E013600432A2422F
:10507C00FBD309F0F9F9FDF7BBFF704700000020E6
:10508C00DC01002088F50008E0010020A4180020B5
:10509C00FEE7000080B500AF084B1B68074A43F0E1
:1050AC0010031360032000F0EFFC0F2000F008F851
:1050BC00FFF7CAFD0023184680BD00BF0020024048
:1050CC0080B582B000AF7860124B1A68124B1B7817
:1050DC0019464FF47A73B3FBF1F3B2FBF3F31846B2
:1050EC0000F007FD0346002B01D001230EE07B6886
:1050FC000F2B0AD8002279684FF0FF3000F0CFFC5C
:10510C00064A7B681360002300E001231846083729
:10511C00BD4680BD100000201800002014000020A7
:10512C0080B400AF054B1B781A46054B1B68134423
:10513C00034A136000BFBD4680BC704718000020B6
:10514C007404002080B400AF024B1B681846BD46A7
:10515C0080BC70477404002080B586B000AF7860C6
:10516C000023FB7500233B610023BB600023FB6025
:10517C007B68002B01D10123BEE07B689B68002B70
:10518C007B689B6A002B09D17B680022DA627B6802
:10519C00002283F824207868FFF788FD786800F0F7
:1051AC00FFFA0346FB757B689B6A03F01003002B28
:1051BC0040F09980FB7D002B40F095807B689B6ACA
:1051CC0023F4885323F0020343F002027B689A62B3
:1051DC007B685A687B68DB691A437B681B7B5B00C6
:1051EC001343BA681343BB607B689B68B3F5807F3D
:1051FC0003D07B689B68012B02D14FF4807300E0D5
:10520C0000233A6913433B617B681B7D012B19D149
:10521C007B681B7B002B09D17B689B69013B5A0384
:10522C003B69134343F400633B610BE07B689B6A6F
:10523C0043F020027B689A627B68DB6A43F00102D0
:10524C007B68DA627B681B685B6823F469417B6866
:10525C001B683A690A435A607B681B689A68284B3A
:10526C0013407A681268B9680B4393607B689B683B
:10527C00B3F5807F03D07B689B68012B04D17B68DE
:10528C001B69013B1B05FB607B681B68DB6A23F415
:10529C0070017B681B68FA680A43DA627B681B68DA
:1052AC009A68184B1340BA689A420BD17B6800225B
:1052BC00DA627B689B6A23F0030343F001027B688C
:1052CC009A6218E07B689B6A23F0120343F0100289
:1052DC007B689A627B68DB6A43F001027B68DA6266
:1052EC000123FB7507E07B689B6A43F010027B6827
:1052FC009A620123FB75FB7D18461837BD4680BDAD
:10530C00FDF7E1FFFE0E1FFF80B586B000AFF86021
:10531C00B9607A600023FB75FB681B68644A934292
:10532C0004D0FB681B68634A934206D1604B5B68F0
:10533C0003F47023002B40F0B380FB6893F8243007
:10534C00012B01D10223AEE0FB68012283F824205B
:10535C00F86800F0CBF90346FB75FB7D002B40F0A1
:10536C009A80FB689B6A23F4706323F0010343F477
:10537C008072FB689A62FB681B684E4A934205D1A7
:10538C004B4B5B6803F47023002B15D1FB689B6AB5
:10539C0023F48012FB689A62FB681B685B6803F459
:1053AC008063002B26D0FB689B6A23F4405343F4A4
:1053BC008052FB689A621DE0FB689B6A43F4801282
:1053CC00FB689A62FB681B68394A934204D0FB68FD
:1053DC001B68384A93420DD1354B5B6803F48063EC
:1053EC00002B07D0FB689B6A23F4405343F4805294
:1053FC00FB689A62FB689B6A03F48053002B06D00F
:10540C00FB68DB6A23F00602FB68DA6202E0FB68E9
:10541C000022DA62FB68002283F82420FB681B6AF6
:10542C00254A9A62FB681B6A244ADA62FB681B6A8B
:10543C00234A1A63FB681B686FF002021A60FB6850
:10544C001B689A68FB681B6842F480729A60FB6860
:10545C00186AFB681B684C331946BA687B6800F005
:10546C00B5FBFB681B689B6803F46023B3F5602FE6
:10547C0008D1FB681B689A68FB681B6842F4A002A1
:10548C009A600FE0FB681B689A68FB681B6842F423
:10549C0080129A6006E0FB68002283F8242001E069
:1054AC000123FB75FB7D18461837BD4680BD00BF38
:1054BC0000240140002801402F580008AB58000878
:1054CC00C758000880B483B000AF786000BF0C37B9
:1054DC00BD4680BC704780B483B000AF786000BF1D
:1054EC000C37BD4680BC704780B483B000AF786089
:1054FC0000BF0C37BD4680BC7047000080B485B03F
:10550C0000AF786039600023FB730023BB607B68BD
:10551C0093F82430012B01D10223DCE07B680122BB
:10552C0083F824203B685B68062B1CD87B681B68BF
:10553C00596B3B685A6813469B001344053B1F226A
:10554C0002FA03F3DB4319403B6818683B685A685E
:10555C0013469B001344053B00FA03F27B681B685F
:10556C000A435A633CE03B685B680C2B1CD87B6895
:10557C001B68196B3B685A6813469B001344233B0A
:10558C001F2202FA03F3DB4319403B6818683B689F
:10559C005A6813469B001344233B00FA03F27B68C2
:1055AC001B680A431A631BE07B681B68D96A3B685B
:1055BC005A6813469B001344413B1F2202FA03F323
:1055CC00DB4319403B6818683B685A6813469B00DC
:1055DC001344413B00FA03F27B681B680A43DA620E
:1055EC003B681B68092B1CD97B681B68D9683B6816
:1055FC001A6813465B0013441E3B072202FA03F39E
:10560C00DB4319403B6898683B681A6813465B009B
:10561C0013441E3B00FA03F27B681B680A43DA60F2
:10562C0019E07B681B6819693B681A6813465B00B4
:10563C001344072202FA03F3DB4319403B689868D2
:10564C003B681A6813465B00134400FA03F27B684C
:10565C001B680A431A613B681B68102B03D03B681C
:10566C001B68112B32D17B681B681D4A934225D1D4
:10567C007B681B689B6803F40003002B26D17B68B6
:10568C001B689A687B681B6842F400029A603B684E
:10569C001B68102B1AD1134B1B68134AA2FB032354
:1056AC009A0C13469B0013445B00BB6002E0BB6882
:1056BC00013BBB60BB68002BF9D107E07B689B6AA0
:1056CC0043F020027B689A620123FB737B68002203
:1056DC0083F82420FB7B18461437BD4680BC7047EA
:1056EC00002401401000002083DE1B4380B584B0F1
:1056FC0000AF78600023FB600023BB607B681B68F5
:10570C009B6803F00103012B40D07B681B689A68EF
:10571C007B681B6842F001029A601F4B1B681F4A92
:10572C00A2FB03239B0CBB6002E0BB68013BBB608C
:10573C00BB68002BF9D1FFF705FDF8601FE0FFF700
:10574C0001FD0246FB68D31A022B18D97B681B6833
:10575C009B6803F00103012B11D07B689B6A43F01B
:10576C0010027B689A627B68DB6A43F001027B68FB
:10577C00DA627B68002283F82420012307E07B682F
:10578C001B689B6803F00103012BD8D1002318463A
:10579C001037BD4680BD00BF1000002083DE1B43C8
:1057AC0080B584B000AF78600023FB607B681B6819
:1057BC009B6803F00103012B2ED17B681B689A6850
:1057CC007B681B6822F001029A60FFF7BBFCF86053
:1057DC001BE0FFF7B7FC0246FB68D31A022B14D967
:1057EC007B681B689B6803F00103012B0DD17B6860
:1057FC009B6A43F010027B689A627B68DB6A43F019
:10580C0001027B68DA62012307E07B681B689B68F6
:10581C0003F00103012BDCD0002318461037BD46E2
:10582C0080BD80B584B000AF78607B685B6AFB603C
:10583C00FB689B6A03F05003002B27D1FB689B6A23
:10584C0043F40072FB689A62FB681B689B6803F464
:10585C006023B3F5602F15D1FB681B7B002B11D196
:10586C00FB689B6A23F48072FB689A62FB689B6AF4
:10587C0003F48053002B05D1FB689B6A43F00102B3
:10588C00FB689A62F868FFF71DFE04E0FB681B6A70
:10589C001B6B7868984700BF1037BD4680BD80B53C
:1058AC0084B000AF78607B685B6AFB60F868FFF7D8
:1058BC0012FE00BF1037BD4680BD80B584B000AF6E
:1058CC0078607B685B6AFB60FB689B6A43F0400214
:1058DC00FB689A62FB68DB6A43F00402FB68DA62DD
:1058EC00F868FFF701FE00BF1037BD4680BD000011
:1058FC0080B485B000AF78607B6803F00703FB6071
:10590C000C4BDB68BB60BA684FF6FF031340BB60FF
:10591C00FB681A02BB68134343F0BF6343F40033C4
:10592C00BB60044ABB68D36000BF1437BD4680BC63
:10593C00704700BF00ED00E080B400AF044BDB68A3
:10594C001B0A03F007031846BD4680BC704700BF16
:10595C0000ED00E080B483B000AF0346FB7197F913
:10596C000730002B0BDBFB7903F01F02064997F97C
:10597C0007305B09012000FA02F241F8232000BF36
:10598C000C37BD4680BC704700E100E080B483B0AA
:10599C0000AF03463960FB7197F90730002B0ADB27
:1059AC003B68DAB20C4997F907301201D2B20B44BA
:1059BC0083F800230AE03B68DAB20849FB7903F06C
:1059CC000F03043B1201D2B20B441A7600BF0C3702
:1059DC00BD4680BC704700BF00E100E000ED00E078
:1059EC0080B489B000AFF860B9607A60FB6803F0EE
:1059FC000703FB61FB69C3F10703042B28BF0423D6
:105A0C00BB61FB690433062B02D9FB69033B00E045
:105A1C0000237B614FF0FF32BB6902FA03F3DA43D8
:105A2C00BB681A407B699A404FF0FF317B6901FAE1
:105A3C0003F3D9437B680B40134318462437BD4608
:105A4C0080BC704780B582B000AF78607B68013B4A
:105A5C00B3F1807F01D301230FE00A4A7B68013B3D
:105A6C0053600F214FF0FF30FFF790FF054B0022E2
:105A7C009A60044B07221A60002318460837BD466B
:105A8C0080BD00BF10E000E080B582B000AF786050
:105A9C007868FFF72DFF00BF0837BD4680BD80B585
:105AAC0086B000AF0346B9607A60FB7300237B615C
:105ABC00FFF742FF78617A68B9687869FFF790FF61
:105ACC00024697F90F3011461846FFF75FFF00BFEB
:105ADC001837BD4680BD80B582B000AF0346FB7160
:105AEC0097F907301846FFF735FF00BF0837BD465A
:105AFC0080BD80B582B000AF78607868FFF7A2FFF8
:105B0C00034618460837BD4680BD80B500AFFCF78C
:105B1C003FF800BF80BD000080B485B000AF786056
:105B2C000023FB607B68002B01D1012343E07B68E1
:105B3C001B681A46224B1344224AA2FB03231B095F
:105B4C009A007B681A647B681F4ADA637B680222BE
:105B5C0083F821207B681B681B68FB60FB6823F4BF
:105B6C007F5323F03003FB607B685A687B689B682B
:105B7C001A437B68DB681A437B681B691A437B6892
:105B8C005B691A437B689B691A437B68DB69134327
:105B9C00FA681343FB607B681B68FA681A607B68C1
:105BAC0000229A637B68012283F821207B68002203
:105BBC0083F82020002318461437BD4680BC70475C
:105BCC00F8FFFDBFCDCCCCCC0000024080B586B038
:105BDC0000AFF860B9607A603B600023FB75FB682E
:105BEC0093F82030012B01D102234BE0FB680122FA
:105BFC0083F82020FB6893F82130DBB2012B3AD1DB
:105C0C00FB68022283F82120FB6800229A63FB6860
:105C1C001B681A68FB681B6822F001021A603B685B
:105C2C007A68B968F86800F037F9FB68DB6A002B12
:105C3C0008D0FB681B681A68FB681B6842F00E02F0
:105C4C001A600FE0FB681B681A68FB681B6822F07F
:105C5C0004021A60FB681B681A68FB681B6842F038
:105C6C000A021A60FB681B681A68FB681B6842F022
:105C7C0001021A6005E0FB68002283F82020022351
:105C8C00FB75FB7D18461837BD4680BD80B584B0CA
:105C9C0000AF78607B68DB6B1B68FB607B681B6804
:105CAC001B68BB607B681B6C04229A40FB6813402A
:105CBC00002B4FD0BB6803F00403002B4AD07B6849
:105CCC001B681B6803F02003002B07D17B681B6843
:105CDC001A687B681B6822F004021A607B681B68D8
:105CEC00664A934229D07B681B68654A934222D04E
:105CFC007B681B68634A93421AD07B681B68624AB4
:105D0C00934212D07B681B68604A93420AD07B682E
:105D1C001B685F4A934202D14FF480030EE04FF0B0
:105D2C0080630BE04FF4802308E04FF4804305E0E0
:105D3C004FF4806302E0402300E00423554A536093
:105D4C007B68DB6A002B00F094807B68DB6A7868E8
:105D5C0098478EE07B681B6C02229A40FB681340CC
:105D6C00002B56D0BB6803F00203002B51D07B688C
:105D7C001B681B6803F02003002B0BD17B681B688E
:105D8C001A687B681B6822F00A021A607B68012281
:105D9C0083F821207B681B68384A934229D07B68A2
:105DAC001B68374A934222D07B681B68354A934262
:105DBC001AD07B681B68344A934212D07B681B68EC
:105DCC00324A93420AD07B681B68314A934202D113
:105DDC004FF400130EE04FF000730BE04FF4003360
:105DEC0008E04FF4005305E04FF4007302E0202369
:105DFC0000E00223274A53607B68002283F82020AE
:105E0C007B689B6A002B34D07B689B6A78689847C8
:105E1C002FE07B681B6C08229A40FB681340002B18
:105E2C0028D0BB6803F00803002B23D07B681B68C9
:105E3C001A687B681B6822F00E021A607B681A6C69
:105E4C007B68DB6B012101FA02F25A607B6801224C
:105E5C009A637B68012283F821207B68002283F8F7
:105E6C0020207B681B6B002B04D07B681B6B786835
:105E7C00984700BF00BF1037BD4680BD08000240E8
:105E8C001C00024030000240440002405800024016
:105E9C006C0002400000024080B485B000AFF86096
:105EAC00B9607A603B60FB681A6CFB68DB6B0121A4
:105EBC0001FA02F25A60FB681B683A685A60FB6888
:105ECC005B68102B08D1FB681B687A689A60FB68CA
:105EDC001B68BA68DA6007E0FB681B68BA689A60EE
:105EEC00FB681B687A68DA6000BF1437BD4680BC5B
:105EFC0070470000F0B587B000AFF860B960C7E933
:105F0C0000230123FB750023BB7500237B752F4BEE
:105F1C001B7E012B01D1022354E02C4B01221A765B
:105F2C004CF2503000F0A8F80346FB75FB7D002BBB
:105F3C0044D1FB68012B02D101237B7507E0FB6880
:105F4C00022B02D102237B7501E004237B75002315
:105F5C00BB752DE0BB7D5A00BB6802EB030CBB7D0F
:105F6C001901D7E90023C1F12006A1F1200022FA82
:105F7C0001F403FA06F6344323FA00F0044323FA3F
:105F8C0001F5A3B21946604600F05AF84CF25030B5
:105F9C0000F072F80346FB750D4B1B690C4A23F09D
:105FAC0001031361FB7D002B07D1BB7D0133BB7556
:105FBC00BA7D7B7D9A42CDD300E000BF034B00221B
:105FCC001A76FB7D18461C37BD46F0BD78040020C0
:105FDC000020024080B483B000AF0023FB710D4B56
:105FEC001B6903F08003002B0DD00A4B0A4A5A6040
:105FFC00084B0A4A5A60074B1B6903F08003002BBD
:10600C0001D00123FB71FB7918460C37BD4680BCCF
:10601C00704700BF0020024023016745AB89EFCDDC
:10602C0080B400AF054B1B69044A43F08003136135
:10603C0000231846BD4680BC704700BF00200240BC
:10604C0080B483B000AF78600B467B80084B002295
:10605C00DA61084B1B69074A43F0010313617B6843
:10606C007A881A8000BF0C37BD4680BC704700BFD1
:10607C00780400200020024080B584B000AF786026
:10608C00FFF760F8F86010E07B68B3F1FF3F0CD0CD
:10609C007B68002B07D0FFF755F80246FB68D31A34
:1060AC007A689A4201D2032325E0154BDB6803F092
:1060BC000103002BE8D1124BDB6803F02003002B0B
:1060CC0002D00F4B2022DA600D4BDB6803F010037B
:1060DC00002B0BD10A4BDB6903F00103002B05D11C
:1060EC00074BDB6803F00403002B03D000F00AF825
:1060FC00012300E0002318461037BD4680BD00BFC9
:10610C000020024080B483B000AF00237B60234B9F
:10611C00DB6803F01003002B09D0214BDB6943F043
:10612C0002031F4AD3617B6843F010037B601B4B57
:10613C00DB6803F00403002B09D0194BDB6943F037
:10614C000103174AD3617B6843F004037B60134B54
:10615C00DB6903F00103002B0BD0114BDB6943F01F
:10616C0004030F4AD3610D4BDB690C4A23F0010386
:10617C00D3617B6840F20112934206D1074BDB6975
:10618C00064A23F00103D36102E0044A7B68D36022
:10619C0000BF0C37BD4680BC704700BF00200240DA
:1061AC007804002080B584B000AF7860396001239A
:1061BC00FB730023BB602F4B1B7E012B01D10223F1
:1061CC0053E02C4B01221A767B681B68022B16D1EC
:1061DC004CF25030FFF750FF0346002B41D1012009
:1061EC0000F04CF84CF25030FFF746FF0346FB73BF
:1061FC00214B1B69204A23F00403136131E04CF25C
:10620C005030FFF739FF0346002B2AD13B684FF083
:10621C00FF321A607B689B68BB6019E0B86800F0BD
:10622C0049F84CF25030FFF727FF0346FB73124B33
:10623C001B69114A23F002031361FB7B002B03D073
:10624C003B68BA681A600CE0BB6803F58063BB60FE
:10625C007B68DB689A027B689B681344BA689A4235
:10626C00DCD3044B00221A76FB7B18461037BD4654
:10627C0080BD00BF780400200020024080B483B0B1
:10628C0000AF7860094B0022DA61094B1B69084AA0
:10629C0043F004031361064B1B69054A43F04003AA
:1062AC00136100BF0C37BD4680BC704778040020DA
:1062BC000020024080B483B000AF78600B4B00220A
:1062CC00DA610B4B1B690A4A43F002031361084A5B
:1062DC007B685361064B1B69054A43F0400313610D
:1062EC0000BF0C37BD4680BC704700BF780400204F
:1062FC000020024080B48BB000AF7860396000237E
:10630C007B6200233B6269E101227B6A02FA03F3A0
:10631C00FB613B681B68FA691340BB61BA69FB6996
:10632C009A4240F058813B685B689A4A93425ED02F
:10633C00984A934275D8984A934258D0964A9342B9
:10634C006FD8964A934252D0944A934269D8944A51
:10635C0093424CD0924A934263D8924A934246D08D
:10636C00904A93425DD8122B2AD8122B59D801A2ED
:10637C0052F823F0FB630008D5630008E7630008BC
:10638C00296400082F6400082F6400082F6400089B
:10639C002F6400082F6400082F6400082F64000885
:1063AC002F6400082F6400082F6400082F64000875
:1063BC002F6400082F640008DD630008F1630008F7
:1063CC00794A934213D02CE03B68DB683B6229E0AE
:1063DC003B68DB6804333B6224E03B68DB680833D2
:1063EC003B621FE03B68DB680C333B621AE03B68A6
:1063FC009B68002B02D104233B6213E03B689B6833
:10640C00012B05D108233B627B68FA691A6109E00C
:10641C0008233B627B68FA695A6103E000233B6204
:10642C0000E000BFBB69FF2B01D87B6801E07B68F3
:10643C0004337B61BB69FF2B02D87B6A9B0002E0B3
:10644C007B6A083B9B003B617B691A680F213B69A7
:10645C0001FA03F3DB431A40396A3B6901FA03F38F
:10646C001A437B691A603B685B6803F08053002B0E
:10647C0000F0B1804D4B9B694C4A43F00103936192
:10648C004A4B9B6903F00103BB60BB68484A7B6ABB
:10649C009B08023352F82330FB607B6A03F0030342
:1064AC009B000F2202FA03F3DB43FA681340FB60F4
:1064BC007B68404A934213D07B683F4A93420DD08D
:1064CC007B683E4A934207D07B683D4A934201D198
:1064DC00032306E0042304E0022302E0012300E08E
:1064EC0000237A6A02F0030292009340FA68134385
:1064FC00FB602F497B6A9B080233FA6841F8232022
:10650C003B685B6803F48013002B06D02D4B9A6814
:10651C002C49BB6913438B6006E02A4B9A68BB6914
:10652C00DB43284913408B603B685B6803F4001322
:10653C00002B06D0234BDA682249BB691343CB608E
:10654C0006E0204BDA68BB69DB431E491340CB6085
:10655C003B685B6803F40033002B06D0194B5A6878
:10656C001849BB6913434B6006E0164B5A68BB696C
:10657C00DB43144913404B603B685B6803F4803386
:10658C00002B21D00F4B1A680E49BB6913430B60CB
:10659C0021E000BF0000321000003110000022107A
:1065AC000000211000001210000011100010024019
:1065BC000000014000080140000C014000100140A7
:1065CC0000140140000401400B4B1A68BB69DB430B
:1065DC00094913400B607B6A01337B623B681A6884
:1065EC007B6A22FA03F3002B7FF48EAE00BF00BF50
:1065FC002C37BD4680BC70470004014080B485B088
:10660C0000AF78600B467B807B689A687B88134070
:10661C00002B02D00123FB7301E00023FB73FB7BF7
:10662C0018461437BD4680BC704780B483B000AFA9
:10663C0078600B467B8013467B707B78002B03D0F5
:10664C007A887B681A6103E07B881A047B681A617C
:10665C0000BF0C37BD4680BC704780B584B000AF1E
:10666C0078607B68002B01D10123E8E07B6893F80C
:10667C009132DBB2002B06D17B68002283F890228A
:10668C00786807F017FC7B68032283F891227B68FB
:10669C0000225A717B681B68184603F0BCFA7B68B1
:1066AC0018687B6804330ECB03F092FA0346002B78
:1066BC0005D07B68022283F891220123BFE07B681E
:1066CC001B680021184603F0C0FA0346002B05D0C6
:1066DC007B68022283F891220123B0E00023FB7334
:1066EC003EE0FA7B796813469B001344DB000B44B5
:1066FC00113301221A70FA7B796813469B001344FC
:10670C00DB000B441033FA7B1A70FA7B7968134662
:10671C009B001344DB000B44133300221A70FA7BEA
:10672C00796813469B001344DB000B442033002292
:10673C001A60FA7B796813469B001344DB000B4408
:10674C00243300221A60FB7B79685A1C13469B0089
:10675C001344DB000B4400221A60FB7B0133FB73F8
:10676C007B681B79FA7B9A42BBD30023FB7344E012
:10677C00FA7B796813469B001344DB000B4403F24D
:10678C00511300221A70FA7B796813469B0013444C
:10679C00DB000B4403F5A873FA7B1A70FA7B79685B
:1067AC0013469B001344DB000B4403F253130022EB
:1067BC001A70FA7B796813469B001344DB000B4478
:1067CC0003F5B07300221A60FA7B796813469B00BC
:1067DC001344DB000B4403F5B27300221A60FA7BFE
:1067EC00796813469B001344DB000B4403F5B47328
:1067FC0000221A60FB7B0133FB737B681B79FA7BED
:10680C009A42B5D37B6818687B6804330ECB03F0CF
:10681C0028FA0346002B05D07B68022283F89122CC
:10682C0001230CE07B6800225A737B68012283F8F9
:10683C0091227B681B68184605F0A7FC00231846BC
:10684C001037BD4680BD80B582B000AF78607B68E4
:10685C0093F89032012B01D1022316E07B680122C0
:10686C0083F890227B681B68184603F0BEF901215F
:10687C00786807F092FD7B681B68184605F07BFC76
:10688C007B68002283F89022002318460837BD4607
:10689C0080BD80B588B000AF78607B681B681846F7
:1068AC0005F07DFCB861BB6903F40043002B03D0F9
:1068BC00786800F01AFB19E1BB6903F48063002BC4
:1068CC0013D07B681B68B3F844309AB27B681B68A2
:1068DC0022F4806292B2A3F84420786807F065FB3A
:1068EC000021786800F005F900E1BB6903F48043EE
:1068FC00002B0CD07B681B68B3F844309AB27B68D1
:10690C001B6822F4804292B2A3F84420EEE0BB69EB
:10691C0003F40053002B0CD07B681B68B3F8443095
:10692C009AB27B681B6822F4005292B2A3F84420FE
:10693C00DCE0BB6903F48053002B27D07B681B6819
:10694C00B3F840309AB27B681B6822F0040292B212
:10695C00A3F840207B681B68B3F840309AB27B6880
:10696C001B6822F0080292B2A3F84020786807F066
:10697C0055FB7B681B68B3F844309AB27B681B6884
:10698C0022F4805292B2A3F84420AFE0BB6903F426
:10699C000063002B00F083800023FB7710E07B6802
:1069AC001B681A46FB7F9B001A44FB7F128892B22D
:1069BC005B0020333B4423F8182CFB7F0133FB771F
:1069CC00FB7F072BEBD97B681B68B3F840309AB27E
:1069DC007B681B6842F0010292B2A3F840207B68EE
:1069EC001B68B3F840309AB27B681B6822F0010236
:1069FC0092B2A3F8402000BF7B681B68B3F8443008
:106A0C009BB203F48063002BF6D07B681B68B3F851
:106A1C0044309AB27B681B6822F4806292B2A3F86D
:106A2C0044200023FB770FE0FB7F7A681268114645
:106A3C00FA7F92000A445B0020333B4433F8183C45
:106A4C001380FB7F0133FB77FB7F072BECD97B6833
:106A5C001B68B3F840309AB27B681B6842F008029E
:106A6C0092B2A3F840207B681B68B3F844309AB20A
:106A7C007B681B6822F4006292B2A3F844207B6806
:106A8C001B68B3F840309AB27B681B6842F0040272
:106A9C0092B2A3F84020786807F0A6FA26E0BB690A
:106AAC0003F40073002B0FD07B681B68B3F84430E1
:106ABC009AB27B681B6822F4007292B2A3F844204D
:106ACC00786807F064FA11E0BB6903F48073002B5B
:106ADC000CD07B681B68B3F844309AB27B681B6897
:106AEC0022F4807292B2A3F8442000BF2037BD4636
:106AFC0080BD80B582B000AF78600B46FB707B68C0
:106B0C0093F89032012B01D1022312E07B68012211
:106B1C0083F890227B68FA785A737B681B68FA7842
:106B2C001146184605F014FB7B68002283F890226E
:106B3C00002318460837BD4680BD80B584B000AF31
:106B4C007860084611461A460346FB700B463B809C
:106B5C001346BB700023FB7297F90330002B0EDA3F
:106B6C00FB7803F0070213469B001344DB00103341
:106B7C007A681344FB60FB6801225A700EE0FB78C4
:106B8C0003F0070213469B001344DB0003F5A873C4
:106B9C007A681344FB60FB6800225A70FB7803F0A0
:106BAC000703DAB2FB681A703A88FB681A61FB6853
:106BBC00BA78DA70BB78022B02D1FB6800221A710A
:106BCC007B6893F89032012B01D102230EE07B6895
:106BDC00012283F890227B681B68F968184603F041
:106BEC005DF87B68002283F89022FB7A18461037F8
:106BFC00BD4680BD80B584B000AF78600B46FB709D
:106C0C0097F90330002B0EDAFB7803F007021346DA
:106C1C009B001344DB0010337A681344FB60FB6861
:106C2C0001225A700EE0FB7803F0070213469B001A
:106C3C001344DB0003F5A8737A681344FB60FB680C
:106C4C0000225A70FB7803F00703DAB2FB681A7063
:106C5C007B6893F89032012B01D102230EE07B6804
:106C6C00012283F890227B681B68F968184603F0B0
:106C7C00D5FB7B68002283F890220023184610373E
:106C8C00BD4680BD80B586B000AFF8607A603B60D1
:106C9C000B46FB72FB7A03F0070213469B0013446E
:106CAC00DB0003F5A873FA6813447B617B697A688F
:106CBC005A617B693A689A617B690022DA617B6967
:106CCC0000225A70FB7A03F00703DAB27B691A7060
:106CDC00FB681B687969184603F08CFD0023184685
:106CEC001837BD4680BD80B483B000AF78600B46CA
:106CFC00FB70FB7803F00702796813469B00134482
:106D0C00DB000B4403F5B6731B6818460C37BD4605
:106D1C0080BC704780B586B000AFF8607A603B608D
:106D2C000B46FB72FB7A03F0070213469B001344DD
:106D3C00DB001033FA6813447B617B697A685A6113
:106D4C007B693A689A617B69012283F824207B690C
:106D5C003A681A627B690022DA617B6901225A70F7
:106D6C00FB7A03F00703DAB27B691A70FB681B68C5
:106D7C007969184603F03EFD002318461837BD46C6
:106D8C0080BD80B584B000AF78600B46FB70FB789B
:106D9C0003F007037A681279934201D901234CE07E
:106DAC0097F90330002B0EDAFB7803F00702134639
:106DBC009B001344DB0010337A681344FB60FB68C0
:106DCC0001225A700CE0FA7813469B001344DB0046
:106DDC0003F5A8737A681344FB60FB6800225A70B1
:106DEC00FB6801229A70FB7803F00703DAB2FB68A8
:106DFC001A707B6893F89032012B01D102231CE0AE
:106E0C007B68012283F890227B681B68F96818461E
:106E1C0005F0A1F8FB7803F00703002B08D17B6881
:106E2C001A687B6803F526731946104605F0C6F9F7
:106E3C007B68002283F89022002318461037BD4649
:106E4C0080BD80B584B000AF78600B46FB70FB78DA
:106E5C0003F00F037A681279934201D9012340E0C1
:106E6C0097F90330002B0EDAFB7803F00702134678
:106E7C009B001344DB0010337A681344FB60FB68FF
:106E8C0001225A700EE0FB7803F0070213469B00B8
:106E9C001344DB0003F5A8737A681344FB60FB68AA
:106EAC0000225A70FB6800229A70FB7803F00703EB
:106EBC00DAB2FB681A707B6893F89032012B01D11F
:106ECC0002230EE07B68012283F890227B681B680A
:106EDC00F968184605F08FF87B68002283F8902239
:106EEC00002318461037BD4680BD80B596B000AF64
:106EFC007860BBE37B681B68B3F84430A7F84E306E
:106F0C00B7F84E30DBB203F00F0387F84D3097F82B
:106F1C004D30002B40F07581B7F84E3003F0100364
:106F2C00002B4ED17B681B681B889BB223F4E1437A
:106F3C0023F07003FB817B681A68FB896FEA43437B
:106F4C006FEA53439BB213807B6810337B657B687D
:106F5C001B68B3F850309BB21A467B6D1B78DB0074
:106F6C00134402335B007A681268134403F58063A0
:106F7C001B88C3F309027B6DDA617B6D5A697B6DEB
:106F8C00DB691A447B6D5A610021786806F0E5FFD5
:106F9C007B685B7BDBB2002B00F068837B6D9B69AD
:106FAC00002B40F063837B685B7BDBB263F07F0379
:106FBC00DAB27B681B68A3F84C207B6800225A73FA
:106FCC0054E37B6803F5A8737B657B681B681B889F
:106FDC00A7F84A30B7F84A3003F40063002B34D0DA
:106FEC007B681B68B3F850309BB21A467B6D1B78DC
:106FFC00DB00134406335B007A681268134403F514
:10700C0080631B88C3F309027B6DDA617B681868A7
:10701C007B6803F526717B6DDA887B6DDB699BB22F
:10702C0005F01DF97B681B681B889AB240F68F73BC
:10703C0013403B827B681B683A8A42F0800292B212
:10704C001A80786806F05CFF10E3B7F94A30002B21
:10705C0080F20C837B681B681B889AB240F68F7396
:10706C001340FB837B681B68FA8B42F0800292B260
:10707C001A807B681B68B3F850309BB21A467B6D44
:10708C001B78DB00134406335B007A6812681344E8
:10709C0003F580631B88C3F309027B6DDA617B6D9A
:1070AC00DB69002B19D07B6D5B69002B15D07B68DD
:1070BC0018687B6D59697B6DDA887B6DDB699BB2D7
:1070CC0005F0CDF87B6D5A697B6DDB691A447B6DDD
:1070DC005A610021786806F025FF7B681B681B88C5
:1070EC00A7F84A30B7F84A3003F40063002B40F09D
:1070FC00BD82B7F84A3003F44053B3F5405F00F05B
:10710C00B5827B681B68BB617B681B68B3F8503029
:10711C009BB21A46BB691344BB61BB6903F20C43B7
:10712C007B617B691B889BB2C3F309039AB27B69B1
:10713C001A807B6D1B693E2B1DD97B6D1B695B090E
:10714C007B647B6D1B6903F01F03002B02D17B6CEE
:10715C00013B7B647B691B889AB27B6C9BB29B0264
:10716C009BB213439BB26FEA43436FEA53439AB209
:10717C007B691A8026E07B6D1B69002B0AD17B6929
:10718C001B889BB26FEA43436FEA53439AB27B6905
:10719C001A8017E07B6D1B695B087B647B6D1B6938
:1071AC0003F00103002B02D07B6C01337B647B6901
:1071BC001B889AB27B6C9BB29B029BB213439AB214
:1071CC007B691A807B681B681B889BB223F4804305
:1071DC0023F070037B827B8A83F480537B827B8ACF
:1071EC0083F400537B827B681A687B8A43F07F436D
:1071FC0043F47F0343F4004343F080039BB21380BA
:10720C0034E27B681B681A4697F84D309B00134498
:10721C001B88A7F84A30B7F94A30002B80F2FC8063
:10722C007B681B681A4697F84D309B0013441B88EB
:10723C009AB240F68F731340A7F848307B681B68EE
:10724C001A4697F84D309B001344B7F8482042F08B
:10725C00800292B21A8097F84D2013469B0013447B
:10726C00DB0003F5A8737A6813447B657B6D1B7B8D
:10727C00002B25D17B681B68B3F850309BB21A46A3
:10728C007B6D1B78DB00134406335B007A68126855
:10729C00134403F580631B88C3F30903A7F850302C
:1072AC00B7F85030002B00F092807B6818687B6D2B
:1072BC0059697B6DDA88B7F8503004F0D0FF86E05E
:1072CC007B6DDB78022B0AD1B7F84A301A46796D00
:1072DC00786800F0D9F90346A7F8503077E07B685E
:1072EC001B681A467B6D1B789B0013441B889BB252
:1072FC0023F4E04323F07003A7F852307B681B683B
:10730C001A467B6D1B789B001A44B7F8523043F039
:10731C007F4343F47F0343F4004343F0C0039BB229
:10732C0013807B681B681A467B6D1B789B0013448B
:10733C001B889BB203F48043002B24D07B681B6812
:10734C00B3F850309BB21A467B6D1B78DB001344AC
:10735C0002335B007A681268134403F580631B8860
:10736C00C3F30903A7F85030B7F85030002B2ED0D8
:10737C007B6818687B6D59697B6D1A89B7F850303A
:10738C0004F06DFF23E07B681B68B3F850309BB2B0
:10739C001A467B6D1B78DB00134406335B007A685E
:1073AC001268134403F580631B88C3F30903A7F821
:1073BC005030B7F85030002B09D07B6818687B6DC3
:1073CC0059697B6D5A89B7F8503004F048FF7B6DD2
:1073DC00DA69B7F850301A447B6DDA617B6D5A6903
:1073EC00B7F850301A447B6D5A617B6D9B69002B4A
:1073FC0005D0B7F850207B6D1B699A4206D27B6D85
:10740C001B781946786806F08DFD05E07B681B68D3
:10741C00796D184603F0EEF9B7F84A3003F08003A3
:10742C00002B00F0238197F84D2013469B0013444A
:10743C00DB0010337A6813447B657B681B681A4643
:10744C0097F84D309B0013441B889BB223F4E14307
:10745C0023F07003A7F842307B681B681A4697F834
:10746C004D309B001A44B7F842306FEA43436FEA41
:10747C0053439BB213807B6DDB78012B40F0A280D1
:10748C007B6D00229A617B6D1B7B002B00F093803F
:10749C00B7F84A3003F04003002B46D07B6D5B7885
:1074AC00002B26D17B681B687B627B681B68B3F85A
:1074BC0050309BB21A467B6A13447B627B6D1B78FF
:1074CC001A017B6A134403F204433B623B6A1B8838
:1074DC009BB2C3F309039AB23B6A1A803B6A1B88BE
:1074EC009BB26FEA43436FEA53439AB23B6A1A80EA
:1074FC0061E07B6D5B78012B5DD17B681B68FB6267
:10750C007B681B68B3F850309BB21A46FB6A134475
:10751C00FB627B6D1B781A01FB6A134403F2044374
:10752C00BB62BB6A00221A8045E07B681B68FB6368
:10753C007B6D5B78002B26D17B681B687B637B683B
:10754C001B68B3F850309BB21A467B6B13447B63B9
:10755C007B6D1B781A017B6B134403F20C433B636A
:10756C003B6B1B889BB2C3F309039AB23B6B1A802B
:10757C003B6B1B889BB26FEA43436FEA53439AB24F
:10758C003B6B1A8017E07B6D5B78012B13D17B680A
:10759C001B68B3F850309BB21A46FB6B1344FB6369
:1075AC007B6D1B781A01FB6B134403F20C43BB631A
:1075BC00BB6B00221A807B6D1B781946786806F02D
:1075CC00CCFC53E0B7F84A3003F48073002B46D15F
:1075DC007B681B68B3F850309BB21A467B6D1B78E6
:1075EC00DB00134402335B007A681268134403F522
:1075FC0080631B88C3F30903A7F840307B6D9A693D
:10760C00B7F840309A4207D97B6D9A69B7F8403089
:10761C00D21A7B6D9A6102E07B6D00229A617B6DC0
:10762C009B69002B06D17B6D1B781946786806F098
:10763C0094FC1BE07B6D5A69B7F840301A447B6DA3
:10764C005A617B6DDA69B7F840301A447B6DDA61A8
:10765C007B681B68796D184603F0CCF806E0B7F828
:10766C004A301A46796D786800F01BF97B681B6804
:10767C00B3F844309BB21BB2002BFFF63BAC00239B
:10768C0018465837BD4680BD80B588B000AFF8604D
:10769C00B9601346FB80FB8803F48043002B7ED03B
:1076AC00FB681B68B3F850309BB21A46BB681B785A
:1076BC00DB00134402335B00FA681268134403F5D1
:1076CC0080631B88C3F309037B83BB689A697B8B3C
:1076DC009A4206D3BB689A697B8BD21ABB689A61B3
:1076EC0002E0BB6800229A61BB689B69002B23D126
:1076FC00FB681B681A46BB681B789B0013441B88ED
:10770C009BB223F4804323F070033B833B8B83F4C5
:10771C0000533B83FB681B681A46BB681B789B00B5
:10772C001A443B8B43F07F4343F47F0343F4004301
:10773C0043F080039BB21380FB8803F04003002BC3
:10774C001FD0FB681B681A46BB681B789B00134450
:10775C001B889BB223F4E04323F07003FB82FB688D
:10776C001B681A46BB681B789B001A44FB8A43F0C3
:10777C007F4343F47F0343F4004343F0C0039BB2C5
:10778C0013807B8B002B00F08780FB681868BB682C
:10779C005969BB681A897B8B04F061FD7CE0FB683E
:1077AC001B68B3F850309BB21A46BB681B78DB00E1
:1077BC00134406335B00FA681268134403F58063C4
:1077CC001B88C3F309037B83BB689A697B8B9A4242
:1077DC0006D3BB689A697B8BD21ABB689A6102E0AC
:1077EC00BB6800229A61BB689B69002B23D1FB68A4
:1077FC001B681A46BB681B789B0013441B889BB202
:10780C0023F4804323F07003FB83FB8B83F400533E
:10781C00FB83FB681B681A46BB681B789B001A44E9
:10782C00FB8B43F07F4343F47F0343F4004343F06B
:10783C0080039BB21380FB8803F04003002B1FD105
:10784C00FB681B681A46BB681B789B0013441B889B
:10785C009BB223F4E04323F07003BB83FB681B68EB
:10786C001A46BB681B789B001A44BB8B43F07F43C2
:10787C0043F47F0343F4004343F0C0039BB21380F3
:10788C007B8B002B08D0FB681868BB685969BB68F8
:10789C005A897B8B04F0E3FC7B8B18462037BD4662
:1078AC0080BD80B5A4B000AFF860B9601346FB8012
:1078BC00FB8803F04003002B00F0DD81FB681B68A4
:1078CC00B3F850309BB21A46BB681B78DB001344EC
:1078DC0002335B00FA681268134403F580631B885B
:1078EC00C3F30903A7F88630BB689A69B7F88630EA
:1078FC009A4207D9BB689A69B7F88630D21ABB6826
:10790C009A6102E0BB6800229A61BB689B69002BFC
:10791C0040F0B980BB685B78002B26D1FB681B68F4
:10792C00FB62FB681B68B3F850309BB21A46FB6ACB
:10793C001344FB62BB681B781A01FB6A134403F205
:10794C000443BB62BB6A1B889BB2C3F309039AB2A4
:10795C00BB6A1A80BB6A1B889BB26FEA43436FEA0F
:10796C0053439AB2BB6A1A801AE0BB685B78012B4E
:10797C0016D1FB681B687B63FB681B68B3F850303F
:10798C009BB21A467B6B13447B63BB681B781A0152
:10799C007B6B134403F204433B633B6B00221A8062
:1079AC00FB681B687B62BB685B78002B26D1FB688D
:1079BC001B68FB61FB681B68B3F850309BB21A461E
:1079CC00FB691344FB61BB681B781A01FB69134408
:1079DC0003F20C43BB61BB691B889BB2C3F3090365
:1079EC009AB2BB691A80BB691B889BB26FEA43438E
:1079FC006FEA53439AB2BB691A8017E0BB685B7895
:107A0C00012B13D1FB681B68B3F850309BB21A469C
:107A1C007B6A13447B62BB681B781A017B6A134434
:107A2C0003F20C433B623B6A00221A80BB681B7852
:107A3C001946F86806F091FAFB8803F48043002B92
:107A4C0000F0FC82FB681B681A46BB681B789B0025
:107A5C0013441B889BB223F4E04323F07003FB8296
:107A6C00FB681B681A46BB681B789B001A44FB8A90
:107A7C0043F07F4343F47F0343F4404343F08003DC
:107A8C009BB21380DAE2FB8803F48043002B21D0F5
:107A9C00FB681B681A46BB681B789B0013441B8849
:107AAC009BB223F4E04323F07003A7F88A30FB6801
:107ABC001B681A46BB681B789B001A44B7F88A30BF
:107ACC0043F07F4343F47F0343F4404343F080038C
:107ADC009BB21380BB6893F82430012B40F0AE822C
:107AEC00BB685A69B7F886301A44BB685A61BB68E0
:107AFC00DA69B7F886301A44BB68DA61BB681A6A6F
:107B0C00BB681B699A420BD3BB681B69C7F88C30E6
:107B1C00BB681A6AD7F88C30D21ABB681A6217E0A5
:107B2C00BB681B6A002B08D1B7F88630C7F88C30BD
:107B3C00BB68002283F824200AE0BB68002283F88B
:107B4C002420BB681B6AC7F88C30BB6800221A6201
:107B5C00BB685B78002B65D1FB681B68FB63FB681B
:107B6C001B68B3F850309BB21A46FB6B1344FB6393
:107B7C00BB681B781A01FB6B134403F20443BB6311
:107B8C00BB6B1B889BB2C3F309039AB2BB6B1A8005
:107B9C00D7F88C303E2B1DD9D7F88C305B09BB64E1
:107BAC00D7F88C3003F01F03002B02D1BB6C013BC8
:107BBC00BB64BB6B1B889AB2BB6C9BB29B029BB227
:107BCC0013439BB26FEA43436FEA53439AB2BB6BC6
:107BDC001A8044E0D7F88C30002B0AD1BB6B1B8881
:107BEC009BB26FEA43436FEA53439AB2BB6B1A8062
:107BFC0035E0D7F88C305B08BB64D7F88C3003F0D9
:107C0C000103002B02D0BB6C0133BB64BB6B1B8824
:107C1C009AB2BB6C9BB29B029BB213439AB2BB6BE6
:107C2C001A801CE0BB685B78012B18D1FB681B68C1
:107C3C007B64FB681B68B3F850309BB21A467B6CB4
:107C4C0013447B64BB681B781A017B6C134403F2EE
:107C5C0004433B64D7F88C309AB23B6C1A80FB68B7
:107C6C001868BB685969BB681A89D7F88C309BB205
:107C7C0004F0AFFAE2E1FB681B68B3F850309BB23A
:107C8C001A46BB681B78DB00134406335B00FA68AA
:107C9C001268134403F580631B88C3F30903A7F828
:107CAC008630BB689A69B7F886309A4207D3BB68AE
:107CBC009A69B7F88630D21ABB689A6102E0BB6841
:107CCC0000229A61BB689B69002B40F0C080BB68A6
:107CDC005B78002B26D1FB681B68FB67FB681B6875
:107CEC00B3F850309BB21A46FB6F1344FB67BB686A
:107CFC001B781A01FB6F134403F20443BB67BB6F81
:107D0C001B889BB2C3F309039AB2BB6F1A80BB6F7B
:107D1C001B889BB26FEA43436FEA53439AB2BB6F23
:107D2C001A801AE0BB685B78012B16D1FB681B68C4
:107D3C007B66FB681B68B3F850309BB21A467B6EAF
:107D4C0013447B66BB681B781A017B6E134403F2E9
:107D5C0004433B663B6E00221A80FB681B687B6702
:107D6C00BB685B78002B2BD1FB681B68FB66FB6840
:107D7C001B68B3F850309BB21A46FB6E1344FB667B
:107D8C00BB681B781A01FB6E134403F20C43C7F853
:107D9C008030D7F880301B889BB2C3F309039AB2AA
:107DAC00D7F880301A80D7F880301B889BB26FEAE6
:107DBC0043436FEA53439AB2D7F880301A8017E0E6
:107DCC00BB685B78012B13D1FB681B68B3F8503090
:107DDC009BB21A467B6F13447B67BB681B781A01F6
:107DEC007B6F134403F20C433B673B6F00221A80FA
:107DFC00BB681B781946F86806F0AFF8FB8803F4EB
:107E0C008043002B40F01A81FB681B681A46BB6844
:107E1C001B789B0013441B889BB223F4E04323F094
:107E2C007003A7F88830FB681B681A46BB681B7880
:107E3C009B001A44B7F8883043F07F4343F47F0328
:107E4C0043F4404343F080039BB21380F6E0FB887D
:107E5C0003F48043002B21D1FB681B681A46BB68D6
:107E6C001B789B0013441B889BB223F4E04323F044
:107E7C007003A7F84E30FB681B681A46BB681B786A
:107E8C009B001A44B7F84E3043F07F4343F47F0312
:107E9C0043F4404343F080039BB21380BB6893F8D8
:107EAC002430012B40F0CA80BB685A69B7F8863081
:107EBC001A44BB685A61BB68DA69B7F886301A4451
:107ECC00BB68DA61BB681A6ABB681B699A420BD340
:107EDC00BB681B69C7F88C30BB681A6AD7F88C3042
:107EEC00D21ABB681A6217E0BB681B6A002B08D158
:107EFC00B7F88630C7F88C30BB68002283F8242092
:107F0C000AE0BB681B6AC7F88C30BB6800221A6297
:107F1C00BB68002283F82420FB681B687B65BB6868
:107F2C005B78002B65D1FB681B68FB65FB681B68E5
:107F3C00B3F850309BB21A46FB6D1344FB65BB681B
:107F4C001B781A01FB6D134403F20C43BB65BB6D2C
:107F5C001B889BB2C3F309039AB2BB6D1A80D7F886
:107F6C008C303E2B1DD9D7F88C305B09BB66D7F80B
:107F7C008C3003F01F03002B02D1BB6E013BBB66A0
:107F8C00BB6D1B889AB2BB6E9BB29B029BB2134318
:107F9C009BB26FEA43436FEA53439AB2BB6D1A80AC
:107FAC0041E0D7F88C30002B0AD1BB6D1B889BB2FB
:107FBC006FEA43436FEA53439AB2BB6D1A8032E0C7
:107FCC00D7F88C305B08BB66D7F88C3003F0010314
:107FDC00002B02D0BB6E0133BB66BB6D1B889AB203
:107FEC00BB6E9BB29B029BB213439AB2BB6D1A80C1
:107FFC0019E0BB685B78012B15D1FB681B68B3F8E3
:10800C0050309BB21A467B6D13447B65BB681B7862
:10801C001A017B6D134403F20C433B65D7F88C308B
:10802C009AB23B6D1A80FB681868BB685969BB68CB
:10803C005A89D7F88C309BB204F0CBF8FB681B68DC
:10804C001A46BB681B789B0013441B889BB223F415
:10805C00E04323F04003BB82BB8A83F01003BB8256
:10806C00BB8A83F02003BB82FB681B681A46BB6883
:10807C001B789B001A44BB8A43F07F4343F47F0375
:10808C0043F4004343F080039BB213800023184653
:10809C009037BD4680BD80B487B000AFF8607B6080
:1080AC000B467B8113463B817B8903F080039BB29B
:1080BC00002B0BD07B8903F0070213469B00134463
:1080CC00DB001033FA6813447B6109E07A891346AC
:1080DC009B001344DB0003F5A873FA6813447B611F
:1080EC003B89002B07D17B6900221A737B689AB2FB
:1080FC007B69DA800BE07B6901221A737B689AB288
:10810C007B691A817B681B0C9AB27B695A810023AC
:10811C0018461C37BD4680BC7047000080B586B041
:10812C0000AF78607B68002B01D1012372E27B6881
:10813C001B6803F00103002B00F08780924B5B68F7
:10814C0003F00C03042B0CD08F4B5B6803F00C0377
:10815C00082B12D18C4B5B6803F48033B3F5803F52
:10816C000BD1894B1B6803F40033002B6CD07B685C
:10817C005B68002B68D101234CE27B685B68B3F52C
:10818C00803F06D1804B1B687F4A43F480331360D9
:10819C002EE07B685B68002B0CD17B4B1B687A4A0A
:1081AC0023F480331360784B1B68774A23F48023C5
:1081BC0013601DE07B685B68B3F5A02F0CD1724B8C
:1081CC001B68714A43F4802313606F4B1B686E4A23
:1081DC0043F4803313600BE06B4B1B686A4A23F447
:1081EC0080331360684B1B68674A23F48023136049
:1081FC007B685B68002B13D0FCF7A4FF386108E0A8
:10820C00FCF7A0FF02463B69D31A642B01D9032368
:10821C0000E25D4B1B6803F40033002BF0D014E03C
:10822C00FCF790FF386108E0FCF78CFF02463B69D5
:10823C00D31A642B01D90323ECE1534B1B6803F4D1
:10824C000033002BF0D100E000BF7B681B6803F00B
:10825C000203002B63D04C4B5B6803F00C03002B28
:10826C000BD0494B5B6803F00C03082B1CD1464B1D
:10827C005B6803F48033002B16D1434B1B6803F06F
:10828C000203002B05D07B681B69012B01D0012355
:10829C00C0E13D4B1B6823F0F8027B685B69DB0097
:1082AC00394913430B603AE07B681B69002B20D0E3
:1082BC00364B01221A60FCF745FF386108E0FCF7E9
:1082CC0041FF02463B69D31A022B01D90323A1E1DA
:1082DC002D4B1B6803F00203002BF0D02A4B1B68BC
:1082EC0023F0F8027B685B69DB00274913430B60C2
:1082FC0015E0264B00221A60FCF724FF386108E0D9
:10830C00FCF720FF02463B69D31A022B01D9032349
:10831C0080E11D4B1B6803F00203002BF0D17B683E
:10832C001B6803F00803002B3AD07B689B69002B79
:10833C0019D0174B01221A60FCF704FF386108E0D2
:10834C00FCF700FF02463B69D31A022B01D9032329
:10835C0060E10D4B5B6A03F00203002BF0D00120AF
:10836C0000F0D0FA1CE00A4B00221A60FCF7EAFE7F
:10837C0038610FE0FCF7E6FE02463B69D31A022B8C
:10838C0008D9032346E100BF00100240000042421E
:10839C0080044242924B5B6A03F00203002BE9D14A
:1083AC007B681B6803F00403002B00F0A6800023FD
:1083BC00FB758B4BDB6903F08053002B0DD1884B85
:1083CC00DB69874A43F08053D361854BDB6903F04B
:1083DC008053BB60BB680123FB75824B1B6803F4A5
:1083EC008073002B18D17F4B1B687E4A43F480733B
:1083FC001360FCF7A7FE386108E0FCF7A3FE024609
:10840C003B69D31A642B01D9032303E1754B1B6819
:10841C0003F48073002BF0D07B68DB68012B06D152
:10842C006F4B1B6A6E4A43F0010313622DE07B68AD
:10843C00DB68002B0CD16A4B1B6A694A23F00103E1
:10844C001362674B1B6A664A23F0040313621CE039
:10845C007B68DB68052B0CD1614B1B6A604A43F0CF
:10846C00040313625E4B1B6A5D4A43F00103136203
:10847C000BE05B4B1B6A5A4A23F001031362584B07
:10848C001B6A574A23F0040313627B68DB68002BDA
:10849C0015D0FCF757FE38610AE0FCF753FE024694
:1084AC003B69D31A41F28832934201D90323B1E0DC
:1084BC004B4B1B6A03F00203002BEED014E0FCF7CD
:1084CC0041FE38610AE0FCF73DFE02463B69D31AD7
:1084DC0041F28832934201D903239BE0404B1B6A43
:1084EC0003F00203002BEED1FB7D012B05D13C4B9D
:1084FC00DB693B4A23F08053D3617B68DB69002B3B
:10850C0000F08780364B5B6803F00C03082B61D0BE
:10851C007B68DB69022B46D1334B00221A60FCF7D7
:10852C0011FE386108E0FCF70DFE02463B69D31AD8
:10853C00022B01D903236DE0294B1B6803F0007358
:10854C00002BF0D17B681B6AB3F5803F08D1244B1C
:10855C005B6823F400327B689B68214913434B60B2
:10856C001F4B5B6823F474127B68196A7B685B6A27
:10857C000B431B4913434B601B4B01221A60FCF746
:10858C00E1FD386108E0FCF7DDFD02463B69D31ADA
:10859C00022B01D903233DE0114B1B6803F0007340
:1085AC00002BF0D035E0104B00221A60FCF7CAFD0E
:1085BC00386108E0FCF7C6FD02463B69D31A022B72
:1085CC0001D9032326E0064B1B6803F00073002B34
:1085DC00F0D11EE07B68DB69012B07D1012319E088
:1085EC000010024000700040600042420B4B5B6880
:1085FC00FB60FB6803F480327B681B6A9A4206D1ED
:10860C00FB6803F470127B685B6A9A4201D0012309
:10861C0000E0002318461837BD4680BD001002400C
:10862C0080B584B000AF786039607B68002B01D1D5
:10863C000123D0E06A4B1B6803F007033A689A42A7
:10864C0010D9674B1B6823F0070265493B6813433D
:10865C000B60634B1B6803F007033A689A4201D026
:10866C000123B8E07B681B6803F00203002B20D0C9
:10867C007B681B6803F00403002B05D0594B5B6827
:10868C00584A43F4E06353607B681B6803F00803AB
:10869C00002B05D0534B5B68524A43F46053536034
:1086AC00504B5B6823F0F0027B689B684D49134389
:1086BC004B607B681B6803F00103002B40D07B6888
:1086CC005B68012B07D1474B1B6803F40033002B6D
:1086DC0015D101237FE07B685B68022B07D1414BEE
:1086EC001B6803F00073002B09D1012373E03D4B91
:1086FC001B6803F00203002B01D101236BE0394B03
:10870C005B6823F003027B685B68364913434B605C
:10871C00FCF718FDF8600AE0FCF714FD0246FB6854
:10872C00D31A41F28832934201D9032353E02D4BE3
:10873C005B6803F00C027B685B689B009A42EBD190
:10874C00274B1B6803F007033A689A4210D2244B5C
:10875C001B6823F0070222493B6813430B60204B34
:10876C001B6803F007033A689A4201D0012332E0F8
:10877C007B681B6803F00403002B08D0194B5B6863
:10878C0023F4E0627B68DB68164913434B607B681B
:10879C001B6803F00803002B09D0124B5B6823F411
:1087AC0060527B681B69DB000E4913434B6000F081
:1087BC0021F802460B4B5B681B0903F00F030A49B7
:1087CC00CB5C22FA03F3094A1360094B1B68184669
:1087DC00FCF776FC002318461037BD4680BD00BF61
:1087EC00002002400010024018F500081000002084
:1087FC001400002080B487B000AF0023FB6000237E
:10880C00BB6000237B6100237B6000233B611E4B1C
:10881C005B68FB60FB6803F00C03042B02D0082B95
:10882C0003D027E0194B3B6127E0FB689B0C03F05E
:10883C000F03174AD35C7B60FB6803F48033002B77
:10884C0010D0114B5B685B0C03F00103114AD35C35
:10885C00BB607B680D4A03FB02F2BB68B2FBF3F30F
:10886C007B6104E07B680C4A02FB03F37B617B6950
:10887C003B6102E0094B3B6100BF3B6918461C376A
:10888C00BD4680BC704700BF00100240001BB70003
:10889C0030F5000840F5000800093D0000127A0090
:1088AC0080B400AF024B1B681846BD4680BC7047B5
:1088BC001000002080B500AFFFF7F2FF0246054B19
:1088CC005B681B0A03F007030349CB5C22FA03F332
:1088DC00184680BD0010024028F5000880B500AF96
:1088EC00FFF7DEFF0246054B5B68DB0A03F007036C
:1088FC000349CB5C22FA03F3184680BD00100240FA
:10890C0028F5000880B485B000AF78600A4B1B686E
:10891C000A4AA2FB03235B0A7A6802FB03F3FB609F
:10892C0000BFFB685A1EFA60002BF9D100BF00BFD4
:10893C001437BD4680BC704710000020D34D621028
:10894C0080B586B000AF786000233B610023FB60EC
:10895C007B681B6803F00103002B7DD00023FB75A3
:10896C004F4BDB6903F08053002B0DD14C4BDB6973
:10897C004B4A43F08053D361494BDB6903F080537E
:10898C00BB60BB680123FB75464B1B6803F480730B
:10899C00002B18D1434B1B68424A43F4807313607D
:1089AC00FCF7D0FB386108E0FCF7CCFB02463B69D6
:1089BC00D31A642B01D903236DE03A4B1B6803F4E3
:1089CC008073002BF0D0364B1B6A03F44073FB60B2
:1089DC00FB68002B2ED07B685B6803F44073FA684D
:1089EC009A4227D02E4B1B6A23F44073FB602E4B0C
:1089FC0001221A602C4B00221A60294AFB68136270
:108A0C00FB6803F00103002B14D0FCF79BFB3861CF
:108A1C000AE0FCF797FB02463B69D31A41F2883215
:108A2C00934201D9032336E01D4B1B6A03F002036A
:108A3C00002BEED01A4B1B6A23F440727B685B68E8
:108A4C00174913430B62FB7D012B05D1144BDB69DA
:108A5C00134A23F08053D3617B681B6803F0020335
:108A6C00002B08D00E4B5B6823F440427B689B685C
:108A7C000B4913434B607B681B6803F01003002BFE
:108A8C0008D0074B5B6823F480027B68DB680449E1
:108A9C0013434B60002318461837BD4680BD00BFFA
:108AAC0000100240007000404004424280B582B089
:108ABC0000AF78607B68002B01D1012341E07B681B
:108ACC0093F83D30DBB2002B06D17B68002283F893
:108ADC003C207868FCF76AF97B68022283F83D2019
:108AEC007B681A687B6804331946104600F03EFB1D
:108AFC007B68012283F846207B68012283F83E20A4
:108B0C007B68012283F83F207B68012283F8402098
:108B1C007B68012283F841207B68012283F8422084
:108B2C007B68012283F843207B68012283F8442070
:108B3C007B68012283F845207B68012283F83D2065
:108B4C00002318460837BD4680BD80B582B000AF03
:108B5C0078607B68002B01D1012341E07B6893F89E
:108B6C003D30DBB2002B06D17B68002283F83C2021
:108B7C00786800F039F87B68022283F83D207B6826
:108B8C001A687B6804331946104600F0EFFA7B68CC
:108B9C00012283F846207B68012283F83E207B6803
:108BAC00012283F83F207B68012283F840207B68F8
:108BBC00012283F841207B68012283F842207B68E4
:108BCC00012283F843207B68012283F844207B68D0
:108BDC00012283F845207B68012283F83D20002385
:108BEC0018460837BD4680BD80B483B000AF7860AE
:108BFC0000BF0C37BD4680BC7047000080B584B008
:108C0C0000AF786039603B68002B09D17B6893F822
:108C1C003E30DBB2012B14BF01230023DBB222E078
:108C2C003B68042B09D17B6893F83F30DBB2012BF6
:108C3C0014BF01230023DBB215E03B68082B09D1DC
:108C4C007B6893F84030DBB2012B14BF0123002367
:108C5C00DBB208E07B6893F84130DBB2012B14BF28
:108C6C0001230023DBB2002B01D001235EE03B6823
:108C7C00002B04D17B68022283F83E2013E03B6872
:108C8C00042B04D17B68022283F83F200BE03B6865
:108C9C00082B04D17B68022283F8402003E07B6818
:108CAC00022283F841207B681B6801223968184630
:108CBC0000F0E8FC7B681B681E4A934207D17B6876
:108CCC001B685A6C7B681B6842F400425A647B68D0
:108CDC001B68184A93420ED07B681B68B3F1804F17
:108CEC0009D07B681B68144A934204D07B681B68CC
:108CFC00124A934211D17B681B689B6803F00703EF
:108D0C00FB60FB68062B10D07B681B681A687B68BD
:108D1C001B6842F001021A6007E07B681B681A6846
:108D2C007B681B6842F001021A600023184610375A
:108D3C00BD4680BD002C01400004004000080040EE
:108D4C0080B582B000AF786039607B681B68002208
:108D5C003968184600F096FC7B681B68294A9342D8
:108D6C0017D17B681B681A6A41F211131340002B50
:108D7C000FD17B681B681A6A40F244431340002BE6
:108D8C0007D17B681B685A6C7B681B6822F4004215
:108D9C005A647B681B681A6A41F211131340002B4A
:108DAC000FD17B681B681A6A40F244431340002BB6
:108DBC0007D17B681B681A687B681B6822F001026C
:108DCC001A603B68002B04D17B68012283F83E209B
:108DDC0013E03B68042B04D17B68012283F83F200D
:108DEC000BE03B68082B04D17B68012283F8402000
:108DFC0003E07B68012283F84120002318460837E2
:108E0C00BD4680BD002C014080B586B000AFF86037
:108E1C00B9607A600023FB75FB6893F83C30012B3A
:108E2C0001D10223AEE0FB68012283F83C207B6871
:108E3C000C2B00F29F8001A252F823F07D8E0008CB
:108E4C00818F0008818F0008818F0008BD8E00087B
:108E5C00818F0008818F0008818F0008FF8E000829
:108E6C00818F0008818F0008818F00083F8F0008D8
:108E7C00FB681B68B968184600F0E6F9FB681B68CC
:108E8C009A69FB681B6842F008029A61FB681B68D0
:108E9C009A69FB681B6822F004029A61FB681B68E4
:108EAC009969BB681A69FB681B680A439A6164E09C
:108EBC00FB681B68B968184600F02CFAFB681B6845
:108ECC009A69FB681B6842F400629A61FB681B6834
:108EDC009A69FB681B6822F480629A61FB681B68C4
:108EEC009969BB681B691A02FB681B680A439A6183
:108EFC0043E0FB681B68B968184600F075FAFB681C
:108F0C001B68DA69FB681B6842F00802DA61FB68CF
:108F1C001B68DA69FB681B6822F00402DA61FB68E3
:108F2C001B68D969BB681A69FB681B680A43DA615C
:108F3C0023E0FB681B68B968184600F0BFFAFB68B1
:108F4C001B68DA69FB681B6842F40062DA61FB6833
:108F5C001B68DA69FB681B6822F48062DA61FB68C3
:108F6C001B68D969BB681B691A02FB681B680A433A
:108F7C00DA6102E00123FB7500BFFB68002283F875
:108F8C003C20FB7D18461837BD4680BD80B584B0AB
:108F9C0000AF786039600023FB737B6893F83C303A
:108FAC00012B01D10223B4E07B68012283F83C2021
:108FBC007B68022283F83D207B681B689B68BB6042
:108FCC00BB6823F07703BB60BB6823F47F43BB60B3
:108FDC007B681B68BA689A603B681B68B3F5005FD6
:108FEC003ED0B3F5005F00F28780B3F5805F00F0F0
:108FFC008680B3F5805F7FD8702B1AD0702B7BD80E
:10900C00602B50D0602B77D8502B3CD0502B73D882
:10901C00402B58D0402B6FD8302B64D0302B6BD8D2
:10902C00202B60D0202B67D8002B5CD0102B5AD073
:10903C0062E07B6818683B6899683B685A683B68D3
:10904C00DB6800F000FB7B681B689B68BB60BB683F
:10905C0043F07703BB607B681B68BA689A604FE08B
:10906C007B6818683B6899683B685A683B68DB68A2
:10907C0000F0E9FA7B681B689A687B681B6842F40D
:10908C0080429A603CE07B6818683B6859683B6892
:10909C00DB681A4600F060FA7B681B6850211846A2
:1090AC0000F0B7FA2CE07B6818683B6859683B689D
:1090BC00DB681A4600F07EFA7B681B686021184654
:1090CC0000F0A7FA1CE07B6818683B6859683B689D
:1090DC00DB681A4600F040FA7B681B684021184692
:1090EC0000F097FA0CE07B681A683B681B6819461D
:1090FC00104600F08EFA03E00123FB7300E000BF82
:10910C007B68012283F83D207B68002283F83C2099
:10911C00FB7B18461037BD4680BD80B485B000AFD0
:10912C00786039603B68002B04D17B6893F83E3043
:10913C00DBB213E03B68042B04D17B6893F83F301F
:10914C00DBB20BE03B68082B04D17B6893F8403012
:10915C00DBB203E07B6893F84130DBB2FB73FB7B43
:10916C0018461437BD4680BC7047000080B485B0EB
:10917C0000AF786039607B681B68FB607B682F4AA6
:10918C0093420BD07B68B3F1804F07D07B682C4A9D
:10919C00934203D07B682B4A934208D1FB6823F09F
:1091AC007003FB603B685B68FA681343FB607B6889
:1091BC00224A93420BD07B68B3F1804F07D07B6877
:1091CC001F4A934203D07B681E4A934208D1FB6826
:1091DC0023F44073FB603B68DB68FA681343FB6065
:1091EC00FB6823F080023B685B691343FB607B6880
:1091FC00FA681A603B689A687B68DA623B681A689E
:10920C007B689A627B680D4A934203D13B681A696A
:10921C007B681A637B6801225A617B681B6903F0C7
:10922C000103002B05D07B681B6923F001027B68CE
:10923C001A6100BF1437BD4680BC7047002C01403A
:10924C00000400400008004080B487B000AF786094
:10925C0039607B681B6A7B617B681B6A23F00102A7
:10926C007B681A627B685B683B617B689B69FB600F
:10927C00FB6823F07003FB60FB6823F00303FB60C7
:10928C003B681B68FA681343FB607B6923F002039D
:10929C007B613B689B687A6913437B617B681C4AE2
:1092AC0093420CD17B6923F008037B613B68DB683C
:1092BC007A6913437B617B6923F004037B617B68D0
:1092CC00134A934211D13B6923F480733B613B6990
:1092DC0023F400733B613B685B693A6913433B6160
:1092EC003B689B693A6913433B617B683A695A60F6
:1092FC007B68FA689A613B685A687B685A637B683A
:10930C007A691A6200BF1C37BD4680BC704700BF2B
:10931C00002C014080B487B000AF786039607B6866
:10932C001B6A7B617B681B6A23F010027B681A62E4
:10933C007B685B683B617B689B69FB60FB6823F423
:10934C00E043FB60FB6823F44073FB603B681B68E5
:10935C001B02FA681343FB607B6923F020037B61DB
:10936C003B689B681B017A6913437B617B681D4AD0
:10937C0093420DD17B6923F080037B613B68DB68F2
:10938C001B017A6913437B617B6923F040037B618A
:10939C007B68144A934213D13B6923F480633B618D
:1093AC003B6923F400633B613B685B699B003A6952
:1093BC0013433B613B689B699B003A6913433B61D8
:1093CC007B683A695A607B68FA689A613B685A68AC
:1093DC007B689A637B687A691A6200BF1C37BD464A
:1093EC0080BC7047002C014080B487B000AF78601F
:1093FC0039607B681B6A7B617B681B6A23F4807213
:10940C007B681A627B685B683B617B68DB69FB602D
:10941C00FB6823F07003FB60FB6823F00303FB6025
:10942C003B681B68FA681343FB607B6923F4007389
:10943C007B613B689B681B027A6913437B617B6889
:10944C001D4A93420DD17B6923F400637B613B6819
:10945C00DB681B027A6913437B617B6923F48063AD
:10946C007B617B68144A934213D13B6923F480538C
:10947C003B613B6923F400533B613B685B691B0117
:10948C003A6913433B613B689B691B013A6913437F
:10949C003B617B683A695A607B68FA68DA613B68C1
:1094AC005A687B68DA637B687A691A6200BF1C377A
:1094BC00BD4680BC704700BF002C014080B487B013
:1094CC0000AF786039607B681B6A3B617B681B6A04
:1094DC0023F480527B681A627B685B687B617B68D3
:1094EC00DB69FB60FB6823F4E043FB60FB6823F45F
:1094FC004073FB603B681B681B02FA681343FB60FC
:10950C003B6923F400533B613B689B681B033A693E
:10951C0013433B617B680F4A934209D17B6923F467
:10952C0080437B613B685B699B017A6913437B6178
:10953C007B687A695A607B68FA68DA613B685A68BA
:10954C007B681A647B683A691A6200BF1C37BD4697
:10955C0080BC7047002C014080B487B000AFF8602D
:10956C00B9607A60FB681B6A7B61FB681B6A23F03D
:10957C000102FB681A62FB689B693B613B6923F043
:10958C00F0033B617B681B013A6913433B617B69C8
:10959C0023F00A037B617A69BB6813437B61FB6828
:1095AC003A699A61FB687A691A6200BF1C37BD463A
:1095BC0080BC704780B487B000AFF860B9607A6047
:1095CC00FB681B6A7B61FB681B6A23F01002FB685B
:1095DC001A62FB689B693B613B6923F470433B61F6
:1095EC007B681B033A6913433B617B6923F0A0033F
:1095FC007B61BB681B017A6913437B61FB683A6929
:10960C009A61FB687A691A6200BF1C37BD4680BC40
:10961C00704780B485B000AF786039607B689B6818
:10962C00FB60FB6823F07003FB603A68FB68134334
:10963C0043F00703FB607B68FA689A6000BF14373D
:10964C00BD4680BC704780B487B000AFF860B9608D
:10965C007A603B60FB689B687B617B6923F47F438A
:10966C007B613B681A027B681A43BB6813437A69B7
:10967C0013437B61FB687A699A6000BF1C37BD4657
:10968C0080BC704780B487B000AFF860B9607A6076
:10969C00BB6803F01F03012202FA03F37B61FB6832
:1096AC001A6A7B69DB431A40FB681A62FB681A6A08
:1096BC00BB6803F01F03796801FA03F31A43FB68D4
:1096CC001A6200BF1C37BD4680BC704780B485B0A1
:1096DC0000AF786039607B6893F83C30012B01D186
:1096EC00022346E07B68012283F83C207B6802223F
:1096FC0083F83D207B681B685B68FB607B681B689C
:10970C009B68BB60FB6823F07003FB603B681B68C5
:10971C00FA681343FB607B681B68FA685A607B68C5
:10972C001B68164A93420ED07B681B68B3F1804FBE
:10973C0009D07B681B68124A934204D07B681B6873
:10974C00104A93420CD1BB6823F08003BB603B688A
:10975C005B68BA681343BB607B681B68BA689A6025
:10976C007B68012283F83D207B68002283F83C2033
:10977C00002318461437BD4680BC7047002C0140AE
:10978C00000400400008004080B582B000AF786053
:10979C007B68002B01D1012342E07B6893F84130B8
:1097AC00DBB2002B06D17B68002283F8402078685E
:1097BC00FBF780FB7B68242283F841207B681B68C5
:1097CC00DA687B681B6822F40052DA60786800F073
:1097DC0071F97B681B681A697B681B6822F49042DC
:1097EC001A617B681B685A697B681B6822F02A0225
:1097FC005A617B681B68DA687B681B6842F400520C
:10980C00DA607B6800225A647B68202283F841204E
:10981C007B68202283F842207B6800225A63002355
:10982C0018460837BD4680BD80B58AB002AFF860D7
:10983C00B9603B601346FB8000237B61FB6893F8A7
:10984C004130DBB2202B75D1BB68002B02D0FB88DA
:10985C00002B01D101236EE0FB6800225A64FB68E7
:10986C00212283F84120FBF76DFC7861FB68FA88B4
:10987C009A84FB68FA88DA84FB689B68B3F5805F8E
:10988C0008D1FB681B69002B04D10023FB61BB686A
:10989C00BB6103E0BB68FB610023BB612EE03B684E
:1098AC0000937B6900228021F86800F048F8034699
:1098BC00002B05D0FB68202283F8412003233AE0DB
:1098CC00FB69002B0BD1BB691B881A46FB681B6814
:1098DC00C2F308025A60BB690233BB6107E0FB6943
:1098EC001A78FB681B685A60FB690133FB61FB68E3
:1098FC00DB8C9BB2013B9AB2FB68DA84FB68DB8C95
:10990C009BB2002BCBD13B6800937B69002240219A
:10991C00F86800F014F80346002B05D0FB682022F1
:10992C0083F84120032306E0FB68202283F84120C2
:10993C00002300E0022318462037BD4680BD80B5C9
:10994C0086B000AFF860B9603B601346FB713BE03A
:10995C003B6AB3F1FF3F37D0FBF7F4FB02463B68A1
:10996C00D31A3A6A9A4202D33B6A002B01D10323E1
:10997C003AE0FB681B68DB6803F00403002B23D080
:10998C00BB68802B20D0BB68402B1DD0FB681B68AC
:10999C001B6803F00803082B16D100237B61FB68BE
:1099AC001B681B687B61FB681B685B687B617B6960
:1099BC00F86800F01DF8FB6808225A64FB68002266
:1099CC0083F8402001230FE0FB681B681A68BB6812
:1099DC001340BA689A420CBF01230023DBB21A462B
:1099EC00FB799A42B4D0002318461837BD4680BD87
:1099FC0080B495B000AF78607B681B680C337B63D8
:109A0C007B6B53E8003F3B633B6B23F49073FB642D
:109A1C007B681B680C33FA6C3A64FB63F96B3A6C29
:109A2C0041E80023BB63BB6B002BE5D17B681B6853
:109A3C0014333B623B6A53E8003FFB61FB6923F044
:109A4C000103BB647B681B681433BA6CFA62BB629B
:109A5C00B96AFA6A41E800237B627B6A002BE5D184
:109A6C007B681B6B012B19D17B681B680C33FB606B
:109A7C00FB6853E8003FBB60BB6823F010037B64BA
:109A8C007B681B680C337A6CBA617B617969BA6943
:109A9C0041E800233B613B69002BE5D17B68202228
:109AAC0083F842207B6800221A6300BF5437BD46FE
:109ABC0080BC704780B584B000AF78607B681B6851
:109ACC001B6923F440517B68DA687B681B680A4386
:109ADC001A617B689A687B681B691A437B685B69AF
:109AEC001343BB607B681B68DB6823F4B05323F023
:109AFC000C037A681268B9680B43D3607B681B68E7
:109B0C005B6923F440717B689A697B681B680A4324
:109B1C005A617B681B682C4A934203D1FEF7DEFE28
:109B2C00F86002E0FEF7C6FEF860FA6813469B0088
:109B3C0013449A001A447B685B689B00B2FBF3F3F6
:109B4C00224AA2FB03235B091901FA6813469B0006
:109B5C0013449A001A447B685B689B00B2FBF3F2D7
:109B6C001A4BA3FB02035B09642000FB03F3D31A1B
:109B7C001B013233154AA2FB03235B0903F0F003EC
:109B8C001944FA6813469B0013449A001A447B68E4
:109B9C005B689B00B2FBF3F20C4BA3FB02035B096B
:109BAC00642000FB03F3D31A1B013233074AA2FBD8
:109BBC0003235B0903F00F027B681B680A449A605D
:109BCC0000BF1037BD4680BD003801401F85EB51EA
:109BDC0080B485B000AFF860384680E80E000023F2
:109BEC0018461437BD4680BC704780B485B000AFB2
:109BFC0078607B680022A3F844204FF43F43FB605D
:109C0C00FB689AB27B68A3F84020002318461437EF
:109C1C00BD4680BC704780B485B000AF78604FF40F
:109C2C003F43FB607B68B3F840309AB2FB689BB251
:109C3C00DB439BB213409AB27B68A3F8402000230D
:109C4C0018461437BD4680BC704780B483B000AF53
:109C5C0078600B46FB70002318460C37BD4680BC61
:109C6C00704780B485B000AFF860384680E80E00CD
:109C7C00FB680122A3F84020FB680022A3F84020D7
:109C8C00FB680022A3F84420FB680022A3F85020B4
:109C9C00002318461437BD4680BC704780B49DB075
:109CAC0000AF78603960002387F86F307A683B68C2
:109CBC001B789B0013441B889BB223F4EC4323F0CA
:109CCC007003A7F86C303B68DB78032B1FD801A21C
:109CDC0052F823F0F19C00080D9D0008239D00080C
:109CEC00FF9C0008B7F86C3043F40073A7F86C3095
:109CFC0012E0B7F86C3043F4C063A7F86C300BE09B
:109D0C00B7F86C3043F48063A7F86C3004E001239F
:109D1C0087F86F3000E000BF7A683B681B789B00C7
:109D2C001A44B7F86C3043F07F4343F47F0343F499
:109D3C00004343F080039BB213807A683B681B7826
:109D4C009B0013441B889BB223F4E04323F0700365
:109D5C009BB23A6812781343A7F866307A683B686E
:109D6C001B789B001A44B7F8663043F07F4343F4EA
:109D7C007F0343F4004343F080039BB213803B68A2
:109D8C001B7B002B40F078813B685B78002B00F04C
:109D9C0084807B68BB617B68B3F850309BB21A46F9
:109DAC00BB691344BB613B681B781A01BB69134444
:109DBC0003F580637B613B68DB885B089BB25B00CF
:109DCC009AB27B691A807A683B681B789B001344B3
:109DDC001B887B827B8A03F04003002B1BD07A68A4
:109DEC003B681B789B0013441B889BB223F4E04315
:109DFC0023F070033B827A683B681B789B001A4403
:109E0C003B8A43F07F4343F47F0343F4004343F026
:109E1C00C0039BB213803B68DB78012B20D07A689F
:109E2C003B681B789B0013441B889BB223F4E043D4
:109E3C0023F04003BB81BB8983F02003BB817A688C
:109E4C003B681B789B001A44BB8943F07F4343F467
:109E5C007F0343F4004343F080039BB21380D5E2AD
:109E6C007A683B681B789B0013441B889BB223F4D5
:109E7C00E04323F04003FB817A683B681B789B002E
:109E8C001A44FB8943F07F4343F47F0343F40043BC
:109E9C0043F080039BB21380B8E27B683B637B6822
:109EAC00B3F850309BB21A463B6B13443B633B6890
:109EBC001B781A013B6B134403F58163FB623B680F
:109ECC00DB885B089BB25B009AB2FB6A1A807B68EA
:109EDC00BB627B68B3F850309BB21A46BB6A134422
:109EEC00BB623B681B781A01BB6A134403F20C4338
:109EFC007B627B6A1B889BB2C3F309039AB27B6AB1
:109F0C001A803B681B693E2B1DD93B681B695B099A
:109F1C00BB663B681B6903F01F03002B02D1BB6EB1
:109F2C00013BBB667B6A1B889AB2BB6E9BB29B02E1
:109F3C009BB213439BB26FEA43436FEA53439AB20B
:109F4C007B6A1A8026E03B681B69002B0AD17B6A6E
:109F5C001B889BB26FEA43436FEA53439AB27B6A06
:109F6C001A8017E03B681B695B08BB663B681B6982
:109F7C0003F00103002B02D0BB6E0133BB667B6A7E
:109F8C001B889AB2BB6E9BB29B029BB213439AB2D4
:109F9C007B6A1A807A683B681B789B0013441B8889
:109FAC007B847B8C03F48043002B1BD07A683B684A
:109FBC001B789B0013441B889BB223F4E04323F0D3
:109FCC0070033B847A683B681B789B001A443B8C7B
:109FDC0043F07F4343F47F0343F4404343F0800357
:109FEC009BB213803B681B78002B24D17A683B68AA
:109FFC001B789B0013441B889BB223F4804323F0F3
:10A00C007003BB83BB8B83F48053BB83BB8B83F408
:10A01C000053BB837A683B681B789B001A44BB8B4C
:10A02C0043F07F4343F47F0343F4004343F0800346
:10A03C009BB21380EAE17A683B681B789B0013445F
:10A04C001B889BB223F4804323F07003FB83FB8BB0
:10A05C0083F40053FB837A683B681B789B001A449B
:10A06C00FB8B43F07F4343F47F0343F4004343F003
:10A07C0080039BB21380C9E13B68DB78022B1ED1B5
:10A08C007A683B681B789B0013441B889BB223F4B3
:10A09C00E04323F07003A7F862307A683B681B78C2
:10A0AC009B001A44B7F8623043F07F4343F47F03BC
:10A0BC0043F4014343F080039BB213801DE07A68A4
:10A0CC003B681B789B0013441B889BB223F4E24330
:10A0DC0023F07003A7F864307A683B681B789B0008
:10A0EC001A44B7F8643043F07F4343F47F0343F4DE
:10A0FC00004343F080039BB213807B68FB657B6855
:10A10C00B3F850309BB21A46FB6D1344FB653B68A9
:10A11C001B781A01FB6D134403F58063BB653B6828
:10A12C001B895B089BB25B009AB2BB6D1A807B6883
:10A13C007B657B68B3F850309BB21A467B6D134439
:10A14C007B653B681B781A017B6D134403F58163B7
:10A15C003B653B685B895B089BB25B009AB23B6DCD
:10A16C001A803B685B78002B40F093807A683B68E0
:10A17C001B789B0013441B88A7F84030B7F840307D
:10A18C0003F48043002B1BD07A683B681B789B0040
:10A19C0013441B889BB223F4E04323F07003FB872A
:10A1AC007A683B681B789B001A44FB8F43F07F4313
:10A1BC0043F47F0343F4404343F080039BB213808A
:10A1CC007A683B681B789B0013441B88BB87BB8F4A
:10A1DC0003F04003002B1BD07A683B681B789B0074
:10A1EC0013441B889BB223F4E04323F070037B875A
:10A1FC007A683B681B789B001A447B8F43F07F4343
:10A20C0043F47F0343F4004343F0C0039BB2138039
:10A21C007A683B681B789B0013441B889BB223F421
:10A22C00804323F070033B873B8F83F480533B8741
:10A23C003B8F83F400533B877A683B681B789B0009
:10A24C001A443B8F43F07F4343F47F0343F40043B2
:10A25C0043F080039BB213807A683B681B789B00A9
:10A26C0013441B889BB223F4E04323F04003FB868A
:10A27C007A683B681B789B001A44FB8E43F07F4343
:10A28C0043F47F0343F4004343F080039BB21380F9
:10A29C00BCE07A683B681B789B0013441B88A7F8CA
:10A2AC004E30B7F84E3003F48043002B1DD07A6843
:10A2BC003B681B789B0013441B889BB223F4E04340
:10A2CC0023F07003A7F84C307A683B681B789B002E
:10A2DC001A44B7F84C3043F07F4343F47F0343F404
:10A2EC00404343F080039BB213807A683B681B7831
:10A2FC009B0013441B88A7F84A30B7F84A3003F088
:10A30C004003002B1DD07A683B681B789B001344DC
:10A31C001B889BB223F4E04323F07003A7F848306A
:10A32C007A683B681B789B001A44B7F8483043F0B6
:10A33C007F4343F47F0343F4004343F0C0039BB2D9
:10A34C0013803B68DB78012B24D07A683B681B7840
:10A35C009B0013441B889BB223F4E04323F040037F
:10A36C00A7F84430B7F8443083F02003A7F8443002
:10A37C007A683B681B789B001A44B7F8443043F06A
:10A38C007F4343F47F0343F4004343F080039BB2C9
:10A39C0013801DE07A683B681B789B0013441B8874
:10A3AC009BB223F4E04323F04003A7F846307A68CD
:10A3BC003B681B789B001A44B7F8463043F07F4348
:10A3CC0043F47F0343F4004343F080039BB21380B8
:10A3DC007A683B681B789B0013441B889BB223F460
:10A3EC00804323F07003A7F842307A683B681B78EF
:10A3FC009B001A44B7F8423043F07F4343F47F0389
:10A40C0043F4004343F080039BB2138097F86F3002
:10A41C0018467437BD4680BC704700BF80B48DB001
:10A42C0000AF786039603B681B7B002B40F08E805E
:10A43C003B685B78002B44D07A683B681B789B00A8
:10A44C0013441B88BB81BB8903F04003002B1BD03A
:10A45C007A683B681B789B0013441B889BB223F4DF
:10A46C00E04323F070037B817A683B681B789B0088
:10A47C001A447B8943F07F4343F47F0343F4004346
:10A48C0043F0C0039BB213807A683B681B789B0037
:10A49C0013441B889BB223F4E04323F040033B811D
:10A4AC007A683B681B789B001A443B8943F07F43D6
:10A4BC0043F47F0343F4004343F080039BB21380C7
:10A4CC0092E17A683B681B789B0013441B887B8263
:10A4DC007B8A03F48043002B1BD07A683B681B7883
:10A4EC009B0013441B889BB223F4E04323F07003BE
:10A4FC003B827A683B681B789B001A443B8A43F08A
:10A50C007F4343F47F0343F4404343F080039BB207
:10A51C0013807A683B681B789B0013441B889BB2A2
:10A52C0023F4804323F07003FB817A683B681B782B
:10A53C009B001A44FB8943F07F4343F47F0343F4AD
:10A54C00004343F080039BB213804DE13B685B7882
:10A55C00002B40F0A5807A683B681B789B00134465
:10A56C001B883B843B8C03F48043002B1BD07A6804
:10A57C003B681B789B0013441B889BB223F4E0437D
:10A58C0023F07003FB837A683B681B789B001A44AA
:10A59C00FB8B43F07F4343F47F0343F4404343F08E
:10A5AC0080039BB213807A683B681B789B00134432
:10A5BC001B88BB83BB8B03F04003002B1BD07A683A
:10A5CC003B681B789B0013441B889BB223F4E0432D
:10A5DC0023F070037B837A683B681B789B001A44DA
:10A5EC007B8B43F07F4343F47F0343F4004343F0FE
:10A5FC00C0039BB213807A683B681B789B001344A2
:10A60C001B889BB223F4E04323F070033B837A68EE
:10A61C003B681B789B001A443B8B43F07F4343F40D
:10A62C007F0343F4004343F0C0039BB213807A686A
:10A63C003B681B789B0013441B889BB223F480431C
:10A64C0023F07003FB827A683B681B789B001A44EA
:10A65C00FB8A43F07F4343F47F0343F4004343F00E
:10A66C0080039BB213807A683B681B789B00134471
:10A67C001B889BB223F4E04323F04003BB827A682F
:10A68C003B681B789B001A44BB8A43F07F4343F41E
:10A69C007F0343F4004343F080039BB21380A3E099
:10A6AC007A683B681B789B0013441B88FB85FB8DE9
:10A6BC0003F48043002B1BD07A683B681B789B000B
:10A6CC0013441B889BB223F4E04323F07003BB8537
:10A6DC007A683B681B789B001A44BB8D43F07F4320
:10A6EC0043F47F0343F4404343F080039BB2138055
:10A6FC007A683B681B789B0013441B887B857B8D99
:10A70C0003F04003002B1BD07A683B681B789B003E
:10A71C0013441B889BB223F4E04323F070033B8566
:10A72C007A683B681B789B001A443B8D43F07F434F
:10A73C0043F47F0343F4004343F0C0039BB2138004
:10A74C007A683B681B789B0013441B889BB223F4EC
:10A75C00E04323F07003FB847A683B681B789B0012
:10A76C001A44FB8C43F07F4343F47F0343F4404390
:10A77C0043F080039BB213807A683B681B789B0084
:10A78C0013441B889BB223F4E04323F04003BB84A7
:10A79C007A683B681B789B001A44BB8C43F07F4360
:10A7AC0043F47F0343F4004343F080039BB21380D4
:10A7BC007A683B681B789B0013441B889BB223F47C
:10A7CC00804323F070037B847A683B681B789B0082
:10A7DC001A447B8C43F07F4343F47F0343F40043E0
:10A7EC0043F080039BB21380002318463437BD46D8
:10A7FC0080BC704780B5C2B000AF07F58473A3F579
:10A80C008273186007F58473A3F58473196007F5D8
:10A81C008473A3F584731B685B78012B40F0B786B7
:10A82C0007F58473A3F584731B689A6907F5847321
:10A83C00A3F584731B681B699A4208D907F58473C6
:10A84C00A3F584731B681B69C7F8043107E007F58F
:10A85C008473A3F584731B689B69C7F8043107F5EF
:10A86C008473A3F584731B681B7B002B3AD107F50B
:10A87C008473A3F584731B68596907F58473A3F576
:10A88C0084731B68DA88D7F804319BB207F584709F
:10A89C00A0F58270006801F09CFC07F58473A3F5A9
:10A8AC0082731B683B6107F58473A3F582731B6885
:10A8BC00B3F850309BB21A463B6913443B6107F521
:10A8CC008473A3F584731B681B781A013B691344CA
:10A8DC0003F20443FB60D7F804319AB2FB681A8088
:10A8EC0000F01FBE07F58473A3F584731B68DB7837
:10A8FC00022B40F0628407F58473A3F584731B6804
:10A90C001A6A07F58473A3F584731B681B699A4252
:10A91C0040F2DF8307F58473A3F582731A6807F599
:10A92C008473A3F584731B681B789B0013441B88EA
:10A93C009BB223F4E04323F07003A7F8563007F5DD
:10A94C008473A3F582731A6807F58473A3F5847373
:10A95C001B681B789B001A44B7F8563043F07F43B2
:10A96C0043F47F0343F4014343F080039BB2138011
:10A97C0007F58473A3F584731B681A6AD7F804313E
:10A98C00D21A07F58473A3F584731B681A6207F552
:10A99C008473A3F582731A6807F58473A3F5847323
:10A9AC001B681B789B0013441B889BB203F040036D
:10A9BC00002B00F0C78107F58473A3F582731B6825
:10A9CC003B6307F58473A3F584731B685B78002BDA
:10A9DC0077D107F58473A3F582731B68BB6207F507
:10A9EC008473A3F582731B68B3F850309BB21A467C
:10A9FC00BB6A1344BB6207F58473A3F584731B68AD
:10AA0C001B781A01BB6A134403F20C437B627B6A0A
:10AA1C001B889BB2C3F309039AB27B6A1A80D7F8DE
:10AA2C0004313E2B21D9D7F804315B09C7F800312A
:10AA3C00D7F8043103F01F03002B04D1D7F80031F1
:10AA4C00013BC7F800317B6A1B889AB2D7F80031FA
:10AA5C009BB29B029BB213439BB26FEA43436FEAD8
:10AA6C0053439AB27B6A1A8050E0D7F80431002B1A
:10AA7C000AD17B6A1B889BB26FEA43436FEA53434C
:10AA8C009AB27B6A1A8041E0D7F804315B08C7F8A8
:10AA9C000031D7F8043103F00103002B04D0D7F8B0
:10AAAC0000310133C7F800317B6A1B889AB2D7F8A2
:10AABC0000319BB29B029BB213439AB27B6A1A8001
:10AACC0024E007F58473A3F584731B685B78012B72
:10AADC001CD107F58473A3F582731B68B3F850304F
:10AAEC009BB21A463B6B13443B6307F58473A3F587
:10AAFC0084731B681B781A013B6B134403F20C43E1
:10AB0C00FB62D7F804319AB2FB6A1A8007F584739A
:10AB1C00A3F584731B685B89A7F8763007F58473FB
:10AB2C00A3F584731B685969D7F804319BB2B7F845
:10AB3C00762007F58470A0F58270006801F049FB5F
:10AB4C0007F58473A3F584731B685A69D7F804312D
:10AB5C001A4407F58473A3F584731B685A6107F5CF
:10AB6C008473A3F584731B681A6A07F58473A3F5C1
:10AB7C0084731B681B699A420FD907F58473A3F57C
:10AB8C0084731B681A6AD7F80431D21A07F58473D8
:10AB9C00A3F584731B681A620EE007F58473A3F5A2
:10ABAC0084731B681B6AC7F8043107F58473A3F51B
:10ABBC0084731B6800221A6207F58473A3F58473EF
:10ABCC001B685B78002B77D107F58473A3F5827330
:10ABDC001B68BB6107F58473A3F582731B68B3F81C
:10ABEC0050309BB21A46BB691344BB6107F58473A2
:10ABFC00A3F584731B681B781A01BB69134403F219
:10AC0C0004437B617B691B889BB2C3F309039AB233
:10AC1C007B691A80D7F804313E2B21D9D7F804313F
:10AC2C005B09C7F8FC30D7F8043103F01F03002B85
:10AC3C0004D1D7F8FC30013BC7F8FC307B691B888A
:10AC4C009AB2D7F8FC309BB29B029BB213439BB2D7
:10AC5C006FEA43436FEA53439AB27B691A8056E01A
:10AC6C00D7F80431002B0AD17B691B889BB26FEAA1
:10AC7C0043436FEA53439AB27B691A8047E0D7F893
:10AC8C0004315B08C7F8FC30D7F8043103F001033A
:10AC9C00002B04D0D7F8FC300133C7F8FC307B69AB
:10ACAC001B889AB2D7F8FC309BB29B029BB2134321
:10ACBC009AB27B691A802AE007F58473A3F5847332
:10ACCC001B685B78012B22D107F58473A3F5827383
:10ACDC001B683B6207F58473A3F582731B68B3F89A
:10ACEC0050309BB21A463B6A13443B6207F584739F
:10ACFC00A3F584731B681B781A013B6A134403F297
:10AD0C000443FB61D7F804319AB2FB691A8007F54A
:10AD1C008473A3F584731B681B89A7F8763007F539
:10AD2C008473A3F584731B685969D7F804319BB2FB
:10AD3C00B7F8762007F58470A0F58270006801F0F2
:10AD4C0048FAEEE307F58473A3F584731B685B780C
:10AD5C00002B77D107F58473A3F582731B68BB6452
:10AD6C0007F58473A3F582731B68B3F850309BB25C
:10AD7C001A46BB6C1344BB6407F58473A3F5847348
:10AD8C001B681B781A01BB6C134403F204437B64ED
:10AD9C007B6C1B889BB2C3F309039AB27B6C1A8041
:10ADAC00D7F804313E2B21D9D7F804315B09C7F809
:10ADBC00F830D7F8043103F01F03002B04D1D7F877
:10ADCC00F830013BC7F8F8307B6C1B889AB2D7F887
:10ADDC00F8309BB29B029BB213439BB26FEA434386
:10ADEC006FEA53439AB27B6C1A8056E0D7F8043161
:10ADFC00002B0AD17B6C1B889BB26FEA43436FEA32
:10AE0C0053439AB27B6C1A8047E0D7F804315B0845
:10AE1C00C7F8F830D7F8043103F00103002B04D045
:10AE2C00D7F8F8300133C7F8F8307B6C1B889AB22E
:10AE3C00D7F8F8309BB29B029BB213439AB27B6C4F
:10AE4C001A802AE007F58473A3F584731B685B787A
:10AE5C00012B22D107F58473A3F582731B683B6524
:10AE6C0007F58473A3F582731B68B3F850309BB25B
:10AE7C001A463B6D13443B6507F58473A3F5847345
:10AE8C001B681B781A013B6D134403F20443FB64EB
:10AE9C00D7F804319AB2FB6C1A8007F58473A3F5CA
:10AEAC0084731B681B89A7F8763007F58473A3F5A8
:10AEBC0084731B685969D7F804319BB2B7F87620B4
:10AECC0007F58470A0F58270006801F082F907F52F
:10AEDC008473A3F584731B685A69D7F804311A4438
:10AEEC0007F58473A3F584731B685A6107F58473A3
:10AEFC00A3F584731B681A6A07F58473A3F584732E
:10AF0C001B681B699A420FD907F58473A3F58473E8
:10AF1C001B681A6AD7F80431D21A07F58473A3F5A3
:10AF2C0084731B681A620EE007F58473A3F58473AF
:10AF3C001B681B6AC7F8043107F58473A3F5847387
:10AF4C001B6800221A6207F58473A3F582731B68D1
:10AF5C003B6407F58473A3F584731B685B78002B43
:10AF6C0077D107F58473A3F582731B68BB6307F570
:10AF7C008473A3F582731B68B3F850309BB21A46E6
:10AF8C00BB6B1344BB6307F58473A3F584731B6815
:10AF9C001B781A01BB6B134403F20C437B637B6B72
:10AFAC001B889BB2C3F309039AB27B6B1A80D7F848
:10AFBC0004313E2B21D9D7F804315B09C7F8F430A2
:10AFCC00D7F8043103F01F03002B04D1D7F8F43069
:10AFDC00013BC7F8F4307B6B1B889AB2D7F8F4307E
:10AFEC009BB29B029BB213439BB26FEA43436FEA43
:10AFFC0053439AB27B6B1A8050E0D7F80431002B84
:10B00C000AD17B6B1B889BB26FEA43436FEA5343B5
:10B01C009AB27B6B1A8041E0D7F804315B08C7F811
:10B02C00F430D7F8043103F00103002B04D0D7F827
:10B03C00F4300133C7F8F4307B6B1B889AB2D7F825
:10B04C00F4309BB29B029BB213439AB27B6B1A8077
:10B05C0024E007F58473A3F584731B685B78012BDC
:10B06C001CD107F58473A3F582731B68B3F85030B9
:10B07C009BB21A463B6C13443B6407F58473A3F5EF
:10B08C0084731B681B781A013B6C134403F20C434A
:10B09C00FB63D7F804319AB2FB6B1A8007F5847303
:10B0AC00A3F584731B685B89A7F8763007F5847366
:10B0BC00A3F584731B685969D7F804319BB2B7F8B0
:10B0CC00762007F58470A0F58270006801F081F895
:10B0DC0027E207F58473A3F584731B681B6AC7F812
:10B0EC00043107F58473A3F582731A6807F584732A
:10B0FC00A3F584731B681B789B0013441B889BB2BD
:10B10C0023F4E24323F07003A7F8623007F584734D
:10B11C00A3F582731A6807F58473A3F584731B680F
:10B12C001B789B001A44B7F8623043F07F4343F41A
:10B13C007F0343F4004343F080039BB2138007F575
:10B14C008473A3F582731B68FB6507F58473A3F501
:10B15C0082731B68B3F850309BB21A46FB6D1344D4
:10B16C00FB6507F58473A3F584731B681B781A01C0
:10B17C00FB6D134403F20443BB65D7F804319AB258
:10B18C00BB6D1A8007F58473A3F584731B681B8948
:10B19C00A7F8763007F58473A3F584731B68596997
:10B1AC00D7F804319BB2B7F8762007F58470A0F578
:10B1BC008270006801F00DF8B3E107F58473A3F514
:10B1CC0084731B681A6AD7F80431D21A07F5847392
:10B1DC00A3F584731B681A6207F58473A3F5827355
:10B1EC001A6807F58473A3F584731B681B789B009E
:10B1FC0013441B889BB203F04003002B00F0C68065
:10B20C0007F58473A3F582731B683B6707F584739A
:10B21C00A3F584731B685B78002B77D107F58473D7
:10B22C00A3F582731B68BB6607F58473A3F5827361
:10B23C001B68B3F850309BB21A46BB6E1344BB6606
:10B24C0007F58473A3F584731B681B781A01BB6E16
:10B25C00134403F20C437B667B6E1B889BB2C3F3D7
:10B26C0009039AB27B6E1A80D7F804313E2B21D990
:10B27C00D7F804315B09C7F8F030D7F8043103F084
:10B28C001F03002B04D1D7F8F030013BC7F8F03086
:10B29C007B6E1B889AB2D7F8F0309BB29B029BB2A4
:10B2AC0013439BB26FEA43436FEA53439AB27B6EEC
:10B2BC001A8050E0D7F80431002B0AD17B6E1B8822
:10B2CC009BB26FEA43436FEA53439AB27B6E1A8088
:10B2DC0041E0D7F804315B08C7F8F030D7F80431F7
:10B2EC0003F00103002B04D0D7F8F0300133C7F87A
:10B2FC00F0307B6E1B889AB2D7F8F0309BB29B0271
:10B30C009BB213439AB27B6E1A8024E007F58473C8
:10B31C00A3F584731B685B78012B1CD107F5847330
:10B32C00A3F582731B68B3F850309BB21A463B6F7F
:10B33C0013443B6707F58473A3F584731B681B7870
:10B34C001A013B6F134403F20C43FB66D7F804312C
:10B35C009AB2FB6E1A8007F58473A3F584731B688D
:10B36C005B89A7F8763007F58473A3F584731B68A3
:10B37C005969D7F804319BB2B7F8762007F5847079
:10B38C00A0F58270006800F024FFCAE007F5847312
:10B39C00A3F584731B685B78002B77D107F5847356
:10B3AC00A3F582731B68FB6707F58473A3F582739F
:10B3BC001B68B3F850309BB21A46FB6F1344FB6703
:10B3CC0007F58473A3F584731B681B781A01FB6F54
:10B3DC00134403F20443BB67BB6F1B889BB2C3F3DC
:10B3EC0009039AB2BB6F1A80D7F804313E2B21D9CE
:10B3FC00D7F804315B09C7F8EC30D7F8043103F007
:10B40C001F03002B04D1D7F8EC30013BC7F8EC300C
:10B41C00BB6F1B889AB2D7F8EC309BB29B029BB2E5
:10B42C0013439BB26FEA43436FEA53439AB2BB6F29
:10B43C001A805CE0D7F80431002B0AD1BB6F1B8853
:10B44C009BB26FEA43436FEA53439AB2BB6F1A80C5
:10B45C004DE0D7F804315B08C7F8EC30D7F804316D
:10B46C0003F00103002B04D0D7F8EC300133C7F8FC
:10B47C00EC30BB6F1B889AB2D7F8EC309BB29B02B6
:10B48C009BB213439AB2BB6F1A8030E007F58473FA
:10B49C00A3F584731B685B78012B28D107F58473A3
:10B4AC00A3F582731B68C7F8843007F58473A3F582
:10B4BC0082731B68B3F850309BB21A46D7F88430AD
:10B4CC001344C7F8843007F58473A3F584731B68A1
:10B4DC001B781A01D7F88430134403F20443C7F8DD
:10B4EC008030D7F804319AB2D7F880301A8007F53B
:10B4FC008473A3F584731B681B89A7F8763007F552
:10B50C008473A3F584731B685969D7F804319BB213
:10B51C00B7F8762007F58470A0F58270006800F00B
:10B52C0058FE07F58473A3F582731A6807F58473C4
:10B53C00A3F584731B681B789B0013441B889BB278
:10B54C0023F4E04323F040037B817B8983F01003D9
:10B55C007B817B8983F020037B8107F58473A3F5C2
:10B56C0082731A6807F58473A3F584731B681B78C0
:10B57C009B001A447B8943F07F4343F47F0343F4DD
:10B58C00004343F080039BB2138000F0DEBC07F550
:10B59C008473A3F584731B681B7B002B40F0BB806A
:10B5AC0007F58473A3F584731B689A6907F5847394
:10B5BC00A3F584731B681B699A4217D907F584732A
:10B5CC00A3F584731B681B69C7F8043107F58473F2
:10B5DC00A3F584731B689A69D7F80431D21A07F55E
:10B5EC008473A3F584731B689A610EE007F584736A
:10B5FC00A3F584731B689B69C7F8043107F5847342
:10B60C00A3F584731B6800229A6107F58473A3F574
:10B61C0082731B68C7F8903007F58473A3F58273A7
:10B62C001B68B3F850309BB21A46D7F890301344CD
:10B63C00C7F8903007F58473A3F584731B681B78E7
:10B64C001A01D7F89030134403F20C43C7F88C302E
:10B65C00D7F88C301B889BB2C3F309039AB2D7F886
:10B66C008C301A80D7F804313E2B24D9D7F804310A
:10B67C005B09C7F8E830D7F8043103F01F03002B3F
:10B68C0004D1D7F8E830013BC7F8E830D7F88C3054
:10B69C001B889AB2D7F8E8309BB29B029BB213433B
:10B6AC009BB26FEA43436FEA53439AB2D7F88C309C
:10B6BC001A8000F010BCD7F80431002B0CD1D7F84D
:10B6CC008C301B889BB26FEA43436FEA53439AB2A8
:10B6DC00D7F88C301A80FEE3D7F804315B08C7F832
:10B6EC00E830D7F8043103F00103002B04D0D7F86D
:10B6FC00E8300133C7F8E830D7F88C301B889AB2A1
:10B70C00D7F8E8309BB29B029BB213439AB2D7F89E
:10B71C008C301A80DFE307F58473A3F584731B6800
:10B72C00DB78022B40F0188207F58473A3F5847341
:10B73C001B685B78002B40F09D8007F58473A3F5A4
:10B74C0082731B68C7F8AC3007F58473A3F582735A
:10B75C001B68B3F850309BB21A46D7F8AC30134480
:10B76C00C7F8AC3007F58473A3F584731B681B789A
:10B77C001A01D7F8AC30134403F20443C7F8A830CD
:10B78C00D7F8A8301B889BB2C3F309039AB2D7F839
:10B79C00A8301A8007F58473A3F584731B681B69A2
:10B7AC003E2B2BD907F58473A3F584731B681B6997
:10B7BC005B09C7F8E43007F58473A3F584731B6841
:10B7CC001B6903F01F03002B04D1D7F8E430013BB5
:10B7DC00C7F8E430D7F8A8301B889AB2D7F8E43011
:10B7EC009BB29B029BB213439BB26FEA43436FEA3B
:10B7FC0053439AB2D7F8A8301A8070E007F58473D7
:10B80C00A3F584731B681B69002B0CD1D7F8A830E7
:10B81C001B889BB26FEA43436FEA53439AB2D7F843
:10B82C00A8301A805BE007F58473A3F584731B685A
:10B83C001B695B08C7F8E43007F58473A3F58473C0
:10B84C001B681B6903F00103002B04D0D7F8E4300C
:10B85C000133C7F8E430D7F8A8301B889AB2D7F870
:10B86C00E4309BB29B029BB213439AB2D7F8A83038
:10B87C001A8034E007F58473A3F584731B685B7836
:10B88C00012B2CD107F58473A3F582731B68C7F8C1
:10B89C00B43007F58473A3F582731B68B3F850308A
:10B8AC009BB21A46D7F8B4301344C7F8B43007F536
:10B8BC008473A3F584731B681B781A01D7F8B43012
:10B8CC00134403F20443C7F8B03007F58473A3F5AF
:10B8DC0084731B681B699AB2D7F8B0301A8007F5CD
:10B8EC008473A3F582731B68C7F8A43007F58473BF
:10B8FC00A3F584731B685B78002B40F09D8007F5E3
:10B90C008473A3F582731B68C7F89C3007F58473A6
:10B91C00A3F582731B68B3F850309BB21A46D7F864
:10B92C009C301344C7F89C3007F58473A3F58473DB
:10B93C001B681B781A01D7F89C30134403F20C4394
:10B94C00C7F89830D7F898301B889BB2C3F309031B
:10B95C009AB2D7F898301A8007F58473A3F58473DC
:10B96C001B681B693E2B2BD907F58473A3F58473D5
:10B97C001B681B695B09C7F8E03007F58473A3F5F6
:10B98C0084731B681B6903F01F03002B04D1D7F8C9
:10B99C00E030013BC7F8E030D7F898301B889AB2FA
:10B9AC00D7F8E0309BB29B029BB213439BB26FEA79
:10B9BC0043436FEA53439AB2D7F898301A8069E040
:10B9CC0007F58473A3F584731B681B69002B0CD1DA
:10B9DC00D7F898301B889BB26FEA43436FEA534306
:10B9EC009AB2D7F898301A8054E007F58473A3F50F
:10B9FC0084731B681B695B08C7F8E03007F5847318
:10BA0C00A3F584731B681B6903F00103002B04D09E
:10BA1C00D7F8E0300133C7F8E030D7F898301B88FE
:10BA2C009AB2D7F8E0309BB29B029BB213439AB206
:10BA3C00D7F898301A802DE007F58473A3F584733A
:10BA4C001B685B78012B25D107F58473A3F58273F2
:10BA5C001B68B3F850309BB21A46D7F8A430134485
:10BA6C00C7F8A43007F58473A3F584731B681B789F
:10BA7C001A01D7F8A430134403F20C43C7F8A030D2
:10BA8C0007F58473A3F584731B681B699AB2D7F806
:10BA9C00A0301A8007F58473A3F584731B68DB69E7
:10BAAC00002B00F0188207F58473A3F582731A68D3
:10BABC0007F58473A3F584731B681B789B001344F0
:10BACC001B88A7F89630B7F8963003F48043002B08
:10BADC0005D0B7F8963003F04003002B0DD1B7F822
:10BAEC00963003F48043002B40F0F581B7F8963084
:10BAFC0003F04003002B40F0EE8107F58473A3F5AF
:10BB0C0082731A6807F58473A3F584731B681B781A
:10BB1C009B0013441B889BB223F4E04323F0700377
:10BB2C00A7F8943007F58473A3F582731A6807F5A8
:10BB3C008473A3F584731B681B789B001A44B7F8B5
:10BB4C00943043F07F4343F47F0343F4004343F0CA
:10BB5C00C0039BB21380BEE107F58473A3F5847315
:10BB6C001B68DB78012B40F0B48107F58473A3F5D7
:10BB7C0084731B689A6907F58473A3F584731B6837
:10BB8C001B699A4217D907F58473A3F584731B6854
:10BB9C001B69C7F8043107F58473A3F584731B681C
:10BBAC009A69D7F80431D21A07F58473A3F5847314
:10BBBC001B689A610EE007F58473A3F584731B6808
:10BBCC009B69C7F8043107F58473A3F584731B686C
:10BBDC0000229A6107F58473A3F584731B685B7864
:10BBEC00002B40F0858007F58473A3F582731B68E6
:10BBFC00C7F8CC3007F58473A3F582731B68B3F8D0
:10BC0C0050309BB21A46D7F8CC301344C7F8CC301E
:10BC1C0007F58473A3F584731B681B781A01D7F896
:10BC2C00CC30134403F20443C7F8C830D7F8C830FB
:10BC3C001B889BB2C3F309039AB2D7F8C8301A8099
:10BC4C00D7F804313E2B23D9D7F804315B09C7F858
:10BC5C00DC30D7F8043103F01F03002B04D1D7F8E4
:10BC6C00DC30013BC7F8DC30D7F8C8301B889AB2FF
:10BC7C00D7F8DC309BB29B029BB213439BB26FEAAA
:10BC8C0043436FEA53439AB2D7F8C8301A8060E046
:10BC9C00D7F80431002B0CD1D7F8C8301B889BB2D5
:10BCAC006FEA43436FEA53439AB2D7F8C8301A800D
:10BCBC004FE0D7F804315B08C7F8DC30D7F8043113
:10BCCC0003F00103002B04D0D7F8DC300133C7F8A4
:10BCDC00DC30D7F8C8301B889AB2D7F8DC309BB26E
:10BCEC009B029BB213439AB2D7F8C8301A8030E04B
:10BCFC0007F58473A3F584731B685B78012B28D13B
:10BD0C0007F58473A3F582731B68C7F8D43007F565
:10BD1C008473A3F582731B68B3F850309BB21A4638
:10BD2C00D7F8D4301344C7F8D43007F58473A3F58F
:10BD3C0084731B681B781A01D7F8D430134403F2B0
:10BD4C000443C7F8D030D7F804319AB2D7F8D030C2
:10BD5C001A8007F58473A3F582731B68C7F8C43087
:10BD6C0007F58473A3F584731B685B78002B40F094
:10BD7C00858007F58473A3F582731B68C7F8BC3004
:10BD8C0007F58473A3F582731B68B3F850309BB22C
:10BD9C001A46D7F8BC301344C7F8BC3007F5847387
:10BDAC00A3F584731B681B781A01D7F8BC301344B5
:10BDBC0003F20C43C7F8B830D7F8B8301B889BB2E5
:10BDCC00C3F309039AB2D7F8B8301A80D7F8043104
:10BDDC003E2B23D9D7F804315B09C7F8D830D7F8F4
:10BDEC00043103F01F03002B04D1D7F8D830013BEA
:10BDFC00C7F8D830D7F8B8301B889AB2D7F8D830F3
:10BE0C009BB29B029BB213439BB26FEA43436FEA14
:10BE1C0053439AB2D7F8B8301A805CE0D7F80431A3
:10BE2C00002B0CD1D7F8B8301B889BB26FEA434378
:10BE3C006FEA53439AB2D7F8B8301A804BE0D7F870
:10BE4C0004315B08C7F8D830D7F8043103F001038C
:10BE5C00002B04D0D7F8D8300133C7F8D830D7F836
:10BE6C00B8301B889AB2D7F8D8309BB29B029BB2E1
:10BE7C0013439AB2D7F8B8301A802CE007F58473C4
:10BE8C00A3F584731B685B78012B24D107F58473AD
:10BE9C00A3F582731B68B3F850309BB21A46D7F8DF
:10BEAC00C4301344C7F8C43007F58473A3F5847306
:10BEBC001B681B781A01D7F8C430134403F20C43E7
:10BECC00C7F8C030D7F804319AB2D7F8C0301A800E
:10BEDC0001E001233AE007F58473A3F582731A6835
:10BEEC0007F58473A3F584731B681B789B001344BC
:10BEFC001B889BB223F4804323F07003A7F88A308D
:10BF0C00B7F88A3083F48053A7F88A30B7F88A30B0
:10BF1C0083F40053A7F88A3007F58473A3F5827372
:10BF2C001A6807F58473A3F584731B681B789B0050
:10BF3C001A44B7F88A3043F07F4343F47F0343F449
:10BF4C00004343F080039BB213800023184607F58F
:10BF5C008477BD4680BD80B485B000AF7860396011
:10BF6C003B685B78002B20D07A683B681B789B0081
:10BF7C0013441B889BB223F4E04323F04003BB81A2
:10BF8C00BB8983F01003BB817A683B681B789B00EC
:10BF9C001A44BB8943F07F4343F47F0343F40043CB
:10BFAC0043F080039BB213801FE07A683B681B78D8
:10BFBC009B0013441B889BB223F4804323F0700333
:10BFCC00FB81FB8983F48053FB817A683B681B7887
:10BFDC009B001A44FB8943F07F4343F47F0343F4F3
:10BFEC00004343F080039BB21380002318461437A0
:10BFFC00BD4680BC704780B487B000AF78603960B4
:10C00C003B681B7B002B40F09D803B685B78002BD2
:10C01C004CD07A683B681B789B0013441B883B828E
:10C02C003B8A03F04003002B1BD07A683B681B78DB
:10C03C009B0013441B889BB223F4E04323F0700352
:10C04C00FB817A683B681B789B001A44FB8943F0A0
:10C05C007F4343F47F0343F4004343F0C0039BB29C
:10C06C0013803B68DB78012B6CD07A683B681B78BB
:10C07C009B0013441B889BB223F4E04323F0400342
:10C08C00BB81BB8983F02003BB817A683B681B783A
:10C09C009B001A44BB8943F07F4343F47F0343F472
:10C0AC00004343F080039BB213804BE07A683B68FB
:10C0BC001B789B0013441B88FB82FB8A03F4804390
:10C0CC00002B1BD07A683B681B789B0013441B88A1
:10C0DC009BB223F4E04323F07003BB827A683B6885
:10C0EC001B789B001A44BB8A43F07F4343F47F03C5
:10C0FC0043F4404343F080039BB213807A683B685F
:10C10C001B789B0013441B889BB223F4804323F0C1
:10C11C0070037B827B8A83F480537B827B8A83F4DB
:10C12C0000537B827A683B681B789B001A447B8A9D
:10C13C0043F07F4343F47F0343F4004343F0800315
:10C14C009BB21380002318461C37BD4680BC704739
:10C15C0080B483B000AF78600B46FB70FB78002B8B
:10C16C0003D17B688022A3F84C20002318460C379F
:10C17C00BD4680BC704780B483B000AF78600023AC
:10C18C0018460C37BD4680BC704780B483B000AFF6
:10C19C007860002318460C37BD4680BC704780B4CD
:10C1AC0085B000AF78607B68B3F844309BB2FB601D
:10C1BC00FB6818461437BD4680BC704780B483B00A
:10C1CC0000AF78603960002318460C37BD4680BC40
:10C1DC00704780B48BB000AFF860B96011461A4656
:10C1EC000B46FB801346BB80BB8801335B08BB61ED
:10C1FC00FB687B61BB68FB61FB885A007B6913445D
:10C20C0003F580633B62BB697B621FE0FB691B78B3
:10C21C007B82FB6901331B781BB21B021AB2B7F984
:10C22C00123013431BB27B823B6A7A8A1A803B6AB8
:10C23C0002333B623B6A02333B62FB690133FB61B5
:10C24C00FB690133FB617B6A013B7B627B6A002BE0
:10C25C00DCD100BF00BF2C37BD4680BC704780B41A
:10C26C008BB000AFF860B96011461A460B46FB80E4
:10C27C001346BB80BB885B089BB2BB61FB687B61D0
:10C28C00BB68FB61FB885A007B69134403F5806330
:10C29C003B62BB697B621BE03B6A1B889BB23B61C8
:10C2AC003B6A02333B623B69DAB2FB691A70FB6989
:10C2BC000133FB613B691B0ADAB2FB691A70FB693B
:10C2CC000133FB613B6A02333B627B6A013B7B625D
:10C2DC007B6A002BE0D1BB8803F001039BB2002BDF
:10C2EC0007D03B6A1B889BB23B613B69DAB2FB69A6
:10C2FC001A7000BF2C37BD4680BC704780B584B027
:10C30C0000AF78600B46FB700023FB737B681B7CD3
:10C31C00002B15D14FF4007302228121786801F0B3
:10C32C0000FF7B680122DA624FF4007302220121C4
:10C33C00786801F0F6FE7B680122C3F86C2112E0EC
:10C34C00402302228121786801F0EBFE7B680122F8
:10C35C00DA62402302220121786801F0E2FE7B6858
:10C36C000122C3F86C21082303228221786801F092
:10C37C00D8FE7B6801221A644FF4077001F0F8FFB5
:10C38C0002467B68C3F8B8227B68D3F8B832002B1E
:10C39C0002D10123FB7326E07B68D3F8B832BB6073
:10C3AC007B68D3F8BC321B689847BB680022C3F883
:10C3BC001422BB680022C3F818227B681B7C002B5C
:10C3CC0009D1BB68D3F804224FF4007301217868BB
:10C3DC0001F097FF07E0BB68D3F80422402301214A
:10C3EC00786801F08EFFFB7B18461037BD4680BD88
:10C3FC0080B584B000AF78600B46FB700023FB73F4
:10C40C008121786801F0B3FE7B680022DA62012199
:10C41C00786801F0ACFE7B680022C3F86C218221A5
:10C42C00786801F0A4FE7B6800221A647B68D3F85C
:10C43C00B832002B0ED07B68D3F8BC325B689847BF
:10C44C007B68D3F8B832184601F09EFF7B68002257
:10C45C00C3F8B822FB7B18461037BD4680BD80B5AB
:10C46C0086B000AF786039607B68D3F8B8323B6136
:10C47C000023FB730023BB810023FB753B681B78F7
:10C48C0003F06003002B39D0202B7FD13B68DB8875
:10C49C00002B29D03B681B785BB2002B11DA7B6830
:10C4AC00D3F8BC329B683A68507839693A68D288BC
:10C4BC00984739693B68DB881A46786801F006FAB8
:10C4CC006BE03B685A783B6983F800223B68DB8859
:10C4DC00DAB23B6983F8012239693B68DB881A467A
:10C4EC00786801F021FA58E07B68D3F8BC329B687D
:10C4FC003A6850780022396898474EE03B685B7880
:10C50C000B2B2ED00B2B38DC002B02D00A2B14D08B
:10C51C0033E07B6893F89C32032B07D107F10C03B3
:10C52C0002221946786801F0D1F92EE03968786852
:10C53C0001F062F90223FB7527E07B6893F89C32CB
:10C54C00032B07D107F10F0301221946786801F07C
:10C55C00BDF91AE03968786801F04EF90223FB75D1
:10C56C0013E07B6893F89C32032B0DD03968786804
:10C57C0001F042F90223FB7506E03968786801F096
:10C58C003BF90223FB7500E000BF06E039687868D0
:10C59C0001F032F90223FB7500BFFB7D18461837FA
:10C5AC00BD4680BD80B584B000AF78600B46FB7093
:10C5BC007B68D3F8B832FB607B68D3F8C032BB60C1
:10C5CC007B68D3F8B832002B3AD0FA7879681346E6
:10C5DC009B0013449B000B441C331B68002B29D07D
:10C5EC00FA78796813469B0013449B000B441C3368
:10C5FC001A68F978B8680B469B000B44DB000344BF
:10C60C0020331B68B2FBF3F101FB03F3D31A002BAD
:10C61C0010D1FA78796813469B0013449B000B44A5
:10C62C001C3300221A60F97800230022786801F08C
:10C63C0045FE03E0FB680022C3F81422002300E04F
:10C64C00022318461037BD4680BD80B584B000AFBC
:10C65C0078600B46FB707B68D3F8B832FB60FB78D4
:10C66C001946786801F070FE0246FB68C3F80C228C
:10C67C007B68D3F8B832002B0DD07B68D3F8BC3272
:10C68C00DB68FA68D2F80402FA6802F50372114604
:10C69C009847002300E0022318461037BD4680BDA2
:10C6AC0080B584B000AF78607B68D3F8B832FB609B
:10C6BC007B68D3F8BC32002B14D0FB6893F80032A3
:10C6CC00FF2B0FD07B68D3F8BC329B68FA6892F8CA
:10C6DC000002F968FA6892F801229847FB68FF2279
:10C6EC0083F80022002318461037BD4680BD000099
:10C6FC0080B483B000AF78607B6843221A80034B10
:10C70C0018460C37BD4680BC704700BFA400002003
:10C71C0080B483B000AF78607B6843221A80034BEF
:10C72C0018460C37BD4680BC704700BF6000002027
:10C73C0080B483B000AF78607B6843221A80034BCF
:10C74C0018460C37BD4680BC704700BFE80000207F
:10C75C0080B483B000AF78607B680A221A80034BE8
:10C76C0018460C37BD4680BC704700BF1C0000202B
:10C77C0080B485B000AF786039600223FB733B68EE
:10C78C00002B05D07B683A68C3F8BC220023FB73EE
:10C79C00FB7B18461437BD4680BC704780B487B00D
:10C7AC0000AFF860B9601346FB80FB68D3F8B83271
:10C7BC007B617B69BA68C3F80822FA887B69C3F885
:10C7CC001022002318461C37BD4680BC704780B42D
:10C7DC0085B000AF786039607B68D3F8B832FB6005
:10C7EC00FB683A68C3F80422002318461437BD4688
:10C7FC0080BC704780B584B000AF78607B68D3F89C
:10C80C00B832FB607B68D3F8B832002B1CD0FB68C5
:10C81C00D3F81432002B15D1FB680122C3F8142273
:10C82C00FB68D3F810227B681A63FB68D3F80822E4
:10C83C00FB68D3F810329BB28121786801F03EFD81
:10C84C00002302E0012300E0022318461037BD4606
:10C85C0080BD80B584B000AF78607B68D3F8B83207
:10C86C00FB607B68D3F8B832002B17D07B681B7C3D
:10C87C00002B09D1FB68D3F804224FF4007301217B
:10C88C00786801F03EFD07E0FB68D3F804224023F2
:10C89C000121786801F035FD002300E002231846E1
:10C8AC001037BD4680BD80B584B000AFF860B9606C
:10C8BC001346FB71FB68002B01D102231AE0FB68C5
:10C8CC00D3F8B432002B03D0FB680022C3F8B42297
:10C8DC00BB68002B03D0FB68BA68C3F8B022FB68B6
:10C8EC00012283F89C22FB68FA791A70F86801F02F
:10C8FC00A3FB002318461037BD4680BD80B485B01D
:10C90C0000AF786039600023FB733B68002B06D0C6
:10C91C007B683A68C3F8B4220023FB7301E002235E
:10C92C00FB73FB7B18461437BD4680BC704780B543
:10C93C0082B000AF7860786801F0D8FB002318460D
:10C94C000837BD4680BD80B483B000AF786000234B
:10C95C0018460C37BD4680BC704780B584B000AF1C
:10C96C0078600B46FB700223FB737B68D3F8B43200
:10C97C00002B0CD07B68D3F8B4321B68FA781146C4
:10C98C00786898470346002B01D10023FB73FB7B8F
:10C99C0018461037BD4680BD80B582B000AF7860B8
:10C9AC000B46FB707B68D3F8B4325B68FA7811469F
:10C9BC0078689847002318460837BD4680BD80B577
:10C9CC0082B000AF786039607B6803F52A733968F0
:10C9DC00184600F0D8FE7B680122C3F894227B68CD
:10C9EC00B3F8AE321A467B68C3F898227B6893F88A
:10C9FC00A83203F01F03022B16D0022B1CD8002BDD
:10CA0C0002D0012B08D017E07B6803F52A73194676
:10CA1C00786800F0CBF91AE07B6803F52A731946A5
:10CA2C00786800F02DFA12E07B6803F52A7319463A
:10CA3C00786800F06DFA0AE07B6893F8A83223F06E
:10CA4C007F03DBB21946786801F0B0FB00BF00230E
:10CA5C0018460837BD4680BD80B586B000AFF8607B
:10CA6C000B467A60FB72FB7A002B4BD1FB6803F50B
:10CA7C00AA737B61FB68D3F89432032B34D17B69A6
:10CA8C00DA687B691B699A4219D97B69DA687B6918
:10CA9C001B69D21A7B69DA607B69DA687B691B696E
:10CAAC009A4203D27B69DB689BB202E07B691B690B
:10CABC009BB21A467968F86800F054FF38E0FB68BE
:10CACC00D3F8B4321B69002B0AD0FB6893F89C3264
:10CADC00032B05D1FB68D3F8B4321B69F86898476F
:10CAEC00F86800F051FF23E0FB68D3F89432052B73
:10CAFC001ED1FB680022C3F894220021F86801F0D3
:10CB0C0055FB15E0FB68D3F8B4329B69002B0DD0B4
:10CB1C00FB6893F89C32032B08D1FB68D3F8B43232
:10CB2C009B69FA7A1146F868984701E0022300E005
:10CB3C00002318461837BD4680BD80B586B000AFBF
:10CB4C00F8600B467A60FB72FB7A002B7FD1FB6896
:10CB5C0014337B61FB68D3F89432022B5CD17B6974
:10CB6C00DA687B691B699A4215D97B69DA687B693B
:10CB7C001B69D21A7B69DA607B69DB689BB21A4647
:10CB8C007968F86800F0BEFE002300220021F868E6
:10CB9C0001F0B7FB4EE07B699B687A691269B3FBC5
:10CBAC00F2F101FB02F29B1A002B1CD17B699A68F3
:10CBBC007B691B699A4216D37B699A68FB68D3F828
:10CBCC0098329A420FD200220021F86800F09AFEA7
:10CBDC00FB680022C3F89822002300220021F86889
:10CBEC0001F08FFB26E0FB68D3F8B432DB68002B36
:10CBFC000AD0FB6893F89C32032B05D1FB68D3F861
:10CC0C00B432DB68F86898478021F86801F0CEFAF6
:10CC1C00F86800F0CCFE0DE0FB68D3F89432042BDE
:10CC2C0004D0FB68D3F89432002B03D18021F86830
:10CC3C0001F0BCFAFB6893F8A032012B1DD1F86807
:10CC4C00FFF781FEFB68002283F8A02215E0FB6849
:10CC5C00D3F8B4325B69002B0DD0FB6893F89C328F
:10CC6C00032B08D1FB68D3F8B4325B69FA7A11460E
:10CC7C00F868984701E0022300E0002318461837B3
:10CC8C00BD4680BD80B582B000AF786040230022E5
:10CC9C000021786801F045FA7B680122C3F858211D
:10CCAC007B684022C3F864214023002280217868ED
:10CCBC0001F037FA7B6801229A617B6840225A6244
:10CCCC007B68012283F89C227B680022C3F89422A3
:10CCDC007B6800225A607B680022C3F8A4227B6820
:10CCEC00D3F8B832002B09D07B68D3F8B4325B6828
:10CCFC007A685268D2B21146786898470023184671
:10CD0C000837BD4680BD80B483B000AF78600B4659
:10CD1C00FB707B68FA781A74002318460C37BD46F2
:10CD2C0080BC704780B483B000AF78607B6893F8A8
:10CD3C009C227B6883F89D227B68042283F89C22CA
:10CD4C00002318460C37BD4680BC704780B483B0B6
:10CD5C0000AF78607B6893F89C32042B05D17B681C
:10CD6C0093F89D227B6883F89C22002318460C378D
:10CD7C00BD4680BC704780B582B000AF78607B68E0
:10CD8C0093F89C32032B0BD17B68D3F8B432DB695C
:10CD9C00002B05D07B68D3F8B432DB6978689847F0
:10CDAC00002318460837BD4680BD000080B584B00E
:10CDBC0000AF786039600023FB733B681B7803F08D
:10CDCC006003402B05D0402B4FD8002B09D0202BD3
:10CDDC004BD17B68D3F8B4329B6839687868984734
:10CDEC0048E03B685B78092B39D801A252F823F054
:10CDFC004DCE000861CE00086BCE000857CE00085F
:10CE0C006BCE00082FCE000825CE00086BCE000894
:10CE1C0043CE000839CE00083968786800F0DCF998
:10CE2C0022E03968786800F03FFB1DE039687868CB
:10CE3C0000F07EFB18E03968786800F007FC13E01E
:10CE4C003968786800F037FC0EE03968786800F0D3
:10CE5C0065FC09E03968786800F074FC04E0396816
:10CE6C00786800F0C9FC00BF04E03968786800F00D
:10CE7C00C3FC00BFFB7B18461037BD4680BD00BF0E
:10CE8C0080B584B000AF786039600023FB733B68D9
:10CE9C001B7803F06003402B05D0402B2ED8002BC1
:10CEAC0001D0202B2AD17B6893F89C32013B022BBA
:10CEBC001DD83B689B88DBB2012B13D87B68D3F859
:10CECC00B4329B683968786898470346FB733B68B3
:10CEDC00DB88002B10D1FB7B002B0DD1786800F088
:10CEEC0053FD09E03968786800F086FC04E0396885
:10CEFC00786800F081FC00E000BF04E039687868D5
:10CF0C0000F07AFC00BF002318461037BD4680BDE8
:10CF1C0080B584B000AF786039600023FB733B6848
:10CF2C009B88BB733B681B7803F06003402B07D0D6
:10CF3C00402B00F24681002B0AD0202B40F041817F
:10CF4C007B68D3F8B4329B683968786898473DE1C0
:10CF5C003B681B7803F06003202B0AD17B68D3F865
:10CF6C00B4329B683968786898470346FB73FB7B3F
:10CF7C002DE13B685B78032B07D0032B00F31B815F
:10CF8C00002B72D0012B3AD015E17B6893F89C32C0
:10CF9C00022B02D0032B15D02BE0BB7B002B0CD02B
:10CFAC00BB7B802B09D0BB7B1946786801F0FEF85F
:10CFBC008021786801F0FAF820E03968786800F090
:10CFCC001BFC1BE03B685B88002B0ED1BB7B002B52
:10CFDC000BD0BB7B802B08D03B68DB88002B04D1AB
:10CFEC00BB7B1946786801F0E1F8786800F0CCFC5E
:10CFFC0004E03968786800F0FFFB00BFE0E07B6874
:10D00C0093F89C32022B02D0032B15D026E0BB7B6D
:10D01C00002B0CD0BB7B802B09D0BB7B19467868CE
:10D02C0001F0C4F88021786801F0C0F81CE0396880
:10D03C00786800F0E1FB17E03B685B88002B12D1AD
:10D04C00BB7B03F07F03002B04D0BB7B19467868B5
:10D05C0001F0CBF8786800F097FC04E03968786848
:10D06C0000F0CAFB00E000BFAAE07B6893F89C329A
:10D07C00022B02D0032B32D097E0BB7B002B07D0C6
:10D08C00BB7B802B04D03968786800F0B5FB91E04D
:10D09C0097F90E30002B0BDABB7B03F07F021346A3
:10D0AC009B0013449B0010337A68134404330BE049
:10D0BC00BB7B03F07F0213469B0013449B0003F5DC
:10D0CC00A8737A6813440433BB60BB6800221A60EF
:10D0DC00BB6802221946786800F0F8FB6AE097F901
:10D0EC000E30002B11DABB7B03F00F02796813466C
:10D0FC009B0013449B000B4418331B68002B17D167
:10D10C003968786800F078FB54E0BB7B03F00F02C1
:10D11C00796813469B0013449B000B4403F5AC73D6
:10D12C001B68002B04D13968786800F065FB41E07E
:10D13C0097F90E30002B0BDABB7B03F07F02134602
:10D14C009B0013449B0010337A68134404330BE0A8
:10D15C00BB7B03F07F0213469B0013449B0003F53B
:10D16C00A8737A6813440433BB60BB7B002B02D0DA
:10D17C00BB7B802B03D1BB6800221A600EE0BB7B0B
:10D18C001946786801F050F80346002B03D0BB68B1
:10D19C0001221A6002E0BB6800221A60BB680222FE
:10D1AC001946786800F092FB04E03968786800F062
:10D1BC0023FB00BF04E03968786800F01DFB00BF5A
:10D1CC0004E03968786800F017FB00BFFB7B184659
:10D1DC001037BD4680BD000080B584B000AF7860CC
:10D1EC00396000233B810023FB600023FB723B680A
:10D1FC005B881B0A9BB2013B062B00F2288101A223
:10D20C0052F823F02DD2000845D2000885D2000830
:10D21C005BD400085BD40008FBD3000827D40008BB
:10D22C007B68D3F8B0321B687A68127C07F108016E
:10D23C0010469847F86012E17B681B7C002B0DD1DF
:10D24C007B68D3F8B4329B6A07F108021046984702
:10D25C00F860FB68013302221A7000E17B68D3F896
:10D26C00B432DB6A07F1080210469847F860FB6895
:10D27C00013302221A70F2E03B685B88DBB2052BAB
:10D28C0000F2AC8001A252F823F000BFB1D200082A
:10D29C00E5D2000819D300084DD3000881D300084B
:10D2AC00B5D300087B68D3F8B0325B68002B0BD089
:10D2BC007B68D3F8B0325B687A68127C07F108019E
:10D2CC0010469847F86091E03968786800F094FA55
:10D2DC00FB7A0133FB7289E07B68D3F8B0329B6830
:10D2EC00002B0BD07B68D3F8B0329B687A68127C29
:10D2FC0007F1080110469847F86077E039687868BC
:10D30C0000F07AFAFB7A0133FB726FE07B68D3F89A
:10D31C00B032DB68002B0BD07B68D3F8B032DB6803
:10D32C007A68127C07F1080110469847F8605DE0B6
:10D33C003968786800F060FAFB7A0133FB7255E0CB
:10D34C007B68D3F8B0321B69002B0BD07B68D3F809
:10D35C00B0321B697A68127C07F1080110469847B5
:10D36C00F86043E03968786800F046FAFB7A0133DC
:10D37C00FB723BE07B68D3F8B0325B69002B0BD0BF
:10D38C007B68D3F8B0325B697A68127C07F10801CC
:10D39C0010469847F86029E03968786800F02CFA54
:10D3AC00FB7A0133FB7221E07B68D3F8B0329B69C6
:10D3BC00002B0BD07B68D3F8B0329B697A68127C57
:10D3CC0007F1080110469847F8600FE03968786853
:10D3DC0000F012FAFB7A0133FB7207E039687868C7
:10D3EC0000F00AFAFB7A0133FB7238E037E07B6815
:10D3FC001B7C002B09D17B68D3F8B4325B6B07F133
:10D40C00080210469847F86029E03968786800F0FF
:10D41C00F3F9FB7A0133FB7221E07B681B7C002B58
:10D42C000DD17B68D3F8B4321B6B07F108021046A0
:10D43C009847F860FB68013307221A700FE03968CF
:10D44C00786800F0D9F9FB7A0133FB7207E0396890
:10D45C00786800F0D1F9FB7A0133FB7200BFFB7ADC
:10D46C00002B1CD13B89002B11D03B68DB88002B97
:10D47C000DD03B68DA883B89934228BF13469BB298
:10D48C003B813B891A46F968786800F01FFA3B68C3
:10D49C00DB88002B04D1786800F076FA00E000BF3E
:10D4AC001037BD4680BD00BF80B584B000AF78603A
:10D4BC0039603B689B88002B30D13B68DB88002BA4
:10D4CC002CD13B685B887F2B28D83B685B88DBB210
:10D4DC0003F07F03FB737B6893F89C32032B04D11E
:10D4EC003968786800F088F91DE07B68FA7B83F86E
:10D4FC009E22FB7B1946786800F0C1FE786800F02C
:10D50C0043FAFB7B002B04D07B68022283F89C221D
:10D51C0009E07B68012283F89C2204E03968786872
:10D52C0000F06AF900BF00BF1037BD4680BD000097
:10D53C0080B582B000AF786039603B685B88DAB246
:10D54C00414B1A70404B1B78012B04D93968786811
:10D55C0000F052F975E07B6893F89C32022B02D0F4
:10D56C00032B23D062E0384B1B78002B1AD0364BA0
:10D57C001B781A467B685A607B68032283F89C22CE
:10D58C00314B1B7819467868FFF7E7F90346022BF5
:10D59C0004D13968786800F02FF952E0786800F00F
:10D5AC00F3F94EE0786800F0EFF94AE0264B1B786F
:10D5BC00002B12D17B68022283F89C22224B1B7811
:10D5CC001A467B685A60204B1B7819467868FFF71F
:10D5DC00E3F9786800F0D8F933E01B4B1B781A4656
:10D5EC007B685B689A421DD07B685B68DBB219462E
:10D5FC007868FFF7D1F9144B1B781A467B685A6090
:10D60C00114B1B7819467868FFF7A7F90346022BD4
:10D61C0004D13968786800F0EFF812E0786800F00F
:10D62C00B3F90EE0786800F0AFF90AE03968786871
:10D63C0000F0E2F8044B1B7819467868FFF7ACF958
:10D64C0000BF0837BD4680BD9804002080B582B06D
:10D65C0000AF786039603B68DB88012B04D03968F7
:10D66C00786800F0C9F822E07B6893F89C32022BB2
:10D67C0002DC002B03DC15E0032B0BD012E07B68E3
:10D68C0000229A607B68083301221946786800F002
:10D69C001DF90CE07B68043301221946786800F010
:10D6AC0015F904E03968786800F0A6F800BF00BFEF
:10D6BC000837BD4680BD80B582B000AF7860396058
:10D6CC007B6893F89C32013B022B1ED83B68DB88AD
:10D6DC00022B04D03968786800F08EF81AE07B6869
:10D6EC000122DA607B68D3F8A432002B05D07B686A
:10D6FC00DB6843F002027B68DA607B680C33022241
:10D70C001946786800F0E2F804E03968786800F0AF
:10D71C0073F800BF00BF0837BD4680BD80B582B02E
:10D72C0000AF786039603B685B88012B06D17B6861
:10D73C000122C3F8A422786800F026F900BF08374C
:10D74C00BD4680BD80B582B000AF786039607B6823
:10D75C0093F89C32013B022B0BD83B685B88012B66
:10D76C000CD17B680022C3F8A422786800F00CF975
:10D77C0004E03968786800F03FF800E000BF00BFB3
:10D78C000837BD4680BD80B483B000AF7860396087
:10D79C003B681A787B681A703B685A787B685A70B9
:10D7AC003B6802331B781A463B6803331B781B0219
:10D7BC009BB213449AB27B685A803B6804331B7843
:10D7CC001A463B6805331B781B029BB213449AB272
:10D7DC007B689A803B6806331B781A463B68073394
:10D7EC001B781B029BB213449AB27B68DA8000BF91
:10D7FC000C37BD4680BC704780B582B000AF7860F6
:10D80C0039608021786800F0D1FC0021786800F044
:10D81C00CDFC00BF0837BD4680BD80B586B000AFDB
:10D82C00F860B9607A600023FB75FB68002B32D07E
:10D83C00F86800F034F8034601339BB25B009AB2EF
:10D84C007B681A80FB7D5A1CFA751A46BB68134418
:10D85C007A6812781A70FB7D5A1CFA751A46BB68E6
:10D86C00134403221A7012E0FB685A1CFA60FA7D0A
:10D87C00511CF9751146BA680A441B781370FB7D6C
:10D88C005A1CFA751A46BB68134400221A70FB68BE
:10D89C001B78002BE8D100BF1837BD4680BD80B483
:10D8AC0085B000AF78600023FB7305E0FB7B013390
:10D8BC00FB737B6801337B607B681B78002BF5D195
:10D8CC00FB7B18461437BD4680BC704780B584B0CE
:10D8DC0000AFF860B9601346FB80FB680222C3F806
:10D8EC009422FA88FB68DA61FA88FB681A62FB8872
:10D8FC00BA680021F86800F0E1FC002318461037E4
:10D90C00BD4680BD80B584B000AFF860B9601346E9
:10D91C00FB80FB88BA680021F86800F0CFFC00237C
:10D92C0018461037BD4680BD80B584B000AFF86096
:10D93C00B9601346FB80FB680322C3F89422FA8873
:10D94C00FB68C3F85C21FA88FB68C3F86021FB888C
:10D95C00BA680021F86800F0D4FC00231846103790
:10D96C00BD4680BD80B584B000AFF860B960134689
:10D97C00FB80FB88BA680021F86800F0C2FC002329
:10D98C0018461037BD4680BD80B582B000AF7860B8
:10D99C007B680422C3F894220023002200217868BB
:10D9AC0000F08CFC002318460837BD4680BD80B5BE
:10D9BC0082B000AF78607B680522C3F89422002304
:10D9CC0000220021786800F09CFC002318460837E0
:10D9DC00BD4680BD80B500AF002212491248FEF74B
:10D9EC0062FF0346002B01D0F5F76CFE0F490E4881
:10D9FC00FEF784FF0346002B01D0F5F763FE0C49BC
:10DA0C000948FEF7B5FE0346002B01D0F5F75AFE88
:10DA1C000548FEF78CFF0346002B01D0F5F752FEAC
:10DA2C0000BF80BD3C0100209C0400202800002089
:10DA3C002C01002080B485B000AF786039601EE006
:10DA4C00144B1B889BB201339BB2DBB2FB81FA896E
:10DA5C00114B1B889BB2DBB29A4203D17B6801331A
:10DA6C007B600CE07B685A1C7A600A4A128892B27E
:10DA7C00D2B21978094B9954064AFB8913803B683A
:10DA8C005A1E3A60002BDBD100BF00BF1437BD46D5
:10DA9C0080BC70476010002062100020600F0020D6
:10DAAC0080B400AF064B1B889AB2064B1B889BB206
:10DABC00D31A9BB2DBB21846BD4680BC704700BF80
:10DACC00601000206210002080B483B000AF104BB7
:10DADC001B889AB20F4B1B889BB29A4202D14FF013
:10DAEC00FF3310E00A4B1B889BB2DBB20A4AD35CB3
:10DAFC007B60074B1B889BB201339BB2DBB29AB2A3
:10DB0C00034B1A807B6818460C37BD4680BC7047A7
:10DB1C006210002060100020600F002080B500AF64
:10DB2C00002205490548FEF739FE05490348FEF772
:10DB3C004EFE0023184680BD600B00209C04002084
:10DB4C006007002080B400AF00231846BD4680BC9F
:10DB5C007047000080B483B000AF03463960FB719E
:10DB6C001346BB80FB79232B4AD801A252F823F031
:10DB7C000DDC00080DDC00080DDC00080DDC0008D5
:10DB8C000DDC00080DDC00080DDC00080DDC0008C5
:10DB9C000DDC00080DDC00080DDC00080DDC0008B5
:10DBAC000DDC00080DDC00080DDC00080DDC0008A5
:10DBBC000DDC00080DDC00080DDC00080DDC000895
:10DBCC000DDC00080DDC00080DDC00080DDC000885
:10DBDC000DDC00080DDC00080DDC00080DDC000875
:10DBEC000DDC00080DDC00080DDC00080DDC000865
:10DBFC000DDC00080DDC00080DDC00080DDC000855
:10DC0C0000BF002318460C37BD4680BC704700BFD0
:10DC1C0080B582B000AF786039603B681B68002B20
:10DC2C0005D03B681B6819467868FFF703FF7968D5
:10DC3C000548FEF7CCFD0448FEF70BFE0023184602
:10DC4C000837BD4680BD00BF9C04002080B584B061
:10DC5C0000AF78600B467B800023FB730D4BD3F831
:10DC6C00B832BB60BB68D3F81432002B01D001234F
:10DC7C000BE07B881A4679680648FEF78FFD05484D
:10DC8C00FEF7B8FD0346FB73FB7B18461037BD4609
:10DC9C0080BD00BF9C04002080B483B000AF03465D
:10DCAC003960FB713B6812221A80034B18460C3703
:10DCBC00BD4680BC704700BF5801002080B483B0C3
:10DCCC0000AF03463960FB713B6804221A80034B9A
:10DCDC0018460C37BD4680BC704700BF6C01002055
:10DCEC0080B582B000AF03463960FB71FB79002B25
:10DCFC0005D13A6807490848FFF78FFD04E03A68F8
:10DD0C0004490548FFF789FD024B18460837BD4604
:10DD1C0080BD00BF64100020D0F3000880B582B035
:10DD2C0000AF03463960FB713A6804490448FFF7B9
:10DD3C0074FD024B18460837BD4680BD64100020A8
:10DD4C00E8F3000880B582B000AF03463960FB7180
:10DD5C003B681A221A8000F043F8024B1846083729
:10DD6C00BD4680BD7001002080B582B000AF034677
:10DD7C003960FB71FB79002B05D13A6807490848DB
:10DD8C00FFF74BFD04E03A6804490548FFF745FDF1
:10DD9C00024B18460837BD4680BD00BF64100020FA
:10DDAC00FCF3000880B582B000AF03463960FB710C
:10DDBC00FB79002B05D13A6807490848FFF72DFD80
:10DDCC0004E03A6804490548FFF727FD024B184662
:10DDDC000837BD4680BD00BF6410002008F4000861
:10DDEC0080B584B000AF0F4B1B68FB600E4B1B68FB
:10DDFC00BB600E4B1B687B60FA687B681344FB604E
:10DE0C00FB68002B09D008220949F86800F014F8C7
:10DE1C0004220849B86800F00FF800BF1037BD465F
:10DE2C0080BD00BFE8F7FF1FECF7FF1FF0F7FF1FE7
:10DE3C00720100208201002080B487B000AFF8602E
:10DE4C00B9601346FB710023FB750023FB7527E0BB
:10DE5C00FB681B0F092B0BD8FB681B0FDAB2FB7D81
:10DE6C005B001946BB680B443032D2B21A700AE020
:10DE7C00FB681B0FDAB2FB7D5B001946BB680B44D9
:10DE8C003732D2B21A70FB681B01FB60FB7D5B0062
:10DE9C000133BA68134400221A70FB7D0133FB7501
:10DEAC00FA7DFB799A42D3D300BF00BF1C37BD4625
:10DEBC0080BC704780B584B000AF78607B681B680D
:10DECC000D4A934213D10D4BDB690C4A43F400030A
:10DEDC00D3610A4BDB6903F40003FB60FB6800228F
:10DEEC0000211420F7F7DBFD1420F7F7F4FD00BF39
:10DEFC001037BD4680BD00BF005C004000100240E2
:10DF0C0080B582B000AF78607B68D3F8D4227B6890
:10DF1C0003F5267319461046FEF751FD00BF08376E
:10DF2C00BD4680BD80B582B000AF78600B46FB70FB
:10DF3C007B68D3F8D402FA78796813469B001344B3
:10DF4C00DB000B4403F5B2731A68FB781946FEF735
:10DF5C0083FD00BF0837BD4680BD80B582B000AFE1
:10DF6C0078600B46FB707B68D3F8D402FA7879683A
:10DF7C0013469B001344DB000B4424331A68FB78D4
:10DF8C001946FEF7DAFD00BF0837BD4680BD80B5E7
:10DF9C0082B000AF78607B68D3F8D4321846FEF7B5
:10DFAC00EAFE00BF0837BD4680BD80B584B000AF27
:10DFBC0078600123FB737B689B79022B01D0F5F70A
:10DFCC0081FB7B68D3F8D432FA7B11461846FEF7F6
:10DFDC009AFE7B68D3F8D4321846FEF753FE00BF86
:10DFEC001037BD4680BD000080B582B000AF7860B0
:10DFFC007B68D3F8D4321846FEF794FE7B689B7A84
:10E00C00002B05D0044B1B69034A43F00603136134
:10E01C0000BF0837BD4680BD00ED00E080B582B082
:10E02C0000AF78607B68D3F8D4321846FEF78EFECA
:10E03C0000BF0837BD4680BD80B582B000AF7860A8
:10E04C00284A7B68C2F8D4327B68264AC3F8C022BF
:10E05C00244B254A1A60234B08221A71214B0222A9
:10E06C009A71204B00229A721E4B0022DA721D4BC1
:10E07C0000221A731B48F8F7F0FA0346002B01D064
:10E08C00F5F720FB7B68D3F8C0021823002200218F
:10E09C00FAF701F87B68D3F8C002582300228021DC
:10E0AC00F9F7F9FF7B68D3F8C002C0230022812165
:10E0BC00F9F7F1FF7B68D3F8C0024FF488730022A4
:10E0CC000121F9F7E8FF7B68D3F8C0024FF48073A5
:10E0DC0000228221F9F7DFFF002318460837BD46DE
:10E0EC0080BD00BF64120020005C004080B584B08D
:10E0FC0000AF78600023FB730023BB737B68D3F8FD
:10E10C00C0321846F8F79FFB0346FB73FB7B18469F
:10E11C0000F04EF90346BB73BB7B18461037BD4667
:10E12C0080BD80B584B000AF7860084611461A46B1
:10E13C000346FB700B46BB7013463B800023FB73FE
:10E14C000023BB737B68D3F8C002BB783A88F9789C
:10E15C00F8F7F3FC0346FB73FB7B184600F028F939
:10E16C000346BB73BB7B18461037BD4680BD80B5DC
:10E17C0084B000AF78600B46FB700023FB73002368
:10E18C00BB737B68D3F8C032FA7811461846F8F79F
:10E19C0031FD0346FB73FB7B184600F009F903467F
:10E1AC00BB73BB7B18461037BD4680BD80B584B0B1
:10E1BC0000AF78600B46FB700023FB730023BB732E
:10E1CC007B68D3F8C032FA7811461846F8F7D9FDB7
:10E1DC000346FB73FB7B184600F0EAF80346BB735F
:10E1EC00BB7B18461037BD4680BD80B584B000AFF0
:10E1FC0078600B46FB700023FB730023BB737B68BA
:10E20C00D3F8C032FA7811461846F8F71AFE0346CE
:10E21C00FB73FB7B184600F0CBF80346BB73BB7B50
:10E22C0018461037BD4680BD80B485B000AF78600D
:10E23C000B46FB707B68D3F8C032FB6097F9033058
:10E24C00002B0BDAFB7803F07F02F96813469B0076
:10E25C001344DB000B4412331B780BE0FB7803F008
:10E26C007F02F96813469B001344DB000B4403F553
:10E27C00A9731B7818461437BD4680BC704780B50F
:10E28C0084B000AF78600B46FB700023FB73002357
:10E29C00BB737B68D3F8C032FA7811461846F8F78E
:10E2AC0028FC0346FB73FB7B184600F081F8034601
:10E2BC00BB73BB7B18461037BD4680BD80B586B09E
:10E2CC0000AFF8607A601A460B46FB7213463B812E
:10E2DC000023FB750023BB75FB68D3F8C0023B8998
:10E2EC00F97A7A68F8F716FD0346FB75FB7D18463C
:10E2FC0000F05EF80346BB75BB7D18461837BD466B
:10E30C0080BD80B586B000AFF8607A601A460B46C7
:10E31C00FB7213463B810023FB750023BB75FB6826
:10E32C00D3F8C0023B89F97A7A68F8F7ABFC03465C
:10E33C00FB75FB7D184600F03BF80346BB75BB7DB7
:10E34C0018461837BD4680BD80B582B000AF7860E6
:10E35C000B46FB707B68D3F8C032FA78114618462E
:10E36C00F8F7C1FC034618460837BD4680BD0000CF
:10E37C0080B483B000AF7860024B18460C37BD46B2
:10E38C0080BC70473C15002080B483B000AF78602F
:10E39C0000BF0C37BD4680BC704780B483B000AF63
:10E3AC0078600B46FB7000BF0C37BD4680BC7047D5
:10E3BC0080B485B000AF0346FB710023FB73FB797F
:10E3CC00032B17D801A252F823F000BFE9E3000891
:10E3DC00EFE30008F5E30008FBE300080023FB7300
:10E3EC000BE00223FB7308E00123FB7305E002231F
:10E3FC00FB7302E00223FB7300BFFB7B1846143750
:10E40C00BD4680BC704700BF0EB46FF0004110B524
:10E41C0000249DB01FAB029006900791049109480F
:10E42C00094953F8042B0591006802A901931B9428
:10E43C0000F092F9029B1C701DB0BDE8104003B0B7
:10E44C00704700BF8C0100200802FFFF0346024406
:10E45C00934200D1704703F8011BF9E7014B186890
:10E46C00704700BF8C01002070B500260C4D0D4C80
:10E47C00641BA410A64209D100F076FC00260A4DBC
:10E48C000A4C641BA410A64205D170BD55F8043B80
:10E49C0098470136EEE755F8043B98470136F2E70A
:10E4AC0080F5000880F5000880F5000884F5000868
:10E4BC007047704738B50546002940D051F8043CE8
:10E4CC000C1F002BB8BFE41800F0DEF81C4A1368D0
:10E4DC0033B9636014602846BDE8384000F0DAB800
:10E4EC00A34208D9206821188B4201BF19685B68C8
:10E4FC0009182160EDE71A465B680BB1A342FAD903
:10E50C0011685018A0420BD1206801445018834266
:10E51C001160E0D118685B68084410605360DAE75A
:10E52C0002D90C232B60D6E7206821188B4201BF3F
:10E53C0019685B680918216063605460CBE738BDCB
:10E54C00A018002070B50F4E0C463168054611B965
:10E55C0000F0A8FB30602146284600F0A3FB431CCA
:10E56C0003D14FF0FF34204670BDC41C24F00304CB
:10E57C00A042F8D0211A284600F094FB0130F2D1C9
:10E58C00EFE700BF9C1800202DE9F843CD1C25F0C7
:10E59C00030508350C2D38BF0C25002D064601DB74
:10E5AC00A94204D90C2333600020BDE8F883DFF8BE
:10E5BC00D48000F069F8D8F800301C4644BB2946DA
:10E5CC003046FFF7BFFF431C044658D1D8F8004033
:10E5DC002746002F43D1002C4BD0236839463046B8
:10E5EC0004EB030900F05EFB814542D12168304603
:10E5FC006D1A2946FFF7A6FF01303AD023682B4449
:10E60C002360D8F800305A6862BBC8F800700FE07D
:10E61C002268521B20D40B2A17D96119A3422560FA
:10E62C0018BF5960636808BFC8F8001062514B608E
:10E63C00304600F02FF804F10B00231D20F00700EA
:10E64C00C21A1CBF1B1AA350AFE76268A3420CBFCF
:10E65C00C8F800205A60EBE723466468AEE73C46F6
:10E66C007F68B6E71A465B68A342FBD10023536070
:10E67C00DEE70C233046336000F00CF894E70560BD
:10E68C00D6E700BFA01800200148FFF711BF00BF5C
:10E69C00981800200148FFF70CBF00BF9818002005
:10E6AC002DE9F0471F468E688246BE420C469046C6
:10E6BC000B682DD8B1F90C2012F4906F26D0656937
:10E6CC00096905EB4505A3EB010905EBD5757B1C29
:10E6DC004B446D109D4238BF1D46530527D5294626
:10E6EC00FFF752FF064660B34A46216900F0F8FA7C
:10E6FC00A38923F4906343F08003A38126614E44E5
:10E70C0026603E466561A5EB0905A560BE4200D9B1
:10E71C003E4632464146206800F0AAFA0020A36823
:10E72C009B1BA360236833442360BDE8F0872A4613
:10E73C0000F0E4FA06460028E0D150462169FFF7C4
:10E74C00B9FE0C23CAF80030A3894FF0FF3043F018
:10E75C004003A381E9E700002DE9F04F98468B892F
:10E76C0007461B060D4614469DB010D50B6973B9B0
:10E77C004021FFF709FF2860286130B90C233B606A
:10E78C004FF0FF301DB0BDE8F08F40236B610023CC
:10E79C00099320238DF8293030234FF00109CDF84F
:10E7AC000C80DFF898818DF82A3023469A4613F8AE
:10E7BC00012B0AB1252AF9D1BAEB040B0BD05B461D
:10E7CC00224629463846FFF76BFF013000F0A78040
:10E7DC00099A5A4409929AF80030002B00F09F8055
:10E7EC0000234FF0FF32CDE905230AF1010A04930F
:10E7FC0007938DF853301A935446052214F8011BD5
:10E80C004E4800F05FFA049AD8B9D00644BF2023D2
:10E81C008DF85330110744BF2B238DF853309AF8E1
:10E82C0000302A2B15D0544600204FF00A0C079AC2
:10E83C00214611F8013B303B092B4BD9B0B1079263
:10E84C0014E0A0EB080309FA03F31343A246049364
:10E85C00D2E7039B191D1B680391002BBBBF5B42C6
:10E86C0042F0020207930793B8BF049223782E2B31
:10E87C000AD163782A2B32D1039B02341A1D1B68F0
:10E88C00039243EAE3730593DFF8B4A003225046E6
:10E89C00217800F017FA38B14022049BA0EB0A0053
:10E8AC00824013430134049314F8011B06222548BB
:10E8BC008DF8281000F006FA002836D0224B1BBB2E
:10E8CC00039B073323F0070308330393099B33445B
:10E8DC0009936AE70C4601200CFB0232A8E70023DF
:10E8EC004FF00A0C194601340593204610F8012B01
:10E8FC00303A092A03D9002BC6D00591C4E7044647
:10E90C0001230CFB0121F0E703AB00932A463846A8
:10E91C000E4B04A9AFF30080421C0646D6D1AB893E
:10E92C005B063FF52DAF09982CE703AB00932A4605
:10E93C003846064B04A900F07DF8EDE742F50008D7
:10E94C0048F500084CF5000800000000ADE6000892
:10E95C002DE9F047164698468A680B69074693429C
:10E96C00B8BF1346336091F843200C46DDF8209075
:10E97C000AB1013333602368990642BF336802330E
:10E98C003360256815F0060506D104F1190AE36811
:10E99C0032689B1AAB422BDC94F843302268003B64
:10E9AC0018BF0123920630D44146384604F1430285
:10E9BC00C847013023D02368226903F00603042BD7
:10E9CC0014BF002533684FF0000608BFE56804F15A
:10E9DC001A0408BFED1A54F8123C08BF25EAE57575
:10E9EC009342C4BF9B1AED18B5421AD1002008E01F
:10E9FC000123524641463846C847013003D14FF0F7
:10EA0C00FF30BDE8F0870135C1E73020E11881F80F
:10EA1C0043005A1C94F845102244023382F84310E8
:10EA2C00C2E70123224641463846C8470130E6D0AA
:10EA3C000136D9E72DE9FF470F7E9146782F8046A6
:10EA4C000C469A460C9E01F1430207D8622F0AD855
:10EA5C00002F00F0D180582F00F0B88004F142064E
:10EA6C0084F842703AE0A7F16303152BF6D801A1A4
:10EA7C0051F823F0D9EA0008EDEA000869EA000829
:10EA8C0069EA000869EA000869EA0008EDEA00088A
:10EA9C0069EA000869EA000869EA000869EA0008FE
:10EAAC00EBEB000817EB0008A5EB000869EA00087F
:10EABC0069EA00080DEC000869EA000817EB000889
:10EACC0069EA000869EA0008ADEB000833681A1D12
:10EADC001B68326004F1420684F8423001239CE04A
:10EAEC0033682068191D3160060601D51D6803E0E6
:10EAFC004506FBD5B3F90050002D03DA2D236D42EA
:10EB0C0084F843300A23584811E02168336808061A
:10EB1C0053F8045B02D4490648BFADB26F2F336083
:10EB2C0014BF0A2308235048002184F84310666858
:10EB3C00002EA66005DB21682E4321F00401216024
:10EB4C004BD01646B5FBF3F103FB1157C75D06F826
:10EB5C00017D2F46BB420D46F4D9082B0BD12368FF
:10EB6C00DF0708D5236961689942DEBF302306F8B8
:10EB7C00013C06F1FF36921B22614B462146404672
:10EB8C00CDF800A003AAFFF7E3FE01304AD14FF005
:10EB9C00FF3004B0BDE8F087236843F02003236006
:10EBAC007827324884F84570236831681F0651F87D
:10EBBC00045B02D45F0648BFADB23160D90744BFD5
:10EBCC0043F0200323601DB11023ADE72648E9E78D
:10EBDC00236823F020032360F6E71646BDE733686D
:10EBEC002568181D616930602E061B6801D51960F7
:10EBFC0002E06806FBD51980002316462361BCE7AA
:10EC0C00336800211A1D32601E686268304600F0BD
:10EC1C0059F808B1801B606063682361002384F895
:10EC2C004330AAE73246494640462369D047013073
:10EC3C00ADD023689B0713D4E068039B9842B8BF00
:10EC4C001846A6E70123324649464046D0470130D4
:10EC5C009DD00135E36803995B1AAB42F2DCEBE71C
:10EC6C00002504F11906F5E753F5000864F50008D2
:10EC7C00884210B501EB020402D98442234607D81E
:10EC8C00431EA14208D011F8012B03F8012FF8E71D
:10EC9C00014602448A4200D110BD13F8014D02F81E
:10ECAC00014DF7E738B50023054D044608462B60A7
:10ECBC00F6F78EF9431C02D12B6803B1236038BDE3
:10ECCC0094180020034610B5C9B20244934218466A
:10ECDC0001D1002003E0047801338C42F6D110BD41
:10ECEC000A44914200F1FF3300D1704710B511F87E
:10ECFC00014B914203F8014FF9D110BD2DE9F041C0
:10ED0C00074614460D4621B91146BDE8F041FFF700
:10ED1C003BBC2AB9FFF7CEFB25462846BDE8F0815F
:10ED2C0000F01AF88442064602D8B4EB500FF4D81F
:10ED3C0021463846FFF728FC804608B94546ECE7E3
:10ED4C00B4422246294628BF3246FFF7C9FF29465E
:10ED5C003846FFF7AFFBF1E751F8043C181F002BC6
:10ED6C00BCBF0B58C0187047F8B500BFF8BC08BC46
:10ED7C009E467047F8B500BFF8BC08BC9E4670476D
:10ED8C00696E666F0A0000000A70776D2025642595
:10ED9C0064256425642564256425642564000000CD
:10EDAC000A3078256C78203078256C7820307825DE
:10EDBC006C78203078256C78203078256C78203071
:10EDCC0078256C78203078256C78203078256C7814
:10EDDC00000000000A503D30782578206368343DEF
:10EDEC0025303564206368353D25303564206368F3
:10EDFC00363D25303564206368373D253035642039
:10EE0C006368383D25303564000000000A73744394
:10EE1C0069636C6F3D2530356420737450756C7369
:10EE2C00616E74693D253035640000000A49443038
:10EE3C0030303030300000000A62307C310000008D
:10EE4C000A3F6D6E73767676767620733D667C62BD
:10EE5C00000000000A3F6D6E737676767676203071
:10EE6C00303030303E3D76767676763C3D393939E9
:10EE7C00393900000A3F6D6E7376767676762031DE
:10EE8C003E3D6D3C3D3400000A3F6D6E73767676E8
:10EE9C00767600000A6565203078253032783D3072
:10EEAC0078253034780000000A656520726561644D
:10EEBC00206572726F722025640000000A3F657233
:10EECC006161206865782076616C7565730000005F
:10EEDC000A3F6572616100000A646F6E65203078CC
:10EEEC00253032783D307825303478000A6565203D
:10EEFC007772697465206572726F722025640000E8
:10EF0C000A3F65776161767676762068657820763B
:10EF1C00616C7565730000000A3F6577616120685C
:10EF2C0065782076616C7565730000000A3F657723
:10EF3C0061617676767600000A3078253032783D3D
:10EF4C00253564200000000072646572722025640F
:10EF5C00200000000A0000000A3F65640000000069
:10EF6C000A3F6578000000000A6D3170776D6170A2
:10EF7C003D2564206D3170776D63683D2564206D8F
:10EF8C003270776D61703D2564206D3270776D63E2
:10EF9C00683D2564206D3370776D61703D2564206C
:10EFAC006D3370776D63683D2564206D3470776DBB
:10EFBC0061703D2564206D3470776D63683D256408
:10EFCC00000000000A6D3154696D656F75744D61F8
:10EFDC006E3D2564206D3254696D656F75744D619D
:10EFEC006E3D2564206D3354696D656F75744D618C
:10EFFC006E3D2564206D3454696D656F75744D617B
:10F00C006E3D2564200000000A7472616D703D2510
:10F01C0064207472616D706D616E3D25640000003A
:10F02C000A6D3170776D4D616E3D2564206D3270C7
:10F03C00776D4D616E3D2564206D3370776D4D613C
:10F04C006E3D2564206D3470776D4D616E3D256489
:10F05C00000000000A61704D3173746172743D25BB
:10F06C00642061704D3173746F703D25642063684A
:10F07C004D3173746172743D25642063684D317336
:10F08C00746F703D256400000A61704D32737461B9
:10F09C0072743D25642061704D3273746F703D2520
:10F0AC00642063684D3273746172743D256420630F
:10F0BC00684D3273746F703D256400000A61704DA9
:10F0CC003373746172743D25642061704D337374B5
:10F0DC006F703D25642063684D3373746172743DA9
:10F0EC0025642063684D3373746F703D2564000094
:10F0FC000A61704D3473746172743D2564206170C3
:10F10C004D3473746F703D25642063684D34737493
:10F11C006172743D25642063684D3473746F703D67
:10F12C00256400000A3F6576000000000A3F657206
:10F13C007C777C647C787C76000000000A3F6572EA
:10F14C006161207C206577616176767676000000BF
:10F15C000A3F00000A70756C73616E74693D255826
:10F16C00000000000A737470756C73616E74693DF5
:10F17C00255800000A73744369636C6F3D25640065
:10F18C000A646F6E652025643D2564000A65652060
:10F19C007772697465206572726F72202564000045
:10F1AC004C6F616445450A000A6D3170776D617072
:10F1BC003D2564206D3170776D63683D2564206D4D
:10F1CC003270776D61703D2564206D3270776D63A0
:10F1DC00683D2564206D3370776D61703D2564202A
:10F1EC006D3370776D63683D2564206D3470776D79
:10F1FC0061703D2564206D3470776D63683D2564C6
:10F20C00000000000A6D3154696D656F75744D61B5
:10F21C006E3D2564206D3254696D656F75744D615A
:10F22C006E3D2564206D3354696D656F75744D6149
:10F23C006E3D2564206D3454696D656F75744D6138
:10F24C006E3D2564200000000A7472616D703D25CE
:10F25C0064207472616D706D616E3D2564000000F8
:10F26C000A6D3170776D4D616E3D2564206D327085
:10F27C00776D4D616E3D2564206D3370776D4D61FA
:10F28C006E3D2564206D3470776D4D616E3D256447
:10F29C00000000000A61704D3173746172743D2579
:10F2AC00642061704D3173746F703D256420636808
:10F2BC004D3173746172743D25642063684D3173F4
:10F2CC00746F703D256400000A61704D3273746177
:10F2DC0072743D25642061704D3273746F703D25DE
:10F2EC00642063684D3273746172743D25642063CD
:10F2FC00684D3273746F703D256400000A61704D67
:10F30C003373746172743D25642061704D33737472
:10F31C006F703D25642063684D3373746172743D66
:10F32C0025642063684D3373746F703D2564000051
:10F33C000A61704D3473746172743D256420617080
:10F34C004D3473746F703D25642063684D34737451
:10F35C006172743D25642063684D3473746F703D25
:10F36C00256400000A6D3161703D256400000000C9
:10F37C000A6D3261703D2564000000000A6D336136
:10F38C00703D2564000000000A6D3461703D2564F9
:10F39C00000000000A6D3163683D25640000000028
:10F3AC000A6D3263683D2564000000000A6D33630A
:10F3BC00683D2564000000000A6D3463683D2564D7
:10F3CC000000000053544D3332205669727475613D
:10F3DC006C20436F6D506F727400000053544D6974
:10F3EC0063726F656C656374726F6E696373000032
:10F3FC0043444320436F6E666967000043444320D7
:10F40C00496E7465726661636500000028003C00FB
:10F41C004600460023002800280028001400140091
:10F42C0014001400E600640082002C0101001B0093
:10F43C000A001E000100010000000000F40114008D
:10F44C003C0046002800280032000A003601C201A8
:10F45C001E0036015401AE011E00AE010A0040012F
:10F46C008C00B801140018012800B80101001B0021
:10F47C000A001E00010001000000000000006400F2
:10F48C003C00460028002800320005000100020064
:10F49C0003000400050006000700080009000A002C
:10F4AC000B000C000D000E000F00100011001200DC
:10F4BC0013001400150016001700180019001A008C
:10F4CC001B001C001D001E001F002000210022003C
:10F4DC0023002400250026002700280029002A00EC
:10F4EC002B002C002D002E002F003000310032009C
:10F4FC0033003400350036003700380039003A004C
:10F50C003B003C003D003E003F004000000000007E
:10F51C0000000000010203040607080900000000B7
:10F52C000102030402030405060708090A0B0C0D6B
:10F53C000E0F10100102232D302B2000686C4C0094
:10F54C0065666745464700303132333435363738D7
:10F55C003941424344454600303132333435363735
:0CF56C00383961626364656600000000CD
:08F57800D40BFF7F010000002D
:04F58000310100084D
:04F584000D0100086D
:10F5880000F80008C8C8640404040404040404005F
:10F5980000127A0010000000010000000A060002B4
:10F5A800000000400100000009C30008FDC3000876
:10F5B8006BC4000800000000ADC60008B1C5000813
:10F5C80057C600080000000000000000000000000E
:10F5D8001DC70008FDC600083DC700085DC7000834
:10F5E80009024300020100C03209040000010202BE
:10F5F8000100052400100105240100010424020271
:10F60800052406000107058203080010090401000B
:10F61800020A000000070501020002000705810236
:10F628000002000009024300020100C03209040080
:10F638000001020201000524001001052401000157
:10F6480004240202052406000107058203080010AD
:10F6580009040100020A0000000705010240000039
:10F66800070581024000000009074300020104C0A9
:10F6780032090400000102020100052400100105FE
:10F688002401000104240202052406000107058262
:10F698000308001009040100020A00000007050120
:10F6A80002400000070581024000000029DB000835
:10F6B80051DB000861DB00081DDC0008A5DC000840
:10F6C800C9DC000829DD0008EDDC000851DD000870
:10F6D80075DD0008B1DD00081201000202020040D9
:10F6E80083044057000201020301000004030904D7
:10F6F8001A030000000000000000000000000000E5
:10F708000000000000000000000000009001002040
:10F71800000000005C170020C41700202C180020EF
:10F7280000000000000000000000000000000000D1
:10F7380000000000000000000000000000000000C1
:10F7480000000000000000000000000000000000B1
:0CF75800000000000000000000000000A5
:04000005080050554A
:00000001FF
